:100000000C94D2030C94EF030C940B2E0C94EF037E
:100010000C94EF030C94EF030C94EF030C94EF0398
:100020000C94EF030C9492450C94EF030C94EF03A3
:100030000C94EF030C94EF030C94EF030C94EF0378
:100040000C94EF030C94EF030C94EF030C94EF0368
:100050000C94EF030C943F540C94EF030C94EF03B7
:100060000C94EF030C94EF030C94EF030C94EF0348
:100070000C94EF030C94EF030C94EF030C94EF0338
:100080000C94EF030C94EF030C94EF030C94EF0328
:100090000C94EF031747624721484748BF48E3489D
:1000A00008490C491C49A751A751A751A751A7516D
:1000B000A751A751A751A751A751A751A751A75180
:1000C000A751A751A751A751A751A751A751A75170
:1000D000A751AF492C494849CE49DE49524B9C4B68
:1000E000294C6B4CA74C1A4DA751A751A751A751AA
:1000F000A751A751A751A751A751A751A751A75140
:10010000A751A751A751A751A751A751A751A7512F
:10011000A7510D4A524A884DA14DD14DE84DA751E6
:10012000A751A751A751A751A751A751A751A7510F
:10013000A751824ADA4AF54D754EF44E364FE950D2
:10014000F850AD4FC14F075119512C51A7513D5196
:10015000BF4AE74A0F4B71518C51774F924FD54FA1
:1001600009502C5078509350BE50CE03C103B303B6
:10017000A30390037A036103470329030803E602FC
:10018000C2029E0276024F02280203026C01B801ED
:1001900096017501560139011F010601EF00DA00D1
:1001A000B5008200A5009600000043414E203100BA
:1001B00000000000000000000043414E203200001B
:1001C000000000000000000043414E20330000000A
:1001D0000000000000000043414E203400000000F9
:1001E00000000000000043414E20350000000000E8
:1001F000000000000043414E2036000000000000D7
:100200000000000043414E203700000000000000C5
:1002100000000043414E20380000000000000000B4
:10022000000043414E2039000000000000000000A3
:100230000043414E2031300000000000000000006B
:1002400043414E2031310000000000000000004317
:10025000414E203132000000000000000000434108
:100260004E20313300000000000000000043414EEA
:1002700020313400000000000000000043414E2007
:10028000313500000000000000000043414E2031E5
:100290003600000000000000000043414E203137CE
:1002A00000000000000000000043414E20313800F3
:1002B000000000000000000043414E2031390000E2
:1002C0000000000000000043414E203230000000DA
:1002D00000000000000043414E20323100000000C9
:1002E000000000000043414E2032320000000000B8
:1002F0000000000043414E203233000000000000A7
:1003000000000043414E2032340000000000000095
:10031000000043414E203235000000000000000084
:100320000043414E20323600000000000000000073
:1003300043414E203237000000000000000000431F
:10034000414E203238000000000000000000434110
:100350004E20323900000000000000000043414EF2
:1003600020333000000000000000000043414E2018
:10037000333100000000000000000043414E2033F4
:1003800032000000000000000000466C617368202D
:10039000310000000000000000466C6173682032EC
:1003A0000000000000000000466C6173682033000C
:1003B00000000000000000466C61736820340000FB
:1003C000000000000000466C6173682035000000EA
:1003D00000000000005357495443482031000000FA
:1003E00000000000535749544348203200000000E9
:1003F00000000053574954434820330000000000D8
:1004000000005357495443482034000000000000C6
:1004100000535749544348203500000000000000B5
:100420005357495443482036000000000000005351
:10043000574954434820370000000000000053573C
:100440004954434820380000000000000053574939
:10045000544348203900000000000000535749541D
:1004600043482031300000000000005357495443F6
:10047000482031310000000000004348414E4E4505
:100480004C20310000000000004348414E4E454CD6
:1004900020320000000000004348414E4E454C20F1
:1004A000330000000000004348414E4E454C2034CC
:1004B0000000000000004348414E4E454C203500EE
:1004C00000000000004348414E4E454C20360000DD
:1004D000000000004348414E4E454C2037000000CC
:1004E0000000004348414E4E454C203800000000BB
:1004F00000004348414E4E454C20390000000000AA
:10050000004348414E4E454C203130000000000071
:100510004348414E4E454C2031310000000000431D
:1005200048414E4E454C2031320000000000434807
:10053000414E4E454C2031330000000000434841FD
:100540004E4E454C20313400000000004348414EDF
:100550004E454C20313500000000004348414E4ECE
:10056000454C20313600000000004348414E4E45C6
:100570004C20313700000000004348414E4E454CAE
:1005800020313800000000004348414E4E454C20C9
:10059000313900000000004348414E4E454C2032A6
:1005A0003000000000004348414E4E454C2032319F
:1005B00000000000004348414E4E454C20323200BE
:1005C000000000004348414E4E454C2032330000AD
:1005D0000000004348414E4E454C2032340000009C
:1005E00000004348414E4E454C203235000000008B
:1005F000004348414E4E454C20323600000000007A
:100600004348414E4E454C20323700000000004325
:1006100048414E4E454C203238000000000043480F
:10062000414E4E454C203239000000000043484105
:100630004E4E454C20333000000000004348414EF0
:100640004E454C20333100000000004348414E4EDF
:10065000454C20333200000000004348414E4E45D7
:100660004C20333300000000004348414E4E454CBF
:1006700020333400000000005649525455414C20AC
:10068000310000000000005649525455414C2032C0
:100690000000000000005649525455414C203300E0
:1006A00000000000005649525455414C20340000CF
:1006B000000000005649525455414C2035000000BE
:1006C0000000005649525455414C203600000000AD
:1006D00000005649525455414C203700000000009C
:1006E000005649525455414C20380000000000008B
:1006F0005649525455414C20390000000000005624
:1007000049525455414C20313000000000005649F8
:10071000525455414C2031310000000000564952DE
:100720005455414C203132000000000056495254CB
:1007300055414C20313300000000005649525455B9
:10074000414C2031340000000000564952545541BC
:100750004C20313500000000005649525455414CA0
:1007600020313600000000005649525455414C20BB
:10077000313700000000005649525455414C203199
:100780003800000000005649525455414C20313980
:1007900000000000005649525455414C20323000B0
:1007A0000000000011241FBECFEFD0E1DEBFCDBF9F
:1007B00011E0A0E0B1E0EAECFCEC00E00BBF02C00D
:1007C00007900D92AA3AB107D9F71EE0AAEAB1E064
:1007D00001C01D92A43FB107E1F70C94FF370C94C0
:1007E0000000282F277099279695879596958795CD
:1007F0009695879533272330310529F1243031052B
:100800004CF421303105B9F022303105C4F4232BEA
:1008100071F02CC025303105F1F025303105BCF0E8
:1008200026303105E1F027303105E9F01FC0A098EE
:10083000A198A2981BC0A09AA198A29817C0A098AE
:10084000A19AA29813C0A09AA19AA2980FC0A098AA
:10085000A198A29A0BC0A09AA198A29A07C0A098AA
:10086000A19AA29A03C0A09AA19AA29A80628093A8
:100870007C0080917A00806480937A0080917A0075
:1008800084FFFCCF80917A00806180937A00209170
:100890007800809179009927880F991F880F991FF8
:1008A0002295269526952370820F911D0895282F55
:1008B000277099279695879596958795969587950C
:1008C00033272330310529F1243031054CF4213010
:1008D0003105B9F022303105C4F4232B71F02CC05E
:1008E00025303105F1F025303105BCF026303105D9
:1008F000E1F027303105E9F01FC0A098A198A29837
:100900001BC0A09AA198A29817C0A098A19AA298DB
:1009100013C0A09AA19AA2980FC0A098A198A29AD9
:100920000BC0A09AA198A29A07C0A098A19AA29AD7
:1009300003C0A09AA19AA29A806280937C008091C1
:100940007A00806480937A0080917A0084FFFCCFE3
:1009500080917A00806180937A0080917900992754
:10096000089540E050E0FC01029625913491621711
:10097000730760F44B5F5F4FFC0102962591349141
:100980006217730718F446395105A4F3CA01089594
:10099000FC01809100018130B1F410920001F093CC
:1009A000B301E093B201F093B101E093B001F09391
:1009B000AF01E093AE01F093AD01E093AC01F09391
:1009C000AB01E093AA016091B0017091B101709305
:1009D000B3016093B2014091AE015091AF015093C9
:1009E000B1014093B0012091AC013091AD01309341
:1009F000AF012093AE018091AA019091AB01909339
:100A0000AD018093AC01F093AB01E093AA01E80F34
:100A1000F91FE20FF31FE40FF51FCF01860F971F99
:100A200065E070E00E94AC65CB01089580E10E9412
:100A3000F1030E94C804BC018AE691E00E94B1045F
:100A40009927089583E10E9457042091720E33275D
:100A5000829FA001839F500D929F500D11249A01F7
:100A6000220F232F221F330B31952F3F310519F011
:100A700010F04FEF01C0422F8091B401882339F468
:100A80004093B6014093B5014093B40118C08091E2
:100A9000B601280F311D9091B501290F311D8091AC
:100AA000B401280F311D9093B6018093B501409396
:100AB000B401C9019695879596958795482F842FFF
:100AC0009927089580E280937C0087E880937A00DC
:100AD000989A999A9A9AA098A198A298089590E0C5
:100AE000892F8295807F8093ED001092EE00109206
:100AF000EF001092F0001092F1001092F2001092AC
:100B0000F3001092F4001092F5001092F60010928B
:100B1000F70080E01092FA008F5F8830D8F39F5F73
:100B20009F30F0F208953091ED0090E020EC892F95
:100B30008295807F8093ED008091EF00822329F4DD
:100B40003093ED00892F992708959F5F9F3078F3A8
:100B50003093ED008FEF90E008958091EE0086FFD6
:100B600003C080E090E008958091EE0085FF03C00F
:100B700081E090E008958091EF00807C19F48FEF80
:100B800090E0089582E090E00895BC0140E08091FB
:100B9000EF0099278F709070892B89F0FB01E40F8B
:100BA000F11D8091FA0080834F5F242F33278091BD
:100BB000EF0099278F709070281739077CF30895FC
:100BC00089E79DE00E944C356FE17EE080E00E9465
:100BD000893567ED7DE081E00E94893561E97DE03E
:100BE00082E00E94893581E08093B7018091790D80
:100BF000813061F480917A0D90917B0D6AE070E014
:100C00000E94AC657093770D6093760D8091200EF5
:100C1000813061F48091210E9091220E6AE070E0A3
:100C20000E94AC657093720D6093710D8091D80D28
:100C3000813061F48091D90D9091DA0D6AE070E015
:100C40000E94AC657093750D6093740D8091920D48
:100C5000813061F48091930D9091940D6AE070E081
:100C60000E94AC6570931E0E60931D0E0895CF9385
:100C7000DF93CDB7DEB7CE55D0400FB6F894DEBFC8
:100C80000FBECDBF19828CE0888F84E690E09B83F5
:100C90008A831D821C821E821F82188619861A86EC
:100CA0001B8689819E01245F3F4FF901E80FF11DEA
:100CB00010828F5F8C30C8F3CE0101960E943C35C4
:100CC000A895198E1A8E84E690E09C8F8B8F1E8ECD
:100CD0001D8E898D9E012F5F3F4FF901E80FF11D99
:100CE000168E8F5F8232C8F3CE0149960E945C3522
:100CF000A89581E0898F1A8E84E690E09C8F8B8F77
:100D00001E8E1D8E8A8D9E012F5F3F4FF901E80FC9
:100D1000F11D168E8F5F8232C8F3CE0149960E9474
:100D20005C35A89582E0898F1A8E84E690E09C8FCE
:100D30008B8F1E8E1D8E8A8D9E012F5F3F4FF90176
:100D4000E80FF11D168E8F5F8034C8F3CE014996EF
:100D50000E945C35C25ADF4F0FB6F894DEBF0FBE5B
:100D6000CDBFDF91CF91089599278832910509F47D
:100D700040C08932910594F48532910559F186324B
:100D8000910534F483329105D9F08497F1F04FC086
:100D90008632910521F1879739F149C08B3291054F
:100DA000B9F18C32910534F48932910539F18A9781
:100DB00051F13DC08C32910581F18D9799F137C089
:100DC00080EC0E945C449927089581EC0E945C4469
:100DD0009927089582EC0E945C449927089581ED3B
:100DE0000E945C449927089584EC0E945C449927F2
:100DF000089585EC0E945C449927089586EC0E9432
:100E00005C449927089587EC0E945C4499270895D3
:100E100083EC0E945C449927089582ED0E945C4413
:100E20009927089583ED0E945C449927089580E0F6
:100E300090E00895EF92FF920F931F93CF93DF936B
:100E4000CDB7DEB765970FB6F894DEBF0FBECDBF46
:100E500080916F0E9091700E01978F5F974008F010
:100E60002BC490916E0E992309F426C48091730DC2
:100E70008F5F8093730D891708F41EC41092730D51
:100E800088E08D8300E0CE010696FC01E00FF11DA5
:100E900010820F5F0830C8F38091780D9927853054
:100EA000910509F4BDC2863091059CF4823091050C
:100EB00009F408C28330910524F4019709F4C8C1EC
:100EC0001EC08330910509F437C2049709F46EC23D
:100ED00016C08830910509F463C38930910544F444
:100EE0008630910509F4D2C2079709F405C307C0FB
:100EF0008930910509F484C30A9709F4BAC3809133
:100F00006F0E9091700EAA27BB2789839A83AB83BB
:100F1000BC8301E00093780D10E080EC0E945C44FB
:100F20008111102F81EC0E945C448111126082ECCF
:100F30000E945C448111146081ED0E945C44811127
:100F4000186084EC0E945C448111106185EC0E9461
:100F50005C448111106286EC0E945C448111106433
:100F600087EC0E945C44811110681E8310E083ECC2
:100F70000E945C44811111E082ED0E945C44811169
:100F8000126083ED0E945C44811114601F8310E0A5
:100F900081E090E00E947557892B09F011E082E012
:100FA00090E00E947557892B09F0126083E090E071
:100FB0000E947557892B09F0146084E090E00E942C
:100FC0007557892B09F0186085E090E00E947557ED
:100FD000892B09F0106186E090E00E947557892BFB
:100FE00009F0106287E090E00E947557892B09F0A4
:100FF000106488E090E00E947557892B09F0106812
:10100000188710E089E090E00E947557892B09F05D
:1010100011E08AE090E00E947557892B09F0126078
:101020008BE090E00E947557892B09F014608CE0EA
:1010300090E00E947557892B09F018608DE090E0D0
:101040000E947557892B09F010618EE090E00E9494
:101050007557892B09F010628FE090E00E94755758
:10106000892B09F0106480E190E00E947557892B6C
:1010700009F01068198710E081E090E00E944911A2
:10108000892B09F011E082E090E00E944911892B40
:1010900009F0126083E090E00E944911892B09F069
:1010A000146084E090E00E944911892B09F01860D7
:1010B00085E090E00E944911892B09F0106186E0DB
:1010C00090E00E944911892B09F0106287E090E0BE
:1010D0000E944911892B09F0106488E090E00E9479
:1010E0004911892B09F010681A8710E089E090E017
:1010F0000E944911892B09F011E08AE090E00E94DA
:101100004911892B09F012608BE090E00E9449118F
:10111000892B09F014608CE090E00E944911892B22
:1011200009F018608DE090E00E944911892B09F0C8
:1011300010618EE090E00E944911892B09F0106245
:101140008FE090E00E944911892B09F0106480E142
:1011500090E00E944911892B09F010681B8710E06C
:1011600081E190E00E944911892B09F011E082E1B0
:1011700090E00E944911892B09F0126083E190E010
:101180000E944911892B09F0146084E190E00E94CB
:101190004911892B09F0186085E190E00E944911FE
:1011A000892B09F0106186E190E00E944911892B9A
:1011B00009F0106287E190E00E944911892B09F043
:1011C000106488E190E00E944911892B09F01068B1
:1011D0001C8710E089E190E00E944911892B09F0F9
:1011E00011E08AE190E00E944911892B09F0126018
:1011F0008BE190E00E944911892B09F014608CE189
:1012000090E00E944911892B09F018608DE190E06F
:101210000E944911892B09F010618EE190E00E9433
:101220004911892B09F010628FE190E00E94491169
:10123000892B09F0106480E290E00E944911892B0B
:1012400009F010681D87CE0101960E94EB4134C25F
:1012500080916F0E9091700E0196AA27BB2789830B
:101260009A83AB83BC8382E08093780D00E00F2EDD
:10127000F6E0EF2EFF24F02DEC0EFD1E802F8F5F89
:101280000E94152CDC01FC01878580FF02C014E65A
:101290000DC0FD01878583FF02C015E607C0FD0173
:1012A0008181803F11F411E001C010E0F701E00FEF
:1012B000F11D10830F5F083008F3CE0101960E94E4
:1012C000EB41FAC180916F0E9091700E0296AA27A1
:1012D000BB2789839A83AB83BC8383E08093780D9B
:1012E00000E00F2EF6E0EF2EFF24F02DEC0EFD1E99
:1012F000802F875F0E94152CDC01FC01878580FF11
:1013000002C014E60DC0FD01878583FF02C015E60B
:1013100007C0FD018181803F11F411E001C010E0A0
:10132000F701E00FF11D10830F5F083008F3CE01C5
:1013300001960E94EB41C0C180916F0E9091700E9A
:101340000396AA27BB2789839A83AB83BC8384E057
:101350008093780D00E00F2EF6E0EF2EFF24F02DA5
:10136000EC0EFD1E802F8F5E0E94152CDC01FC010F
:10137000878580FF02C014E60DC0FD01878583FFCD
:1013800002C015E607C0FD018181803F11F411E024
:1013900001C010E0F701E00FF11D10830F5F08306E
:1013A00008F3CE0101960E94EB4186C180916F0E39
:1013B0009091700E0496AA27BB2789839A83AB83EA
:1013C000BC8385E08093780D00E00F2EF6E0EF2ED1
:1013D000FF24F02DEC0EFD1E802F875E0E94152C41
:1013E000DC01FC01878580FF02C014E60DC0FD0111
:1013F000878583FF02C015E607C0FD018181803F1C
:1014000011F411E001C010E0F701E00FF11D1083AD
:101410000F5F083008F3CE0101960E94EB414CC1EA
:1014200080916F0E9091700E0596AA27BB27898335
:101430009A83AB83BC8386E08093780D00E00F2E07
:10144000F6E0EF2EFF24F02DEC0EFD1E802F8F5FB7
:101450000E94152CFC018181803F61F49701200FCF
:10146000311D8089918965E070E00E94AC65F901C9
:10147000608304C0F701E00FF11D10820F5F083098
:1014800028F3CE0101960E94EB4116C180916F0EA8
:101490009091700E0696AA27BB2789839A83AB8307
:1014A000BC8387E08093780D00E00F2EF6E0EF2EEE
:1014B000FF24F02DEC0EFD1E802F875F0E94152C5F
:1014C000FC018181803F61F49701200F311D8089EB
:1014D000918965E070E00E94AC65F901608304C009
:1014E000F701E00FF11D10820F5F083028F3CE01E5
:1014F00001960E94EB41E0C080916F0E9091700EBA
:101500000796AA27BB2789839A83AB83BC8388E08D
:101510008093780D00E00F2EF6E0EF2EFF24F02DE3
:10152000EC0EFD1E802F8F5E0E94152CFC01818128
:10153000803F61F49701200F311D8089918965E01A
:1015400070E00E94AC65F901608304C0F701E00F10
:10155000F11D10820F5F023028F30830E0F40F2EE7
:10156000F6E0EF2EFF24F02DEC0EFD1E16E0802F8E
:101570008F5E0E94152CFC018181803F29F4F701C8
:10158000E00FF11D108304C0F701E00FF11D108280
:101590000F5F083060F3CE0101960E94EB418CC0D2
:1015A00080916F0E9091700E0896AA27BB278983B1
:1015B0009A83AB83BC8389E08093780D00E00F2E83
:1015C000F6E0EF2EFF24F02DEC0EFD1E16E0802F2E
:1015D000875E0E94152CFC018181803F29F4F70170
:1015E000E00FF11D108304C0F701E00FF11D108220
:1015F0000F5F083060F3CE0101960E94EB415CC0A2
:1016000080916F0E9091700E0996AA27BB2789834F
:101610009A83AB83BC838AE08093780DCE010E96CB
:101620000E94FB2B8889682F7727CB01880F991F91
:10163000880F991F880F991F860F971F680F791FB2
:10164000872F99278E836F838989682F772784E670
:1016500090E0689F9001699F300D789F300D1124B4
:10166000832F992788872987CE0101960E94EB4115
:1016700023C080916F0E9091700E0A96AA27BB2707
:1016800089839A83AB83BC831092780DCE010E962A
:101690000E94FB2B1E821F82188619868E859F85CD
:1016A00064E170E00E94AC65872F99278A876B8779
:1016B000CE0101960E94EB418091760D9091770DBD
:1016C000009709F479C001979093770D8093760D78
:1016D000892B09F071C080917A0D90917B0D6AE0A1
:1016E00070E00E94AC657093770D6093760D8091E9
:1016F0007C0D90917D0DAA27BB2789839A83AB83AC
:10170000BC8388E08D838091B7018E8380917E0DAC
:101710000E949F2C96958795969587958F838091AB
:101720007F0D0E949F2C9695879596958795888723
:101730008091800D0E949F2C969587959695879510
:1017400089878091810D0E949F2C9695879596950B
:1017500087958A878091820D0E949F2C9695879508
:10176000969587958B878091830D0E949F2C9695E7
:101770008795969587958C872091B70189E79DE09D
:10178000FC01E20FF11D82850E949F2C96958795A2
:10179000969587958D878091B701982F9F5F90933D
:1017A000B7018091900D891718F481E08093B701FB
:1017B000CE0101960E94EB418091710D9091720DC6
:1017C000009709F405C101979093720D8093710DF4
:1017D000892B09F0FDC0CE010E960E94FB2B809153
:1017E000210E9091220E6AE070E00E94AC65709329
:1017F000720D6093710D8091230E9091240EAA2793
:10180000BB2789839A83AB83BC8388E08D83EE24D6
:101810000F2EF0E8FF2EF02D0E2D802F9927FC01C2
:10182000E15EF14F1681133238F4812F0E94B52BFF
:10183000882379F0EF280DC01E3238F4812F0E94E2
:10184000B406882331F0EF2804C01E3211F4A499A5
:10185000EF28F6940F5F083000F3EE82EE240F2E8F
:10186000F0E8FF2EF02D0E2D802F9927FC01E15E70
:10187000F14F1685133238F4812F0E94B52B88233F
:1018800079F0EF280DC01E3238F4812F0E94B40683
:10189000882331F0EF2804C01E3211F4A499EF28F8
:1018A000F6940F5F083000F3EF82EE240F2EF0E87D
:1018B000FF2EF02D0E2D802F9927FC01E15EF14FB8
:1018C0001689133238F4812F0E94B52B882379F0C2
:1018D000EF280DC01E3238F4812F0E94B4068823F1
:1018E00031F0EF2804C01E3211F4A499EF28F694C9
:1018F0000F5F083000F3E886EE240F2EF0E8FF2E8D
:10190000F02D0E2D802F9927FC01E15EF14F168DF1
:10191000133238F4812F0E94B52B882379F0EF28F9
:101920000DC01E3238F4812F0E94B406882331F096
:10193000EF2804C01E3211F4A499EF28F6940F5F2B
:10194000083000F3E986EE241091450E133250F46E
:10195000812F0E94B52B882399F00F2EF0E8EF2EEF
:10196000F02D0EC01E3240F4812F0E94B406882351
:1019700039F030E8E32A04C01E3211F4A499EF28AC
:101980001091460E133240F4812F0E94B52B88230C
:1019900089F080E4E82A0EC01E3240F4812F0E94B4
:1019A000B406882339F0E0E4EE2A04C01E3211F4B4
:1019B000A499EF28EA868E859F856AE070E00E94F0
:1019C000AC656B871C861D86CE0101960E94EB419B
:1019D0008091740D9091750D009709F4FCC00197EA
:1019E0009093750D8093740D892B09F0F4C080914C
:1019F000D90D9091DA0D6AE070E00E94AC657093A9
:101A0000750D6093740D8091DB0D9091DC0DAA270C
:101A1000BB2789839A83AB83BC8388E08D83EE24C4
:101A20000F2EF0E8FF2EF02D0E2D802F9927FC01B0
:101A3000E952F24F1681133238F4812F0E94DB2BCA
:101A4000882379F0EF280DC01E3238F4812F0E94D0
:101A5000B406882331F0EF2804C01E3211F4A49993
:101A6000EF28F6940F5F083000F3EE82EE240F2E7D
:101A7000F0E8FF2EF02D0E2D802F9927FC01E95262
:101A8000F24F1685133238F4812F0E94DB2B882306
:101A900079F0EF280DC01E3238F4812F0E94B40671
:101AA000882331F0EF2804C01E3211F4A499EF28E6
:101AB000F6940F5F083000F3EF82EE240F2EF0E86B
:101AC000FF2EF02D0E2D802F9927FC01E952F24FA9
:101AD0001689133238F4812F0E94DB2B882379F08A
:101AE000EF280DC01E3238F4812F0E94B4068823DF
:101AF00031F0EF2804C01E3211F4A499EF28F694B7
:101B00000F5F083000F3E886EE240F2EF0E8FF2E7A
:101B1000F02D0E2D802F9927FC01E952F24F168DE2
:101B2000133238F4812F0E94DB2B882379F0EF28C1
:101B30000DC01E3238F4812F0E94B406882331F084
:101B4000EF2804C01E3211F4A499EF28F6940F5F19
:101B5000083000F3E986EE241091FD0D133250F4A5
:101B6000812F0E94DB2B882399F00F2EF0E8EF2EB7
:101B7000F02D0EC01E3240F4812F0E94B40688233F
:101B800039F0F0E8EF2A04C01E3211F4A499EF28CE
:101B90001091FE0D133240F4812F0E94DB2B88231D
:101BA00089F020E4E22A0EC01E3240F4812F0E9408
:101BB000B406882339F030E4E32A04C01E3211F45D
:101BC000A499EF28EA8688898B871C861D86CE011A
:101BD00001960E94EB4180911D0E90911E0E009780
:101BE00009F45CC1019790931E0E80931D0E892B02
:101BF00009F054C18091930D9091940D6AE070E0CA
:101C00000E94AC6570931E0E60931D0E8091950D21
:101C10009091960DAA27BB2789839A83AB83BC83B7
:101C200088E08D83EE240F2EF0E8FF2EF02D0E2D90
:101C3000802F9927FC01EF56F24F1681133238F4AA
:101C4000812F0E94B52B882379F0EF280DC01E321A
:101C500038F4812F0E94B406882331F0EF2804C0A5
:101C60001E3211F4A499EF28F6940F5F083000F3A8
:101C7000EE82EE240F2EF0E8FF2EF02D0E2D802F99
:101C80009927FC01EF56F24F1685133238F4812F55
:101C90000E94B52B882379F0EF280DC01E3238F44E
:101CA000812F0E94B406882331F0EF2804C01E3231
:101CB00011F4A499EF28F6940F5F083000F3EF8237
:101CC000EE240F2EF0E8FF2EF02D0E2D802F9927F9
:101CD000FC01EF56F24F1689133238F4812F0E941F
:101CE000B52B882379F0EF280DC01E3238F4812FF0
:101CF0000E94B406882331F0EF2804C01E3211F48C
:101D0000A499EF28F6940F5F083000F3E886EE24DC
:101D10000F2EF0E8FF2EF02D0E2D802F9927FC01BD
:101D2000EF56F24F168D133238F4812F0E94B52BE7
:101D3000882379F0EF280DC01E3238F4812F0E94DD
:101D4000B406882331F0EF2804C01E3211F4A499A0
:101D5000EF28F6940F5F083000F3E986EE240F2E8B
:101D6000F0E8FF2EF02D0E2D802F9927FC01EF5665
:101D7000F24F16A1133238F4812F0E94DB2B8823F7
:101D800079F0EF280DC01E3238F4812F0E94B4067E
:101D9000882331F0EF2804C01E3211F4A499EF28F3
:101DA000F6940F5F083000F3EA86EE240F2EF0E879
:101DB000FF2EF02D0E2D802F9927FC01EF56F24FAC
:101DC00016A5133238F4812F0E94DB2B882379F07B
:101DD000EF280DC01E3238F4812F0E94B4068823EC
:101DE00031F0EF2804C01E3211F4A499EF28F694C4
:101DF0000F5F083000F3EB86EE240F2EF0E8FF2E85
:101E0000F02D0E2D802F9927FC01EF56F24F16A9C9
:101E1000133238F4812F0E94DB2B882379F0EF28CE
:101E20000DC01E3238F4812F0E94B406882331F091
:101E3000EF2804C01E3211F4A499EF28F6940F5F26
:101E4000083000F3EC86EE240F2EF0E8FF2EF02D84
:101E50000E2D802F9927FC01E153F24F1081133290
:101E600038F4812F0E94DB2B882379F0EF280DC0F6
:101E70001E3238F4812F0E94B406882331F0EF28F7
:101E800004C01E3211F4A499EF28F6940F5F0830B5
:101E900000F3ED86CE0101960E94EB4165960FB6E8
:101EA000F894DEBF0FBECDBFDF91CF911F910F9190
:101EB000FF90EF9008958091650E9091660E885E78
:101EC000934031F084EF91E09093660E8093650E1D
:101ED0002FE030E03093680E2093670E89E999E097
:101EE00090936A0E8093690E10926B0E10926C0E96
:101EF00010926D0E10926E0E1092700E10926F0E68
:101F0000E5E6FEE0A0E7B0E02115310551F081E003
:101F10002030380719F40E9460660895122E0E943E
:101F200060660895BF92CF92DF92EF92FF920F9377
:101F30001F93CF93DF93CDB7DEB7AE970FB6F8946C
:101F4000DEBF0FBECDBFBB24BE016F5F7F4F8B2DA9
:101F50000E9472338B2D99279C0122953295307FF8
:101F60003227207F3227B90169537E4F9981492F4B
:101F70004170DB018C91887F9670842B892B8C9328
:101F80000F2EF8EBCF2EF1E0DF2EF02DC20ED31E78
:101F90008A819B81F601918380838C819D819383CB
:101FA00082834E815F815583448388859985978399
:101FB0008683D901A054BE4F2A858B85982F929590
:101FC000907F822F8F70892B8C938C8581878D8554
:101FD00082878E8583878F8584878F8D8170982FE8
:101FE000990F990F990FFB018081877F892B80833F
:101FF00088A1F601858789A186878AA18170982F9B
:102000009295907FFB0180818F7E892B80838C91BC
:102010008F70833090F5CA01AA2797FDA095BA2F3B
:10202000BC01CD010E94C462DC01CB0128A539A509
:102030004AA55BA5BC01CD010E94DE617B018C013C
:102040008CA5992787FD9095A92FB92FBC01CD01AB
:102050000E94C462DC01CB019C01AD01C801B70143
:102060000E94A961DC01CB01BC01CD010E942A6064
:10207000DC01CB01F601958384838B2D99279C018C
:1020800022953295307F3227207F3227F901E054A4
:10209000FE4F808182958F708330D8F50F2EF8EB3C
:1020A000CF2EF1E0DF2EF02DC20ED31E888599854C
:1020B000AA2797FDA095BA2FBC01CD010E94C4624A
:1020C000DC01CB0128A539A54AA55BA5BC01CD0142
:1020D0000E94DE617B018C018CA5992787FD90957C
:1020E000A92FB92FBC01CD010E94C462DC01CB0134
:1020F0009C01AD01C801B7010E94A961DC01CB01BF
:10210000BC01CD010E942A60DC01CB01F60197835E
:1021100086832B2D3327C90182959295907F98272E
:10212000807F9827FC01E953FE4F8081869583705C
:10213000813029F4F901E854FC4F808306C08B2DCF
:102140009927FC01E854FC4F10828B2D9927880FAA
:10215000991FFC01E951FC4F11821082B394FFE1F9
:10216000FB1508F0F1CEFE01BD96AAEEB8E082E0C4
:1021700090E021E08030920719F40E944F6603C07E
:10218000182E0E944F668DA58093E5038EA580933F
:10219000E6031092D9031092D803AE960FB6F894C6
:1021A000DEBF0FBECDBFDF91CF911F910F91FF908A
:1021B000EF90DF90CF90BF9008951F93CF93DF9360
:1021C000CDB7DEB7AE970FB6F894DEBF0FBECDBF6A
:1021D00010E0A8958981887F89831B821A821D82DD
:1021E0001C821F821E82198618861A861B861C86F0
:1021F00081E08D871E868F871F8E18A219A21AA2D2
:1022000080E090E0A0E8BFE388A799A7AAA7BBA7B2
:102210001CA685E0FE01B39611928A95E9F78FE03E
:10222000FE017096DF01282F1D922A95E9F7189F6D
:10223000C001112486559E4FBC01CF010E944F65FD
:10224000BE016F5F7F4F812F0E943A331F5F1032B4
:1022500008F4BFCF1EA61DA6FE01BD96AAEEB8E0EB
:1022600082E090E021E08030920719F40E946066DD
:1022700003C0182E0E946066AE960FB6F894DEBFBB
:102280000FBECDBFDF91CF911F9108958093D803EA
:1022900008950F93CF93DF93CDB7DEB721970FB695
:1022A000F894DEBF0FBECDBF89838150803270F0BD
:1022B00000E021E0AE014F5F5F4F69E071E081E037
:1022C00091E00E943D2F80E090E007C0898199272E
:1022D000FC01E954FC4F8081992721960FB6F894B0
:1022E000DEBF0FBECDBFDF91CF910F9108958091DA
:1022F000E503882381F08091E6030E945C448823F3
:1023000051F4482F88EB93E0FC01E40FF11D10829B
:102310004F5F4032C8F340E067EE73E0A8EBB3E0F4
:1023200051E0242F3327C901820F931FFC01E60FD0
:10233000F71F80819181009709F101979183808334
:10234000892BE1F4C90182959295907F9827807F2F
:102350009827FC01E953FE4F808186958370992769
:102360008130910539F0029749F0F901EA0FFB1F1E
:10237000108204C0FD01E40FF11D50834F5F403215
:1023800080F208958091D803882399F08091D90331
:10239000882379F089ED93E0AC014C5F5F4F609149
:1023A000DC038091DA039091DB030E94ED511092DF
:1023B000D90308958F929F92AF92BF92CF92DF92EE
:1023C000EF92FF920F931F93CF93DF938C01EE2434
:1023D000FF2499248091E503882339F08091E60356
:1023E0000E945C44882309F432C28091690E909166
:1023F0006A0E9C0144275527F80180819181A281B2
:10240000B38182179307A407B50799F480916B0EE7
:10241000E80FF11D858190916C0E8923891749F48D
:102420000E9486530E942B211092890E82E2809393
:10243000110160E07091D8030F2EF8EBAF2EF3E09E
:10244000BF2EF02D88248394C090670ED090680E24
:10245000862F992782959295907F9827807F98273D
:10246000EC01C854DE4F88819981AA2797FDA09579
:10247000BA2FF8012081318142815381821793075D
:10248000A407B50759F08A819B81AA2797FDA095DB
:10249000BA2F82179307A407B507C1F4462F552713
:1024A000CA01840F951FFC01E951FC4FD182C08203
:1024B000872F733048F099279C012F733070CA0121
:1024C00003962817390711F4992493948F8583FF75
:1024D00009C08D85F801E80FF11D9E85858198174B
:1024E00009F062C1288139812115310509F45CC1E7
:1024F000442737FD4095542FF80180819181A281B6
:10250000B381281739074A075B0709F09DC091E09E
:102510008985882379F0E80FF11D8481E82EFF2456
:10252000FE2CEE248A85F801E80FF11D8481E80E67
:10253000F11C14C08A85882381F0F801E80FF11D91
:102540008481E82EFF248F8584FF08C0EE2034F4B8
:1025500020E03FEFE22AF32A01C090E0992309F43A
:1025600073C088858F70992782309105B9F18330C7
:1025700091052CF4009779F00197C1F065C0843083
:10258000910509F44DC0843091050CF43EC00597C7
:1025900009F451C059C08C819D818E159F0509F0A9
:1025A00053C0F501E60FF11D80824EC08F8584FF78
:1025B0000BC08C819D818E159F050CF045C0F501E7
:1025C000E60FF11D808240C08C819D818E159F0594
:1025D000D8F5F501E60FF11D808236C08F8584FFA6
:1025E0000AC08C819D81E816F90674F5F501E60FA5
:1025F000F11D808229C08C819D81E816F90620F5A5
:10260000F501E60FF11D80821FC08C819D818E2116
:102610009F21892BC9F0F501E60FF11D808214C0BE
:102620008C819D818E219F21892B71F4F501E60F0C
:10263000F11D808209C08C819D818E159F0521F03E
:10264000F501E60FF11D80828A819B819C01442760
:1026500037FD4095542FF80180819181A281B3818B
:10266000281739074A075B0709F09EC091E08B8560
:10267000882379F0E80FF11D8481E82EFF24FE2CD9
:10268000EE248C85F801E80FF11D8481E80EF11C21
:1026900014C08C85882381F0F801E80FF11D848136
:1026A000E82EFF248F8584FF08C0EE2034F420E05C
:1026B0003FEFE22AF32A01C090E0992309F474C0A5
:1026C000888582958F70992782309105B9F1833082
:1026D00091052CF4009779F00197C1F065C0843022
:1026E000910509F44DC0843091050CF43EC0059766
:1026F00009F451C059C08E819F818E159F0509F044
:1027000053C0F501E60FF11D10824EC08F8584FF86
:102710000BC08E819F818E159F050CF045C0F50181
:10272000E60FF11D108240C08E819F818E159F059E
:10273000D8F5F501E60FF11D108236C08F8584FFB4
:102740000AC08E819F81E816F90674F5F501E60F3F
:10275000F11D108229C08E819F81E816F90620F5AF
:10276000F501E60FF11D10821FC08E819F818E2121
:102770009F21892BC9F0F501E60FF11D108214C0CD
:102780008E819F818E219F21892B71F4F501E60FA7
:10279000F11D108209C08E819F818E159F0521F049
:1027A000F501E60FF11D10826F5F603208F450CE24
:1027B0008091D803882309F44AC0992019F4823003
:1027C00009F045C08091D903823009F440C080915E
:1027D000DA039091DB039C0144275527F80180819F
:1027E0009181A281B381281739074A075B0799F4C1
:1027F0009091DC038481981771F4892F99279801AF
:102800002B5F3F4FAC01B90189ED93E004960E9424
:102810005665892BC9F082E08093D903F8012481A1
:102820002093DC03808191819093DB038093DA0312
:10283000822F992798012B5F3F4FAC01B9018DED95
:1028400093E00E94636503C081E08093D903DF9128
:10285000CF911F910F91FF90EF90DF90CF90BF909D
:10286000AF909F908F9008950E946F058091D8003F
:1028700082608093D8000895CF93DF93EC01898123
:10288000833089F48985882309F403C1888182957E
:10289000807F8093ED008091EF008F738093EF0035
:1028A00018821986F6C00E949305982F81E08987C7
:1028B0009F3F09F4EBC09883892F8295807F809396
:1028C000ED001092EE001092EF001092F7001092BF
:1028D000F6001092F5001092F4001092F000898139
:1028E00099278130910509F46BC0823091051CF461
:1028F000892B29F0C9C0029709F4BBC0C5C08A85DD
:1029000081FF30C08D81982F990F990F990F8C817D
:10291000829586958770890F8093F3008C81982F1C
:10292000990F990F990F8B81829586958770890FE2
:102930008093F2008B81982F990F990F990F8A81BC
:10294000829586958770890F8093F1008A81880F20
:10295000880F880F8093F0008091EF008061809352
:10296000EF0012C08B81982F9295990F907E8A81EB
:10297000869586958695890F8093F3008A81829546
:10298000880F807E8093F20020E08E81181660F41C
:102990008F819885FC01E20FF11D80818093FA0000
:1029A0002F5F8E812817A0F39091EF008E81892BE5
:1029B0008093EF008091EF0080648093EF0069C006
:1029C0008A8581FF35C08D81982F990F990F990FB6
:1029D0008C81829586958770890F8093F3008C8116
:1029E000982F990F990F990F8B81829586958770F3
:1029F000890F8093F2008B81982F990F990F990F6F
:102A00008A81829586958770890F8093F1008A81EB
:102A1000880F880F880F8093F0008091EF0080610D
:102A20008093EF008091F00084608093F00015C0E7
:102A30008B81982F9295990F907E8A8186958695A5
:102A40008695890F8093F3008A818295880F807E16
:102A50008093F20084E08093F0009091EF008E81EB
:102A6000892B8093EF008091EF0080648093EF00CA
:102A700010C08091EF008F738093EF008091EF0082
:102A800080688093EF0005C0198603C08FEF90E047
:102A900002C080E090E0DF91CF910895CF93DF9363
:102AA000EC018985882319F482E090E082C0888156
:102AB0008295807F8093ED000E94AD05813009F002
:102AC0006CC019868091EF008F708E838F819885FE
:102AD0000E94C5058091F0009927847090709595AB
:102AE000879595958795982F91708A85282F2E7FA9
:102AF000292B2A878091EF0084FF31C0822F8260CA
:102B00008A878091F3008695869586958D8380913E
:102B1000F200982F9695969596958091F300829560
:102B2000880F807E890F8C838091F100982F969575
:102B3000969596958091F2008295880F807E890FF8
:102B40008B838091F000982F96959695969580911D
:102B5000F1008295880F807E890F8A8316C08A854E
:102B60008D7F8A878091F3008295869587708B830D
:102B70008091F200982F9295969597708091F3002E
:102B8000880F880F880F890F8A838091EF008F73D9
:102B90008093EF0080E090E00CC0882349F489879F
:102BA0008091EF008F738093EF0080E090E001C090
:102BB0009927DF91CF910895982F8F3F19F481E0E5
:102BC00090E00895805C843128F4892F0E945C4451
:102BD00099270895892F8150803228F4892F0E94E7
:102BE000491199270895892F8152843128F4892F1A
:102BF0000E94CE579927089580E090E00895982F7D
:102C00008F3F19F481E090E00895805C843128F4CE
:102C1000892F0E943B4399270895892F8150803244
:102C200028F4892F0E94491199270895892F8152EC
:102C3000843128F4892F0E94CE579927089580E087
:102C400090E008958091750E8F5F8093750E80914E
:102C5000780E8F5F8093780E8091760E833008F423
:102C60004AC08F5F8093760E843031F440E061E497
:102C700086E00E943F3C3FC08091750E823390F405
:102C80008091760E853031F440E061E486E00E9468
:102C90008A3C31C08091760E873069F583E080935D
:102CA000760E29C08091750E843688F48091760E58
:102CB000863029F440E061E40E948A3C1CC0809187
:102CC000760E8730C1F483E08093760E14C0809135
:102CD000750E823868F48091760E873061F440E09A
:102CE00061E486E00E948A3C83E08093760E03C014
:102CF00081E08093760E8091770E833008F44AC08D
:102D00008F5F8093770E843031F441E061E486E098
:102D10000E943F3C08958091780E823390F4809118
:102D2000770E853031F441E061E486E00E948A3C10
:102D300008958091770E873069F583E08093770E50
:102D400008958091780E843688F48091770E8630CD
:102D500029F441E061E40E948A3C08958091770E55
:102D60008730C1F483E08093770E08958091780EC8
:102D7000823868F48091770E873061F441E061E435
:102D800086E00E948A3C83E08093770E089581E07C
:102D90008093770E089580917A0E0E94DC15882327
:102DA00021F085E08093E00946C080917F0E0E946B
:102DB000DC15882341F08091800E8093E30983E045
:102DC0008093E00938C08091790E0E94DC15882339
:102DD00021F084E08093E0092EC080917B0E0E9458
:102DE000DC15882369F08091E009873049F086304E
:102DF00039F086E08093E0098AE08093E2091BC005
:102E00008091E009853021F482E08093E00913C0CD
:102E10008091E009833041F48091E309882321F413
:102E200081E08093E00907C08091E009843019F4C3
:102E300081E08093E0098091E0098150823058F46C
:102E400080917C0E0E94FF1590917D0E981719F4C9
:102E50001092E00917C08091E209882399F48091CB
:102E6000E009863079F480917C0E0E94FF159091E4
:102E70007D0E981739F487E08093E00980917E0EEB
:102E80008093E1098BE599E00E94952D0E94051938
:102E900008951F93CF93DF9310E0812F9927EC01C2
:102EA000C80FD91FFE01EF57F14F8081882309F425
:102EB000B4C00E94DC15882309F4AFC0FE01EE57B0
:102EC000F14F808183FDB3C088608083877099272C
:102ED0008230910539F1833091051CF4019729F076
:102EE000A6C0039709F452C0A2C0812F9927880F6A
:102EF000991FFC01EE57F14F9081892F82958F70B9
:102F0000877021F0892F8F78808391C0812F992736
:102F1000880F991FFC01EE57F14F80818F788061F7
:102F2000808385C0812F9927880F991FFC01EE5758
:102F3000F14F808182958F7087709927009719F0E3
:102F4000019769F018C0812F9927880F991FFC01FC
:102F5000EE57F14F80818F788061808368C0812F28
:102F60009927880F991FFC01EE57F14F80818F78C8
:102F7000806280835CC0812F9927880F991FFC0194
:102F8000EE57F14F80818F78808351C0812F992730
:102F9000880F991FFC01EE57F14F808182958F7049
:102FA0008770992781309105A9F0823091051CF432
:102FB000892B21F027C00297C9F024C0812F9927BF
:102FC000880F991FFC01EE57F14F80818F78806147
:102FD00080832DC0812F9927880F991FFC01EE5700
:102FE000F14F80818F788062808321C0812F992763
:102FF000880F991FFC01EE57F14F80818F78806315
:10300000808315C0812F9927880F991FFC01EE57E7
:10301000F14F80818F7880830AC0812F9927880F94
:10302000991FFC01EE57F14F8081877F80831F5FDE
:10303000143008F432CF0E94FF210E9494200E9495
:103040007A2310E085E2189FC0011124EC01C25DD3
:10305000DB4F8C899D89009719F001979D8B8C8B94
:103060008D859E85009761F001979E878D87998554
:103070009F3F31F085E0989FC00111249B878A878C
:103080002A853B852115310561F089858F3F49F0FF
:10309000C90101979B878A87892B19F48F858062E4
:1030A0008F878A8D9B8D009779F001979B8F8A8FF0
:1030B000892B51F48F8586FD04C0812F8F5F0E947C
:1030C0001B328F8580648F878F81882311F0815018
:1030D0008F831F5F123208F4B5CFDF91CF911F911C
:1030E00008958091E209882319F081508093E209C4
:1030F0008091E0098730B9F48091E109882321F0BB
:1031000081508093E1090FC080917B0E0E94DC15F5
:10311000882339F086E08093E0098AE08093E20911
:1031200002C01092E0098091E309882319F08150D0
:103130008093E309A49B23C02091DD092F3710F46D
:10314000220F01C02FEF80916D0E8A30D0F0909148
:10315000740E981710F0921730F48091740E8F5FF0
:103160008093740E0EC08091890E882351F48F5F76
:103170008093890E0E9486530E942B2102C01092D8
:10318000740E90915209809162099817E0F420E042
:1031900042E659E065E270E0FA01E20FF11D82813A
:1031A000823268F49927869FF001879FF00D969FE1
:1031B000F00D1124EE5CFB4F8081816080832F5FD6
:1031C0002C3050F30895909152098091630989172A
:1031D000D8F420E042E659E065E270E0FA01E20F3F
:1031E000F11D8281823268F49927869FF001879FC2
:1031F000F00D969FF00D1124EE5CFB4F80818E7FC9
:1032000080832F5F2C3050F30895CF92DF92EF929E
:10321000FF920F931F93CF93DF938091280488230D
:1032200009F004C1F82E0F2EFAE0EF2EF02D8EE0FB
:10323000F89EC0011124EC01C956D64F00E08A81E6
:103240008F3F11F401E01DC09A81892F805C843189
:1032500028F4892F0E945C44082F13C09A81892F7B
:103260008150803228F4892F0E944911082F09C00B
:103270009A81892F8152843120F4892F0E94CE5760
:10328000082F8981992781309105C9F182309105F4
:103290001CF4892B29F0C5C0029709F4BFC0C1C036
:1032A000013009F0BEC08F818E9DC00111249C8326
:1032B0008B8389858E9DC00111249E838D83888197
:1032C0008460888310E025E230E0FE01E10FF11D0B
:1032D00082858F3F71F09927829FA001839F500DB7
:1032E000929F500D1124FA01EE5CFB4F80818460A7
:1032F00080831F5F143048F381E0898392C08B8103
:103300009C81009709F48DC001979C838B83892B46
:1033100081F5288122FF17C08F818E9DC001112465
:103320009C838B83822F8B7F888310E0FE01E10FCB
:10333000F11D82858F3F19F060E00E941F1A1F5F08
:103340001430A0F316C088858E9DC00111249C8383
:103350008B8388818460888310E0FE01E10FF11D7A
:1033600082858F3F19F061E00E941F1A1F5F1430A1
:10337000A0F38881282F227081FD28C08D819E8135
:10338000009709F44EC001979E838D83892B09F025
:1033900048C082E08983122F25E230E0FE01E10F70
:1033A000F11D82858F3F71F09927829FA001839F35
:1033B000500D929F500D1124FA01EE5CFB4F80815D
:1033C0008B7F80831F5F143048F32BC0002349F5A7
:1033D000102F0F2EF5E2CF2EDD24F02DFE01E10F90
:1033E000F11D22852F3F99F0822F99278C9DA001F6
:1033F0008D9D500D9C9D500D1124FA01EE5CFB4FEC
:1034000080818B7F808361E0822F0E941F1A1C8243
:103410001B821F5F143010F3198203C0002309F4CC
:103420000983F39454E05F1508F001CFDF91CF9149
:103430001F910F91FF90EF90DF90CF900895DF9252
:10344000EF92FF920F931F93CF93DF93CDB7DEB729
:1034500021970FB6F894DEBF0FBECDBF8983162F1C
:10346000DD24833260F00D2D21E0AE014F5F5F4F10
:1034700067ED72E082E191E00E943D2F4EC099819C
:1034800085E2989F700111248EE294E0E80EF91E07
:10349000F701858D9927807F9070803A910529F4F6
:1034A0000F2EF1E4DF2EF02D18C0F701858D99273E
:1034B000807F9070803B910529F40F2EF2E4DF2E7F
:1034C000F02D0BC000E021E0AE014F5F5F4F63EED7
:1034D00072E082E191E00E943D2F112379F483E0B4
:1034E000F701878380EF818387858F7B8787858D31
:1034F00041A16D2D8F700E943F3C0FC0113069F4C7
:10350000F70117828FE08183878586798787858D8C
:1035100041A16D2D8F700E948A3C21960FB6F894C0
:10352000DEBF0FBECDBFDF91CF911F910F91FF90F6
:10353000EF90DF90089520E040E759E065E270E009
:103540008170382F330FFA01E20FF11D8181823231
:1035500070F49927869FF001879FF00D969FF00DDC
:103560001124EE5CFB4F80818D7F832B80832F5F46
:103570002E3048F3089520E040E759E065E270E01E
:103580008170382F330FFA01E20FF11D81898232E9
:1035900070F49927869FF001879FF00D969FF00D9C
:1035A0001124EE5CFB4F80818D7F832B80832F5F06
:1035B0002E3048F3089580912A0490912B040895A9
:1035C0008091290499270895EF92FF921F93CF933A
:1035D000DF937A01809362096093630910E0C12F41
:1035E000DD27F701EC0FFD1F80810E94222A823225
:1035F00020F4FE01EE59F64F82831F5F1C3078F3F2
:10360000DF91CF911F91FF90EF9008957F928F925D
:103610009F92AF92BF92CF92DF92EF92FF920F9361
:103620001F93CF93C0E00E94232C0E94122D0E9472
:103630003D2D8BE599E00E948A2D10925009109241
:103640004F09C0935109C0935309C0935409C093C3
:103650005509C093560982E1E8E1F9E011928A9593
:10366000E9F74AE259E028EB31E08C2F9927880FDF
:10367000991FFC01E40FF51F31832083CF5FC23116
:10368000A0F3C0E047E959E02EE030E08C2F992705
:10369000829FB001839F700D929F700D1124FB01DA
:1036A000E40FF51F11821482138216821582FB012A
:1036B000E956F64F808184608083CF5FC53030F358
:1036C0000E94CA35803221F487E68093100103C03E
:1036D0008EE680931001AEE2B4E041E040932E0408
:1036E00028EC30E0309341042093400452EA509398
:1036F0004B0462EB60934C0410924F049FEF909345
:103700004D0450934E0483E0809350048D010B5D73
:103710001F4F40935304FD0130AF27ABF801558F85
:10372000668F41A3978F0F2EF7EAEF2EF02DE0A2C0
:103730000F2EFFE0BF2EF02DB2A2FD01E65BFF4F82
:1037400040937804338B228B0F2EF3EADF2EF02D7B
:10375000D58E83EB868F41A3978F90A389E082A3B8
:10376000FD01E159FF4F40939D04338B228BE58E81
:103770000F2EF7EBCF2EF02DC68E41A3978F90A37F
:103780008BE082A3FD01EC56FF4F4093C204338BC4
:10379000228B11EA158F0F2EF1EBFF2EF02DF68EF6
:1037A00041A3978F90A38EE082A3FD01E754FF4FC2
:1037B0004093E704338B228B55EA558F05EB068F38
:1037C00041A3978F90A38DE082A3C6E0FD01E25252
:1037D000FF4F40930C05338B228B60EA658F70EBB3
:1037E000768F11A2978F50A3C2A3FD01ED5FFE4F0C
:1037F00040933105338B228B558F068F11A2978F03
:1038000090A384E082A3FD01E85DFE4F409356053E
:10381000338B228B658F768F41A3978F60A38AE0CD
:1038200082A3FD01E35BFE4F40937B05338B228B2C
:10383000758F54EB568F75E071A3978F90A382E13B
:1038400082A3FD01EE58FE4F4093A005338B228BDF
:1038500064EA658F568F41A3978FD0A288E082A338
:10386000FD01E956FE4F4093C505338B228B56EA86
:10387000558F86EB868F11A2978F60A342A3CCE071
:10388000FD01E454FE4F4093EA05338B228B558FA4
:10389000868F41A3978F10A3C2A3FD01EF51FE4F66
:1038A00040930F06338B228BE58EC68E11A2978F25
:1038B00090A382E082A3FD01EA5FFD4F40933406AE
:1038C000338B228B158FF68E11A2978F90A387E0F2
:1038D00082A3FD01E55DFD4F40935906338B228B9A
:1038E000F58E068F71A3978F2B2D3327AD0185E2BF
:1038F00090E0289FB001299F700D389F700D112412
:10390000FB01EA0FFB1F9FEF90A381E182A3FD0162
:10391000E05BFD4F61E060937E0628EC30E0338B86
:10392000228BB4EAB58F0F2EF4EBFF2EF02DF68E1E
:1039300011A2978F0F2EF6EAEF2EF02DE0A285E070
:1039400082A3FA01EB58FD4F6093A306338B228BC1
:103950008D2CD58E03EB068F11A2978F90A312A208
:10396000FA01E656FD4F70E47093C8062FEF3FEF63
:10397000338B228B0F2EF7EADF2EF02DD58EF68EAD
:1039800063E061A3E78E90A392A3FA01E154FD4F97
:103990007093ED06338B228BE58E15EB168F61A3AA
:1039A000E78E90A392A3FA01EC51FD4F709312079A
:1039B000338B228BA5EAA58F0F2EF6EB7F2EF02DF1
:1039C000768E61A3D78E90A392A3FA01E75FFC4F96
:1039D00070933707338B228BB58FC68E61A3D78E3A
:1039E00090A392A3FA01E25DFC4F70935C07338BC6
:1039F000228B80EA858F068F61A3A78F90A392A365
:103A0000FA01ED5AFC4F70938107338B228B0F2EF6
:103A1000F1EABF2EF02DB58E0F2EF2EBAF2EF02D6A
:103A2000A68E61A3A78F90A392A3FA01E858FC4F3A
:103A30007093A607338B228B0F2EF2EA9F2EF02D68
:103A4000958EA1EBA68F61A3B78F90A392A3FA01E5
:103A5000E356FC4F7093CB07338B228B858E0F2E52
:103A6000F0EBCF2EF02DC68E61A3B78F90A392A35B
:103A7000FA01EE53FC4F7093F007338B228B858F46
:103A8000068F82E081A3178F90A392A3FA01E951D8
:103A9000FC4F70931508338B228BB58EA68E81A3B5
:103AA000178F90A392A3FA01E45FFB4F70933A083B
:103AB000338B228B958EA68F81A3F78E90A392A332
:103AC000FA01EF5CFB4F70935F08338B228B858E7E
:103AD000C68E81A3F78E90A392A3FA01EA5AFB4FF8
:103AE00070938408338B228BD58EF68E81A3778ECC
:103AF00090A392A3FA01E558FB4F7093A908338B6A
:103B0000228BE58EFA01E558FB4F168F9A01FA01D8
:103B1000E558FB4F52E051A3778E4FEF40A342A3ED
:103B2000F901E056FB4FA72F7093CE086FEF7FEFA0
:103B3000738B628B85EA858F768E51A397EB978F77
:103B400040A342A3F901EB53FB4FA093F308738BFF
:103B5000628BB58F968F51A3978F40A342A3C0E08D
:103B6000B90145E250E02FE001E21EE130E18C2F87
:103B70009927849FF001859FF00D949FF00D1124EB
:103B8000CF01E60FF71F158A148ADC01AE5CBB4F2C
:103B90008C918C7D8C931786168A218314A213A294
:103BA0001686158614861386128611868C918B7F55
:103BB0008C93178A17820087168335832283118E90
:103BC000108E138E128E148ECF5FC23280F2CF9180
:103BD0001F910F91FF90EF90DF90CF90BF90AF902B
:103BE0009F908F907F900895E8E1F9E082E1DF01F6
:103BF0001D928A95E9F7CF010E94FC3420E06AE229
:103C000079E048EB51E0822F9927880F991FFC013A
:103C1000E60FF71F518340832F5F2231A0F38AE222
:103C200099E00E941C350895AF92BF92CF92DF9227
:103C3000EF92FF920F931F93CF93DF93CDB7DEB731
:103C4000C35CD0400FB6F894DEBF0FBECDBF10E00E
:103C50000F2EF5E6EF2EFF24F02DEC0EFD1E212F8A
:103C6000332785E290E0289FA001299F500D389FBF
:103C7000500D11249A01225D3B4FF90182899389ED
:103C8000892F9927D7018C938289F7018183F901C4
:103C90008681F7018283158214821682F90185815B
:103CA000F7018383F9018085F70187838FE0189FEF
:103CB000C001112486589B4FBC01C70108960E9481
:103CC0004F65F701178A108E1F5F612FC7010E9491
:103CD0001A34A895123218F28E0102581F4F84E64A
:103CE000D8018C9388E7F80181834CE050E06FEFB6
:103CF00070E0C80102960E947065C8010E945A32A5
:103D00008E0104571F4FF80181EC81934EE050E083
:103D10006FEF70E0CF010E947065F80117868AE0AE
:103D2000808B4EE050E06FEF70E0C80141960E943A
:103D30007065C8010E948832A89510E00F2EF4E14A
:103D4000DF2EF02D7E010894E11CF11C0FE0D7015D
:103D5000ED2D1D92EA95E9F7109FC00111248B52B9
:103D60009C4FBC01C7010E944F65188A1F5FB701B5
:103D7000812F0E94B1341B3050F3A89510E00F2E14
:103D8000F5EBAF2EBB24F02DAC0EBD1E0F2EFFE0C9
:103D9000CF2EF02D0F2EFBEAEF2EFF24F02DEC0E90
:103DA000FD1EDD24D3940FEFD501EC2D1D92EA9575
:103DB000E9F71C9DC001112486579C4FBC01C70127
:103DC0000A960E944F65D7011C92F7011182128258
:103DD000D382D4828AE085838081F701E80FF11DC8
:103DE00006838F5F8430C8F3BE0165557F4F812FF6
:103DF0000E94C8321F5F1530B8F2EFE8F9E018E012
:103E0000DF01212F1D922A95E9F7CF010E94A832E8
:103E10000E94052DA895E9E7FEE0DF011D921A95A5
:103E2000E9F781E080937D0E8EE180937E0E82E340
:103E30008093800EAEE6BFE088E090E021E0803025
:103E4000920719F40E94606603C0182E0E946066F3
:103E50009E012B5E3F4F8CE4D9011D928A95E9F7B4
:103E60008CE0A0E2B1E0FE017796482F0D90019220
:103E70004A95E1F7ACE2B1E0FE01BA96582F0D90F9
:103E800001925A95E1F7A8E3B1E0FE01FD96982F63
:103E90000D9001929A95E1F7A4E4B1E0FE01E05B98
:103EA000FF4F0D9001928A95E1F7F901AEE8BFE06E
:103EB0008CE490E021E08030920719F40E94606663
:103EC00003C0182E0E94606688E0E1E8FEE01192CF
:103ED0008A95E9F7CD53DF4F0FB6F894DEBF0FBEDA
:103EE000CDBFDF91CF911F910F91FF90EF90DF90A9
:103EF000CF90BF90AF900895CF92DF92EF92FF9254
:103F00000F931F93CF93DF93CDB7DEB7E4970FB630
:103F1000F894DEBF0FBECDBF00E0102F1F5F612FF2
:103F2000CE0101960E945F34202F332785E290E076
:103F3000289FA001299F500D389F500D1124FA0190
:103F4000E25DFB4F89819927982F88272A81820F6C
:103F5000911D938B828B8B818683888580878C8152
:103F60008583888D8487898D81878D819E81918FBE
:103F7000808F8F81848F012F123278F282E699E050
:103F80000E94783280E799E00E94983288E199E0B7
:103F90000E940C358AE299E00E942C358FE899E066
:103FA0000E94B8320E94052D00E0BE01665E7F4F80
:103FB000802F0E940133202F33278EE090E0289F2E
:103FC000F001299FF00D389FF00D11249F01E95653
:103FD000F64F8A8D582F51708081482F4C7F8B8DE2
:103FE0008170982F990F842F852B892B8083F9015D
:103FF000E956F64F8C8D82838D8D87838E8D8087D9
:104000008F8D8187F901EF55F64F88A199A1AAA15B
:10401000BBA180839183A283B3830F5F053028F215
:10402000E9E7FEE0AEE6BFE088E090E021E0803026
:10403000920719F40E944F6603C0182E0E944F6623
:1040400000E073E142E050E0642F0F2EF1E8CF2E44
:10405000FEE0DF2EF02D0F2EF3E3EF2EFF24F02DE8
:10406000EC0EFD1EFE01F396079FC0011124DC013A
:10407000A257B04F4115510551F081E0403058072B
:1040800019F40E944F6603C0162E0E944F66802FBF
:1040900099279C01280F391FF901EC0DFD1D8BA9F3
:1040A0008083D901AE57B14FF7018181982F977066
:1040B0008C918078892B8C930F5F043098F2E49672
:1040C0000FB6F894DEBF0FBECDBFDF91CF911F9129
:1040D0000F91FF90EF90DF90CF900895CF93DF93F3
:1040E000EC01862F0E94222A8332D8F4282F33270E
:1040F00085E290E0289FA001299F500D389F500D28
:104100001124FA01E25DFB4F8F898487888199270A
:10411000982F88272981820F911D938B828B8A810A
:104120008683DF91CF9108951F93CF93C0E01C2F1A
:1041300090917009892F8150803238F4892F0E9424
:1041400049118823B1F011E014C090917009892FB2
:104150008152843138F4892F0E94CE57882349F048
:1041600011E007C0809170090E945C44813009F41D
:10417000182F90917F09892F8150803220F4892F48
:104180000E9449110EC090917F09892F815284317C
:1041900020F4892F0E94CE5704C080917F090E948D
:1041A0005C448E3FF1F08130B9F48091DE098430B7
:1041B00020F48F5F8093DE0909C01092DE098091A0
:1041C000DF09882319F081508093DF098091DF098E
:1041D000882359F4C1E009C0809180098093DF09E8
:1041E00004C0809180098093DF09113021F4812F70
:1041F0000E949B1A0CC0C13021F48C2F0E94BB1A64
:1042000006C080E00E949B1A80E00E94BB1ACF91FA
:104210001F910895FC018481982F986080EF82831C
:10422000878586798787168A892F8F7D8483848501
:1042300025E0829FC001112496878587892B41F450
:1042400081858F3F29F0829FC00111249387828747
:1042500083E0878308951F93CF93C0E015E2C19F49
:10426000C0011124FC01E25DFB4F8785992783FD86
:1042700002C080FF03C0CF010E940A21CF5FC2327B
:1042800070F3CF911F91089599278C33910509F40C
:1042900066C08D339105A4F488339105A1F189336B
:1042A00091051CF4C79721F1A7C089339105B1F19D
:1042B0008A33910509F43DC0CB9709F445C09CC0F1
:1042C0008034910509F477C08134910544F48E332C
:1042D000910509F45AC0CF970CF062C04BC08134ED
:1042E000910509F473C08234910509F47AC084C041
:1042F0008091820E8077803119F481E090E00895FA
:1043000080E090E008958091820E8077803219F4E9
:1043100081E090E0089580E090E008958091820E21
:104320008077803319F481E090E0089580E090E098
:1043300008958091840E8077803119F481E090E0B7
:10434000089580E090E008958091840E8077803217
:1043500019F481E090E0089580E090E00895809164
:10436000840E8077803319F481E090E0089580E036
:1043700090E008958091860E8077803119F481E075
:1043800090E0089580E090E008958091860E807717
:10439000803219F481E090E0089580E090E0089583
:1043A0008091860E8077803319F481E090E0089543
:1043B00080E090E008958091880E8077803119F434
:1043C00081E090E0089580E090E008958091880E6B
:1043D0008077803219F481E090E0089580E090E0E9
:1043E00008958091880E8077803319F481E090E001
:1043F000089580E090E0089580E090E00895FF92B5
:104400000F931F93CF93DF9310E00F2EFFE0FF2E4B
:10441000F02D82E00E94024585E2189FC001112420
:10442000EC01C25DDB4F8885882361F48981803F80
:1044300009F0F4C08C8188608C838F85867B8F87A0
:10444000FA82ECC02885822F81508032D0F58F858A
:10445000992783FD24C080FD22C0822F0E9449112C
:10446000882341F089818F3009F0D8C0CE010E94A5
:104470000A21D4C08981803F09F0D0C089858F3F4F
:1044800009F4CCC08A859B85892B09F0C7C08C8133
:1044900088608C838F85867B8F87FA82BFC08885F2
:1044A0000E944911882309F0B9C08981803F09F031
:1044B000B5C08C8188608C838F85867B8F87FA82DC
:1044C000ADC02885822F81528431D0F58F85992700
:1044D00083FD24C080FD22C0822F0E94CE578823F6
:1044E00041F089818F3009F099C0CE010E940A21E4
:1044F00095C08981803F09F091C089858F3F09F47B
:104500008DC08A859B85892B09F088C08C81886045
:104510008C838F85867B8F87FA8280C088850E94F6
:10452000CE57882309F07AC08981803F09F076C090
:104530008C8188608C838F85867B8F87FA826EC0A2
:1045400000E08885853371F49091E009892F8350CC
:10455000823020F0913011F0963011F491E01DC0BE
:1045600090E01BC08885863351F48091E009853046
:1045700011F0823011F491E010C090E00EC09885E7
:10458000892F87538C3028F4892F0E944421982F3B
:1045900004C088850E945C44982F9E3FA9F08885BE
:1045A000803C21F49130A1F4092F12C08D8181301B
:1045B00021F4913011F4092F0BC08D81803141F429
:1045C000992331F401E004C088858F3F09F401E0AC
:1045D000002369F089818F3009F58F85992783FD44
:1045E0001DC080FD1BC0CE010E940A2117C0898119
:1045F000803F31F08F85992783FD02C080FF0EC078
:1046000089858F3F59F08A859B85892B39F48C8168
:1046100088608C838F85867B8F87FA8289818F3033
:1046200079F48F85992789709070892B49F480914E
:104630001101811729F482E2809311011092890EF1
:104640001F5F123208F4E5CEDF91CF911F910F91D9
:10465000FF90089560932804623019F48FEF8093DF
:104660004E090895CF93DF93EC0188818150823207
:1046700018F080E090E03BC088810E94222A282F19
:10468000898199278F30910521F0803F9105A1F014
:104690002CC0332785E290E0289FA001299F500D70
:1046A000389F500D1124FA01E25DFB4F8FE08183AA
:1046B0008785867F878719C0332785E290E0289F0A
:1046C000A001299F500D389F500D1124FA01E25D81
:1046D000FB4F80EF81838785867F8787168AFA0163
:1046E000EE5CFB4F80818F7D808381E090E0DF91E5
:1046F000CF9108956F927F928F929F92AF92BF92C7
:10470000CF92DF92EF92FF920F931F93CF93DF939D
:10471000CDB7DEB721970FB6F894DEBF0FBECDBF81
:10472000BB24B9829B2CAB2C8B2C1092500910927D
:104730004F09B0925309B0925509B09254090E94A2
:1047400022058093520980912804882309F0C1C36F
:10475000B9828B2D823208F03EC67724689471F8B6
:104760000F2EF3E06F2EF02D82E00E940245992477
:10477000998185E2989FC00111240F2EFEE2CF2E71
:10478000F4E0DF2EF02DC80ED91EF601858D992795
:10479000807F9070803A910529F40F2EF1E4AF2EBE
:1047A000F02D18C0F601858D9927807F9070803B91
:1047B000910529F40F2EF2E4AF2EF02D0BC000E08E
:1047C00021E0AE014F5F5F4F61ED77E082E191E064
:1047D0000E943D2FF601118A108A248122FDFAC120
:1047E000808199278130910509F4FBC080349105BF
:1047F00009F0FDC1818199278F30910509F497C097
:10480000803F910509F0F3C1822F837019F48785E9
:1048100085FF1BC089818B3031F48091760E88230F
:1048200011F07092760E89818C3031F48091770E80
:10483000882311F07092770EF601858D41A16A2DC3
:104840008F700E948A3C99244BC0F601858596851D
:10485000892B09F045C0878580FD42C089818B3056
:10486000C9F48091760E8823A9F0823048F4858DB2
:1048700041A16A2D8F700E943F3C9924939430C0CF
:104880008091760E813061F56092760E1092750EF1
:10489000992426C089818C30D1F48091770E8823A9
:1048A000B1F0823050F4F601858D41A16A2D8F70F0
:1048B0000E943F3C9924939413C08091770E8130DD
:1048C00079F46092770E1092780E992409C0F6015F
:1048D000858D41A16A2D8F700E943F3C992493944D
:1048E000F601848183FF83C1877F848382818F3037
:1048F00009F07DC189818B3031F48091760E882357
:1049000011F07092760E89818C3031F48091770E9F
:10491000882311F07092770E8FE0F6018183858DE8
:1049200041A16A2D8F700E948A3C992460C1F601D2
:10493000248123FF5CC1822F877F84838281803F13
:1049400009F055C1818385859685892B09F04FC172
:10495000822F837009F04BC189818B30D1F4809113
:10496000760E8823B1F0823048F4858D41A16A2DFE
:104970008F700E943F3C9924939439C18091760EA8
:10498000823009F034C16092760E1092750E99242F
:104990002EC189818C30D9F48091770E8823B9F0AB
:1049A000823050F4F601858D41A16A2D8F700E94EE
:1049B0003F3C992493941BC18091770E823009F07B
:1049C00016C16092770E1092780E992410C1F601EC
:1049D000858D41A16A2D8F700E943F3C992493944C
:1049E00006C1F601818199278F30910509F49AC09B
:1049F000803F910509F0FBC08481837019F487859D
:104A000085FF1BC089818B3031F48091760E88231D
:104A100011F07092760E89818C3031F48091770E8E
:104A2000882311F07092770EF601858D41A16A2DD1
:104A30008F700E948A3C99244EC0F6018585968528
:104A4000892B09F048C08785992780FD44C083FDE4
:104A500042C089818B30C9F48091760E8823A9F0F9
:104A6000823048F4858D41A16A2D8F700E943F3CB1
:104A70009924939430C08091760E823061F56092D3
:104A8000760E1092750E992426C089818C30D1F44F
:104A90008091770E8823B1F0823050F4F601858D35
:104AA00041A16A2D8F700E943F3C9924939413C0BA
:104AB0008091770E823079F46092770E1092780EA2
:104AC000992409C0F601858D41A16A2D8F700E943D
:104AD0003F3C99249394F601848183FF88C0877FAB
:104AE000848382818F3009F082C089818B3031F4D8
:104AF0008091760E882311F07092760E89818C3029
:104B000031F48091770E882311F07092770E8FE048
:104B1000F6018183858D41A16A2D8F700E948A3CA8
:104B2000992465C0F601248123FF61C0822F877F0D
:104B300084838281803F09F05AC081838585968570
:104B4000892B09F054C0822F837009F050C08981ED
:104B50008B30C9F48091760E8823A9F0823048F416
:104B6000858D41A16A2D8F700E943F3C99249394BA
:104B70003EC08091760E8230D1F56092760E109212
:104B8000750E992434C089818C30D1F48091770ED0
:104B90008823B1F0823050F4F601858D41A16A2D51
:104BA0008F700E943F3C9924939421C08091770E8E
:104BB0008230E9F46092770E1092780E992417C033
:104BC000F601858D41A16A2D8F700E943F3C99248A
:104BD00093940DC0F601818199278F30910531F0B2
:104BE000803F910521F49924939401C09924F60102
:104BF0008181803F09F058C082A18F3F09F454C0E1
:104C00000E94F1037C0100271127F601F4A2E3A220
:104C100089819927FC01E85EF64F80819927AA27B0
:104C2000BB278E159F05A007B10724F0EE24FF24B3
:104C300087010AC089819927FC01E85EF64F8081CF
:104C4000E81AF10801091109F3E0EF16F104010572
:104C50001105CCF089819927880F991FFC01E65D29
:104C6000F64F808191819C0144275527C801B701E7
:104C70000E94816520EE31E040E050E00E94F56541
:104C800079018A0103C0EE24FF248701F601F18A2D
:104C9000E08A80914F09909150098E0D9F1D90934D
:104CA000500980934F0903C0F601118A108A992098
:104CB00039F4F601828D938D892B11F0138E128EAB
:104CC000F60187859927AC014870507083FD70C04C
:104CD000208931898289938982179307E0F5828D33
:104CE000938D892B11F0538F428FF601848185FFBC
:104CF00026C084899589892B09F05AC087858860E8
:104D00008787809153098F5F809353098081813019
:104D100071F4858D41A16A2D8F700E948A3C99247F
:104D2000898180931101F60186818093DD09898153
:104D3000F601608971898F5F0E94B03139C0F60138
:104D4000848180628483968185E0989FC0011124CC
:104D5000958B848B2DC0F60184818F7D8483208D7B
:104D6000318D2115310521F19920A1F0808991899A
:104D70008217930778F4828D938D892BC9F48785E8
:104D800086FD16C0948D85E0989FC0011124938FF5
:104D9000828F0EC0F601828D938D892B49F0208978
:104DA0003189808D918D8217930710F4138E128EA6
:104DB000F601868D9927807F9070803A910529F4BD
:104DC0000F2EF1E48F2EF02D18C0F601868D992755
:104DD000807F9070803B910529F40F2EF2E48F2E96
:104DE000F02D0BC000E021E0AE014F5F5F4F6FE49C
:104DF00079E082E191E00E943D2FF601868D41A18C
:104E0000682D8F700E940D3D282FF6018181803F13
:104E100009F042C08785992783FD3EC080FD3CC0D4
:104E200090915209809110018917B0F5F1E09F1619
:104E300089F5222379F5F6018781882369F5848530
:104E4000882351F587898F3F11F08F5F878BF6019B
:104E50008789863008F186898F5F868B843150F48C
:104E6000858D41A16A2D8F700E948A3CF601178AB8
:104E7000678212C0F601858D41A16A2D8F700E9454
:104E80008A3CF60187858160878789818F5F0E94D0
:104E9000E83102C0F601178AF601878580FF05C058
:104EA000809155098F5F80935509F601878583FFAF
:104EB00005C0809153098F5F80935309F601878560
:104EC0008111B39489818F5F8983823208F44CCC3D
:104ED00082C280912804813009F0B0C11982898191
:104EE000482F823208F077C2242F332785E290E0E2
:104EF000289FB001299F700D389F700D1124FB0170
:104F0000E25DFB4F87858F7D878785E2489FC001E3
:104F100011240F2EFEE2CF2EF4E0DF2EF02DC80E6E
:104F2000D91EF601858D9927807F9070803A910572
:104F300029F40F2EF1E4AF2EF02D0CC0F601858D73
:104F40009927807F9070803B910521F40F2EF2E429
:104F5000AF2EF02DF601848182FD4FC0808199270C
:104F60008130910569F18034910509F046C0818155
:104F700099278F30910561F0803F9105F1F5858D7E
:104F800041A16A2D8F700E943F3C9924939435C0B3
:104F90008981282F332785E290E0289FA001299F4F
:104FA000500D389F500D1124FA01E25DFB4F858DA5
:104FB000F60141A16A2D8F700E948A3C99241DC080
:104FC000F601818199278F30910561F0803F91052D
:104FD000A1F4858D41A16A2D8F700E943F3C9924D8
:104FE00093940BC0F601858D41A16A2D8F700E94AC
:104FF0008A3C8FE0F60181839924F6018181803F0C
:1050000009F057C082A18F3F09F453C00E94F103F9
:105010007C0100271127F601F4A2E3A289819927D8
:10502000FC01E85EF64F80819927AA27BB278E15E1
:105030009F05A007B10724F0EE24FF2487010AC0D2
:1050400089819927FC01E85EF64F8081E81AF10812
:1050500001091109F3E0EF16F10401051105CCF087
:1050600089819927880F991FFC01E65DF64F8081A1
:1050700091819C0144275527C801B7010E94816591
:1050800020EE31E040E050E00E94F56579018A01B0
:1050900003C0EE24FF248701F601F18AE08A8091A3
:1050A0004F09909150098E0D9F1D90935009809348
:1050B0004F09F601208931898289938982179307E4
:1050C00088F5848185FF22C084899589892B81F5A3
:1050D000878588608787809153098F5F8093530904
:1050E0008081813059F4858D41A16A2D8F700E9495
:1050F0008A3C99248FE0F601818382838981F601BD
:10510000608971898F5F0E94B03112C0F60184817D
:1051100080628483968185E0989FC0011124958BDD
:10512000848B06C0F60184818F7D8483158A148A5E
:10513000F601868D9927807F9070803A910529F439
:105140000F2EF1E48F2EF02D0CC0F601868D9927DD
:10515000807F9070803B910521F40F2EF2E48F2E1A
:10516000F02DF601868D41A1682D8F700E940D3DB6
:10517000282FF6018785992783FD42C080FD40C016
:1051800090915209809110018917D0F5F1E09F1696
:10519000A9F5222399F5F6018781882389F584856D
:1051A000882371F58181803F59F587898F3F11F000
:1051B0008F5F878BF6018789863010F186898F5F34
:1051C000868B843158F4858D41A16A2D8F700E94A1
:1051D0008A3CF601178A83E0878312C0F601858D29
:1051E00041A16A2D8F700E948A3CF60187858160FB
:1051F000878789818F5F0E94E83102C0F601178A94
:10520000F601878580FF05C0809155098F5F8093E7
:105210005509F601878583FF05C0809153098F5F8B
:1052200080935309F60187858111B39489818F5F3B
:105230008983482F823208F457CECDC0809128044C
:10524000823009F0C8C019828981982F823208F013
:10525000C2C085E2989FC00111240F2EFEE2CF2E1E
:10526000F4E0DF2EF02DC80ED91EF601858D9927AA
:10527000807F9070803A910529F40F2EF1E4AF2ED3
:10528000F02D0CC0F601858D9927807F9070803BB2
:10529000910521F40F2EF2E4AF2EF02D40914E092E
:1052A0004423D1F0898199279C012F5F3F4F842FA0
:1052B00099272817390741F4F601858D41A16A2DF8
:1052C0008F700E943F3C0FC0F601858D41A16A2D71
:1052D0008F700E948A3C07C0F601858D41A16A2D1E
:1052E0008F700E943F3CF60182A18F3F09F46CC091
:1052F0000E94F1037C0100271127F601F4A2E3A22A
:105300008091270480FF1CC089819927FC01E85EF9
:10531000F64F80819927AA27BB278E159F05A007E6
:10532000B10724F0EE24FF2487010AC08981992760
:10533000FC01E85EF64F8081E81AF10801091109C5
:10534000F3E0EF16F1040105110574F180912704D3
:1053500081FF19C089819927880F991FFC01E65D9B
:10536000F64F808191819C0144275527C801B701E0
:105370000E94816520EE31E040E050E00E94F5653A
:1053800079018A0114C0C801B70128EB31E040E07F
:1053900050E00E94816520EE31E040E050E00E9444
:1053A000F56579018A0103C0EE24FF248701F60127
:1053B000F18AE08A80914F09909150098E0D9F1DCE
:1053C0009093500980934F0989818F5F8983982F2B
:1053D000823208F43ECFBB2031F4B0925409B0922F
:1053E0005509B09256090E941605982F80935109CD
:1053F00080912904891710F49093290420914F0972
:105400003091500980912A0490912B0482179307C0
:1054100020F430932B0420932A0421960FB6F8949D
:10542000DEBF0FBECDBFDF91CF911F910F91FF90D7
:10543000EF90DF90CF90BF90AF909F908F907F9034
:105440006F900895815099270895CF93DF93EC01D1
:10545000862F0E94222A833278F4282F332785E270
:1054600090E0289FA001299F500D389F500D1124D6
:10547000FA01E25DFB4FC683DF91CF910895EF9271
:10548000FF921F93CF937C01C0E080EC0E945C44AC
:105490008111C1E081EC0E945C448111C26082EC08
:1054A0000E945C448111C46081ED0E945C448111C2
:1054B000C86084EC0E945C448111C06185EC0E944C
:1054C0005C448111C06286EC0E945C448111C0641E
:1054D00087EC0E945C448111C06810E083EC0E945C
:1054E0005C44811111E082ED0E945C4481111260E4
:1054F00083ED0E945C4481111460F701C083118325
:10550000C0E081E00E9449118111C1E082E00E9467
:1055100049118111C26083E00E9449118111C46068
:1055200084E00E9449118111C86085E00E94491100
:105530008111C06186E00E9449118111C06287E03B
:105540000E9449118111C06488E00E9449118111B3
:10555000C068F701C283C0E089E00E94491181114F
:10556000C1E08AE00E9449118111C2608BE00E9473
:1055700049118111C4608CE00E9449118111C860F9
:105580008DE00E9449118111C0618EE00E94491195
:105590008111C0628FE00E9449118111C06480E1D5
:1055A0000E9449118111C068F701C383C0E081E105
:1055B0000E9449118111C1E082E10E9449118111CB
:1055C000C26083E10E9449118111C46084E10E949C
:1055D00049118111C86085E10E9449118111C061A2
:1055E00086E10E9449118111C06287E10E94491140
:1055F0008111C06488E10E9449118111C068F701DE
:10560000C483C0E089E10E9449118111C1E08AE1AF
:105610000E9449118111C2608BE10E9449118111E0
:10562000C4608CE10E9449118111C8608DE10E9423
:1056300049118111C0618EE10E9449118111C0623E
:105640008FE10E9449118111C06480E20E944911DA
:105650008111C068F701C583CF911F91FF90EF9032
:1056600008951F93CF93DF93182FEB010E94222AF6
:10567000482F833218F080E090E073C0992725E22C
:1056800030E0829FB001839F700D929F700D1124B6
:10569000FB01EE5CFB4F208122FD24C0FB01E25D9B
:1056A000FB4F8181803F71F485859685892B39F484
:1056B00021FD05C020FD03C0878585FF03C08FE065
:1056C000888335C0242F332785E290E0289FF0019E
:1056D000299FF00D389FF00D1124E25DFB4F818171
:1056E000888325C030E0232F5EE0259FC001112470
:1056F000DC01A956B64FFD018181813099F490E01B
:105700007FE060EFFD01E90FF11D8285841739F418
:1057100031E08C9182FF02C0788301C068839F5F73
:10572000943080F32F5F253010F43323F1F2242FCF
:10573000332785E290E0289FA001299F500D389FD4
:10574000500D1124FA01E25DFB4F87858983808922
:1057500091899C838B83812F0E9433328A8381E0DD
:1057600090E0DF91CF911F9108950E94222A833209
:1057700018F080E090E00895282F332785E290E02C
:10578000289FA001299F500D389F500D1124FA0128
:10579000E25DFB4F8181803F59F4FA01EE5CFB4FE3
:1057A000208121FD05C020FD03C081E090E0089527
:1057B00080E090E008950E94222A833218F080E071
:1057C00090E00895282F332785E290E0289FA001DC
:1057D000299F500D389F500D1124FA01E25DFB4FB7
:1057E0002785283011F0213019F481E090E00895E8
:1057F00080E090E00895FC0180914F09909150095C
:10580000918380838091510982838091520983839F
:10581000809153098483809154098583809155092F
:1058200086838091560987830895982F815082320C
:1058300038F485E2989FC0011124875F9B4F08953B
:1058400080E090E008959EEF81B1892381B982B113
:10585000892382B917B818B891EF8AB189238AB918
:105860008BB189238BB908950F930E94222A282F88
:10587000833168F000E0202F40E050E064EF7BE0EF
:1058800082E191E00E943D2F80E090E007C088E136
:1058900099E0FC01E20FF11D808199270F91089595
:1058A0000F930E94222A833168F000E0202F40E00D
:1058B00050E062E07CE082E191E00E943D2F80E6D2
:1058C00092E212C09927880F991FFC01E65DF64FFE
:1058D0002081318184E190E0289FA001299F500D13
:1058E000389F500D1124CA010F9108950F93CF9343
:1058F000DF93EB010E94222A833158F000E0202F31
:1059000040E050E061E17CE082E191E00E943D2FC7
:1059100012C099272AE239E0880F991FFC01E20F93
:10592000F31FCE0164E170E00E94AC657183608377
:10593000C9010E941C35DF91CF910F9108950E94FB
:10594000222A833118F080E090E00895282F332731
:1059500085E290E0289FA001299F500D389F500DAF
:105960001124FA01E25DFB4F8089918908950E941C
:10597000222A833118F080E090E00895282F332701
:1059800085E290E0289FA001299F500D389F500D7F
:105990001124FA01E25DFB4F83A194A10895809345
:1059A000270460934E0908951F93CF93C0E015E23A
:1059B000C19FC0011124FC01E25DFB4F82A18F3F1A
:1059C00041F00E94F1032C2F3327F901E85EF64FD6
:1059D0008083CF5FC23160F388E199E00E94FC349C
:1059E000CF911F910895CF9380912804833059F06F
:1059F00083E080932804C0E061E08C2F0E941F1A8E
:105A0000CF5FC232C8F3CF91089580919009882367
:105A100041F00E94122D0E943D2D8BE599E00E94DD
:105A20008A2D0895259A2D98269A2E988AEA809391
:105A3000800089E18093810010928500109284009B
:105A400080E395E090938700809386001092890010
:105A50001092880010928B0010928A0010928D0094
:105A600010928C0060E070E081E00E94682D60E0A0
:105A700070E082E00E94682D08951092900084E00A
:105A800080939100109295001092940010929700CC
:105A900010929600109299001092980010929B001C
:105AA00010929A0010929D0010929C00109258093A
:105AB0001092570910925A09109259098091690061
:105AC00088608093690010926A00E99AE19A0895CB
:105AD00099278230910581F0833091051CF401975C
:105AE00021F00895039779F00895872F99278093DF
:105AF0008900609388000895872F992780938B00F1
:105B000060938A000895872F992780938D00609372
:105B10008C000895FC01118210821382128285E0AC
:105B200090E09583848316820895EF92FF920F93FD
:105B30001F93CF93DF93EC018E81982F8F5F8E831D
:105B4000963068F060E375E081E00E94682D60E3C4
:105B500075E082E00E94682D86E08E8355C08A81C0
:105B60009B819C0144275527888199817C010027CE
:105B70001127DA01C901689412F8880F991FAA1F2A
:105B8000BB1F1694D1F7820F931FA41FB51F280FB8
:105B9000391F4A1F5B1FCA01B90125E830E040E008
:105BA00050E00E948165A80197010E94D365E90138
:105BB000C901845490408652944010F0C0E3D5E06F
:105BC00080919009882349F08091E804803F29F46E
:105BD000BE0181E00E94682D05C060E375E081E0B0
:105BE0000E94682D80919109882349F080911006C8
:105BF000803F29F4BE0182E00E94682D05C060E369
:105C000075E082E00E94682DDF91CF911F910F9186
:105C1000FF90EF9008951F920F920FB60F921124EC
:105C20002F933F938F939F9380919400282F332736
:105C3000322F2227809195009927282B392B80918C
:105C4000690099278C7090700C97E1F430935C098F
:105C500020935B09109294001092950080912C047F
:105C600090912D0490935E0980935D0910922D040C
:105C700010922C0410926109809169008B7F8093AF
:105C8000690010C08091690099278C709070089706
:105C900049F430932D0420932C0480916900846092
:105CA000809369009F918F913F912F910F900FBE2C
:105CB0000F901F901895CF93DF93CDB7DEB7239742
:105CC0000FB6F894DEBF0FBECDBFFE013196A0E83F
:105CD000B1E083E090E021E08030920719F40E9467
:105CE0004F6603C0182E0E944F6643E050E060E507
:105CF00071E0CE0101960E947654882391F00E94B3
:105D00009B2EE0E5F1E0A0E8B1E083E090E021E047
:105D10008030920719F40E94606603C0182E0E941A
:105D20006066279823960FB6F894DEBF0FBECDBFEE
:105D3000DF91CF910895CF93DF93CDB7DEB76E9704
:105D40000FB6F894DEBF0FBECDBF84E1FE013B96D7
:105D500011928A95E9F740E064E124E130E0522FA6
:105D6000FE013B96469FC0011124DC01AC57BE4F9B
:105D70002115310551F081E02030380719F40E94D7
:105D8000606603C0152E0E946066A8954F5F48307C
:105D900038F31982FE013196A3E8B1E081E090E08A
:105DA00021E08030920719F40E94606603C0182E2B
:105DB0000E9460666E960FB6F894DEBF0FBECDBF30
:105DC000DF91CF910895CF93DF93CDB7DEB72197C1
:105DD0000FB6F894DEBF0FBECDBFFE013196A3E82B
:105DE000B1E081E090E021E08030920719F40E9458
:105DF0004F6603C0182E0E944F668981893010F0CB
:105E000088E089838981992721960FB6F894DEBFAF
:105E10000FBECDBFDF91CF910895CF93DF93CDB764
:105E2000DEB764970FB6F894DEBF0FBECDBF9B01FF
:105E3000FE01319694E1899FD0011124A059BE4FF3
:105E400084E190E041E08030940719F40E944F66AD
:105E500003C0182E0E944F6684E1FE013196D901DD
:105E600001900D928A95E1F764960FB6F894DEBF23
:105E70000FBECDBFDF91CF9108956F927F928F9229
:105E80009F92AF92BF92CF92DF92EF92FF920F93C9
:105E90001F93CF93DF93CDB7DEB7A9970FB6F894D2
:105EA000DEBF0FBECDBF6C015B013A01022FFE01C8
:105EB000B996A3E8B1E081E090E021E0803092075C
:105EC00019F40E944F6603C0182E0E944F6689A5E0
:105ED000883008F0D4C09924FE01759684E1DF0172
:105EE0001D928A95E9F7B601CF010E947A65192DB6
:105EF00089A5981608F05EC00F2EF4E18F2EF02DC4
:105F00000F2EF4E1EF2EFF24F02DFE013196189DA7
:105F1000C0011124DC01AC57BE4FE114F10459F06B
:105F200020E0E21621E0F20619F40E944F6603C059
:105F30001E2C0E944F668D859E858A159B0599F5BE
:105F400046E050E0B601CE0101960E9476548823C7
:105F500051F5992493948F858A3008F090C0890D6B
:105F60008F87053008F004E0198A1A8A1B8A1C8A78
:105F7000802F9927AC01B301CE0141960E94636541
:105F8000FE013196189DD0011124AC57BE4F84E11B
:105F900090E021E08030920719F40E94606603C00F
:105FA000182E0E9460661F5F89A5181718F49920A3
:105FB00009F4ABCF992009F052C089A5883008F0C8
:105FC0004EC08F5F89A78CE0FE01319611928A95B1
:105FD000E9F7F60101900020E9F731972E2F2C19EF
:105FE0002C3008F02BE010E0121780F4AE014F5F68
:105FF0005F4F812F9927DC01A40FB51FF601E80F31
:10600000F91F80818C931F5F121798F3BE86AD86AF
:1060100081E08F87053008F004E0088B198A1A8A1E
:106020001B8A1C8A802F9927AC01B301CE014196AF
:106030000E946365FE01319699A584E1989FD00185
:106040001124A059BE4F84E190E021E080309207F6
:1060500019F40E94606603C0182E0E946066FE015B
:10606000B996A3E8B1E081E090E021E080309207AA
:1060700019F40E94606603C0182E0E946066A996FB
:106080000FB6F894DEBF0FBECDBFDF91CF911F9149
:106090000F91FF90EF90DF90CF90BF90AF909F90C7
:1060A0008F907F906F900895089582E1EAE8FEE076
:1060B00011928A95E9F780E1ECE9FEE011928A9568
:1060C000E9F7EEEBFEE0A8E8B0E082E190E021E045
:1060D0008030920719F40E944F6603C0182E0E9468
:1060E0004F66E0EDFEE0AAE9B0E082E190E021E059
:1060F0008030920719F40E944F6603C0182E0E9448
:106100004F66E2EEFEE0ACEAB0E080E190E021E034
:106110008030920719F40E944F6603C0182E0E9427
:106120004F66ECEAFEE0ADEBB0E082E190E021E00A
:106130008030920719F40E944F6603C0182E0E9407
:106140004F66E4EEF9E0A5E8B0E081E090E021E000
:106150008030920719F40E944F6603C0182E0E94E7
:106160004F66E5EEF9E0A6E8B0E082E090E021E0DD
:106170008030920719F40E944F660895182E0E94ED
:106180004F660895CF93DF93CDB7DEB762970FB612
:10619000F894DEBF0FBECDBFFE01319682E1DF0174
:1061A0001D928A95E9F7A8E8B0E082E190E021E04D
:1061B0008030920719F40E94606603C0182E0E9476
:1061C0006066FE013196AAE9B0E082E190E021E04C
:1061D0008030920719F40E94606603C0182E0E9456
:1061E0006066FE013196ACEAB0E080E190E021E02B
:1061F0008030920719F40E94606603C0182E0E9436
:106200006066FE013196ADEBB0E082E190E021E006
:106210008030920719F40E94606603C0182E0E9415
:1062200060660E94553062960FB6F894DEBF0FBECE
:10623000CDBFDF91CF9108950E94E01A982F8091F1
:10624000E409891790F49093E409E4EEF9E0A5E8F5
:10625000B0E081E090E021E08030920719F40E94E4
:10626000606603C0182E0E9460660E94DB1A9C01C3
:106270008091E5099091E60982179307A0F4309385
:10628000E6092093E509E5EEF9E0A6E8B0E082E052
:1062900090E021E08030920719F40E946066089532
:1062A000182E0E94606608958091E4099927089548
:1062B0008091E5099091E609089590E04AE85EE052
:1062C000292F3327F901E40FF51F808180FF17C0C4
:1062D0008E7F8083D901A857BF4FF901E254F14F57
:1062E0008081082E0E945466D901A656BF4FF9013D
:1062F000E053F14F8081082E0E9454660895E92FE3
:10630000FF27DF01A40FB51F8C9181FF0CC08D7F8B
:106310008C93DF01A354BF4FE455F14F8081082EC9
:106320000E94546608959F5F923150F290E02CE9EC
:106330003EE0E92FFF27DF01A20FB31F8C918130D0
:1063400059F41C92DF01A455BF4FEE51F14F8081EB
:10635000082E0E94546608959F5F903150F308956F
:10636000282F2150223198F58EEB9EE0FC01E20FA0
:10637000F11D3081832F9927929582958F708927FF
:106380009F7089278F30910514F5482F4F5F942F08
:106390009295907F832F8F70890F8083CB018370BC
:1063A0009070892B11F041E001C040E03327F901E2
:1063B000E053F14FCB019695879596958795840F7D
:1063C0008083F901E657F14F8081816080830895D1
:1063D000E82FE150E231C0F4FF27DF01A254B14FB2
:1063E0002C91822F99278F7090700F971CF5822F18
:1063F0008F708F5F922F907F890F8C93E657F14FAC
:1064000080818160808308958351803198F4E82FE2
:10641000FF27DF01AE51B14F2C91822F99278F704A
:1064200090700F973CF4822F8F5F8C93E456F14F5E
:1064300081E08083089581508231A0F4E82FFF2706
:10644000DF01A455B14F2C91822F99278F70907046
:106450000F9744F4822F8F5F8C93E657F14F808122
:10646000826080830895E82FE150E23188F42E2F76
:106470003327F901E254F14F8081882331F4F90187
:10648000E455F14F8081882391F081E090E00895F8
:10649000282F2351203158F482EE9EE0FC01E20FB8
:1064A000F11D8081882319F081E090E0089580E05B
:1064B00090E00895CF93DF93EC01FC0120E532E0FA
:1064C0008EE090E041E08030940721F4D9010E94F1
:1064D000606604C0D901182E0E946066CE01029643
:1064E000AC01698188810E94E41ADF91CF910895FF
:1064F000FC01A0E5B2E08EE090E021E08030920760
:1065000019F40E944F660895182E0E944F66089550
:10651000FC01A0E6B2E08FE190E021E0803092073C
:1065200019F40E9460660895182E0E94606608950E
:10653000FC01A0E6B2E08FE190E021E0803092071C
:1065400019F40E944F660895182E0E944F66089510
:10655000FC01ACE7BBE088E090E021E080309207EE
:1065600019F40E9460660895182E0E9460660895CE
:10657000FC01ACE7BBE088E090E021E080309207CE
:1065800019F40E944F660895182E0E944F660895D0
:106590000F93CF93DF93CDB7DEB721970FB6F89463
:1065A000DEBF0FBECDBF8983853060F000E021E003
:1065B000AE014F5F5F4F67E470E084E591E00E94B9
:1065C0003D2F15C0898199E1899FC0011124FB01EC
:1065D000DC01A252B14F89E190E021E080309207C6
:1065E00019F40E94606603C0182E0E94606621960E
:1065F0000FB6F894DEBF0FBECDBFDF91CF910F91E4
:1066000008950F93CF93DF93CDB7DEB721970FB6E1
:10661000F894DEBF0FBECDBF8983853060F000E007
:1066200021E0AE014F5F5F4F64E570E084E591E0EB
:106630000E943D2F15C0898199E1899FC0011124D5
:10664000FB01DC01A252B14F89E190E021E08030F2
:10665000920719F40E944F6603C0182E0E944F66DD
:1066600021960FB6F894DEBF0FBECDBFDF91CF915C
:106670000F9108950F93CF93DF93CDB7DEB7219796
:106680000FB6F894DEBF0FBECDBF8983803260F0B5
:1066900000E021E0AE014F5F5F4F60E670E084E50F
:1066A00091E00E943D2F14C0FB0199818CE2989FDC
:1066B000D0011124A659BC4F8CE290E021E080303B
:1066C000920719F40E94606603C0182E0E9460664B
:1066D00021960FB6F894DEBF0FBECDBFDF91CF91EC
:1066E0000F9108950F93CF93DF93CDB7DEB7219726
:1066F0000FB6F894DEBF0FBECDBF8983803260F045
:1067000000E021E0AE014F5F5F4F6AE670E084E594
:1067100091E00E943D2F14C0FB0199818CE2989F6B
:10672000D0011124A659BC4F8CE290E021E08030CA
:10673000920719F40E944F6603C0182E0E944F66FC
:1067400021960FB6F894DEBF0FBECDBFDF91CF917B
:106750000F9108950F93CF93DF93CDB7DEB72197B5
:106760000FB6F894DEBF0FBECDBF8983843160F0D1
:1067700000E021E0AE014F5F5F4F64E770E084E529
:1067800091E00E943D2F14C0FB01998188E1989F00
:10679000D0011124A451B74F88E190E021E080306E
:1067A000920719F40E94606603C0182E0E9460666A
:1067B00021960FB6F894DEBF0FBECDBFDF91CF910B
:1067C0000F9108950F93CF93DF93CDB7DEB7219745
:1067D0000FB6F894DEBF0FBECDBF8983843160F061
:1067E00000E021E0AE014F5F5F4F6EE770E084E5AF
:1067F00091E00E943D2F14C0FB01998188E1989F90
:10680000D0011124A451B74F88E190E021E08030FD
:10681000920719F40E944F6603C0182E0E944F661B
:1068200021960FB6F894DEBF0FBECDBFDF91CF919A
:106830000F910895CF93DF93CDB7DEB769970FB669
:10684000F894DEBF0FBECDBFFC01862F815082328F
:1068500018F080E090E02AC06150808189838181B6
:106860008A8382818B8383818C83878188878789D0
:10687000888F808D898F848195819E838D83868189
:106880008F83DF0118968FE0FE0139960D900192FB
:106890008A95E1F789E1689FC00111248457944FDC
:1068A000BC01CE0101960E94EB34992769960FB680
:1068B000F894DEBF0FBECDBFDF91CF9108950F9347
:1068C0001F93CF93DF93CDB7DEB769970FB6F894D8
:1068D000DEBF0FBECDBF8C01962F91509232B0F526
:1068E00089E1989FC00111249E012F5F3F4FDC0179
:1068F000A457B44F89E190E041E08030940721F43F
:10690000F9010E944F6604C0F901182E0E944F66DB
:106910008981F80180838A8181838B8182838C8144
:10692000838388858783888D878B898D808F8D81F0
:106930009E81958384838F818683D80118968FE00A
:10694000FE01399601900D928A95E1F769960FB68E
:10695000F894DEBF0FBECDBFDF91CF911F910F9195
:10696000089581508B30C8F4FB01A82FBB27CD01BF
:1069700082959295907F9827807F9827DC01A45379
:10698000B54F80E190E021E08030920719F40E9439
:1069900060660895182E0E946066089581508B30BD
:1069A000C8F4FB01A82FBB27CD0182959295907F5B
:1069B0009827807F9827DC01A453B54F80E190E0B1
:1069C00021E08030920719F40E944F660895182E36
:1069D0000E944F660895FC01DB0189E190E021E00F
:1069E0008030920719F40E94606603C0182E0E943E
:1069F000606681E090E00895FC01A0E1B0E082E1F2
:106A000090E021E08030920719F40E9460660895BA
:106A1000182E0E9460660895FC01A0E1B0E082E1BA
:106A200090E021E08030920719F40E944F660895AB
:106A3000182E0E944F660895FC01A0E3B0E084E2A6
:106A400090E021E08030920719F40E94606608957A
:106A5000182E0E9460660895FC01A0E3B0E084E275
:106A600090E021E08030920719F40E944F6608956B
:106A7000182E0E944F660895FC01A0E8B2E088E15C
:106A800090E021E08030920719F40E94606608953A
:106A9000182E0E9460660895FC01A0E8B2E088E12B
:106AA00090E021E08030920719F40E944F6608952B
:106AB000182E0E944F6608950F93FC018081882351
:106AC00019F488E992E016C08081813019F48EEDC6
:106AD00092E010C08081823019F484E293E00AC011
:106AE00000E021E0AF0167E471E084E591E00E94FD
:106AF0003D2F0DC0DC0186E490E021E0803092075C
:106B000019F40E94606603C0182E0E9460660F91FF
:106B100008950F93CF93DF93CDB7DEB721970FB6CC
:106B2000F894DEBF0FBECDBF8983882319F488E9AE
:106B300092E018C08981813019F48EED92E012C084
:106B40008981823019F484E293E00CC000E021E0F6
:106B5000AE014F5F5F4F60E671E084E591E00E9417
:106B60003D2F0EC0FB01DC0186E490E021E0803087
:106B7000920719F40E944F6603C0182E0E944F66B8
:106B800021960FB6F894DEBF0FBECDBFDF91CF9137
:106B90000F910895CF93DF93CDB7DEB760970FB60F
:106BA000F894DEBF0FBECDBFFE013196A0E0B0E08D
:106BB00080E190E021E08030920719F40E944F6656
:106BC00003C0182E0E944F668B858F3119F48FE118
:106BD00090E008C08B85803219F480E290E002C01A
:106BE0008FE190E060960FB6F894DEBF0FBECDBF88
:106BF000DF91CF9108950F931F93CF93DF93CDB77C
:106C0000DEB76E970FB6F894DEBF0FBECDBFFE01A4
:106C10003196A0E0B0E084E090E021E0803092077F
:106C200019F40E944F6603C0182E0E944F6644E07C
:106C300050E068E671E0CE0101960E947654882308
:106C400009F44DC08E010F5F1F4F8EE1D8011D92D8
:106C50008A95E9F785E0E8E6F1E0D80101900D9228
:106C60008A95E1F71D821E821F82188619861A8670
:106C70001B860E94F41DF801A0E0B0E080E190E0E6
:106C800021E08030920719F40E94606603C0182E3C
:106C90000E946066FE01319684E1DF011D928A95B3
:106CA000E9F7AAEDBFE084E190E021E080309207AF
:106CB00019F40E94606603C0182E0E946066FE01EF
:106CC0003196A0E0B0E084E090E021E080309207CF
:106CD00019F40E94606603C0182E0E946066FE01CF
:106CE0003196A0E3B2E08AE090E021E080309207A4
:106CF00019F40E944F6603C0182E0E944F664AE0A6
:106D000050E064E871E0CE0101960E947654882339
:106D100079F10E94141E0E94DD100E9449560E94C3
:106D200037060E945B0FFE0131968EE1DF011D9256
:106D30008A95E9F7AEE5BFE080E190E021E08030A0
:106D4000920719F40E94606603C0182E0E946066C4
:106D5000E4E8F1E0A0E3B2E08AE090E021E08030F6
:106D6000920719F40E94606603C0182E0E946066A4
:106D7000FE013196A0E8B1E083E090E021E08030B0
:106D8000920719F40E944F6603C0182E0E944F66A6
:106D900043E050E06DE671E0CE0101960E9476542A
:106DA000882391F00E949B2EEDE6F1E0A0E8B1E08F
:106DB00083E090E021E08030920719F40E94606641
:106DC00003C0182E0E946066FE013196A0E8B0E074
:106DD00085E090E021E08030920719F40E944F6630
:106DE00003C0182E0E944F6645E050E061E771E055
:106DF000CE0101960E947654882309F475C0FE01E5
:106E000031968EE1DF011D928A95E9F7ACEBB0E097
:106E100081E090E021E08030920719F40E946066E2
:106E200003C0182E0E946066FE013196A5E8B0E00E
:106E300081E090E021E08030920719F40E946066C2
:106E400003C0182E0E946066FE013196A6E8B0E0ED
:106E500082E090E021E08030920719F40E946066A1
:106E600003C0182E0E946066FE013196A8E8B0E0CB
:106E700082E190E021E08030920719F40E94606680
:106E800003C0182E0E946066FE013196ACEAB0E0A5
:106E900080E190E021E08030920719F40E94606662
:106EA00003C0182E0E946066FE013196ADEBB0E083
:106EB00082E190E021E08030920719F40E94606640
:106EC00003C0182E0E946066E1E7F1E0A0E8B0E0A0
:106ED00085E090E021E08030920719F40E9460661E
:106EE00003C0182E0E946066FE013196AAEDBFE035
:106EF00089E090E021E08030920731F40E944F66F3
:106F000006C00E94606630C0182E0E944F6690E056
:106F10009E012F5F3F4F8981181634F5AE014F5FF8
:106F20005F4FF901E90FF11D808180538A3090F0A5
:106F300089E0F90111928A95E9F7F901AAEDBFE01C
:106F400089E090E021E080309207D9F2182E0E946B
:106F500060660AC09F5F983038F49A01FA01E90F21
:106F6000F11D80811816ECF2FE013196A3EEBFE010
:106F700089E090E021E08030920731F40E944F6672
:106F800006C00E94606630C0182E0E944F6690E0D6
:106F90009E012F5F3F4F8981181634F5AE014F5F78
:106FA0005F4FF901E90FF11D808180538A3090F025
:106FB00089E0F90111928A95E9F7F901A3EEBFE0A2
:106FC00089E090E021E080309207D9F2182E0E94EB
:106FD00060660AC09F5F983038F49A01FA01E90FA1
:106FE000F11D80811816ECF26E960FB6F894DEBF94
:106FF0000FBECDBFDF91CF911F910F910895CFEFBD
:10700000D0E1DEBFCDBF0E9469530E94393A0E9491
:10701000061B0E9462050E947B530E94A8450E94A5
:107020005B2E0E94FB35E5E6FEE0A0E7B0E08FE0D6
:1070300090E021E08030920719F40E944F6603C06F
:10704000182E0E944F668091650E9091660E8A3FC1
:10705000910531F18B3F910538F48436910561F04B
:107060008D37910599F039C021E0843F920711F1E5
:10707000885E934049F131C086E28093E20084E06B
:107080008093E30083E18093E40027C08EE1809346
:10709000E20084E08093E30083E18093E4001DC07C
:1070A0008EE08093E20084E08093E30083E18093AC
:1070B000E40013C086E08093E20084E08093E30064
:1070C00083E18093E40009C082E08093E20084E0E1
:1070D0008093E30083E18093E4000E94920F80910B
:1070E000670E9091680E059738F485E090E09093D4
:1070F000680E8093670E0DC08091670E9091680EA8
:10710000815D974030F080ED97E09093680E80931A
:10711000670E8091690E90916A0E28E08030920788
:1071200038F08959994021F010926A0E1092690E38
:107130008091710E80FF04C082E08093760E02C0C1
:107140001092760E8091710E81FF04C082E08093D0
:10715000770E02C01092770E8091720E8A50813F96
:1071600018F08FE48093720E0E944B3D0E94F855F8
:107170000E947C1F0E94ED4487E00E94DF5F7894AC
:107180000E94D051A89580E00E9402450E94B3451C
:10719000FACF1F93162FA398992787709070880FA6
:1071A000991F81640E947453812F0E94745380E060
:1071B0000E947453A39A99271F9108950F931F93C8
:1071C000162F042FA398992787709070880F991F06
:1071D00080640E947453812F0E947453802F0E94F8
:1071E0007453A39A1F910F9108951F93CF93C09149
:1071F000E709CC2389F511E01093E7094CE16AE037
:107200008C2F0E94DE384C2F6C2F8C2F0E94DE3882
:107210004FEF612F8C2F0E94DE384C2F62E08C2FB5
:107220000E94DE384C2F63E08C2F0E94DE384C2FFA
:1072300064E08C2F0E94DE384C2F65E08C2F0E947A
:10724000DE384C2F6CE08C2F0E94DE384C2F6DE026
:107250008C2F0E94DE380AC1C091E709C13089F540
:107260004CE16AE08C2F0E94DE3840E0642F8C2FC6
:107270000E94DE384FEF6C2F8C2F0E94DE3840E0EA
:1072800062E08C2F0E94DE3840E063E08C2F0E9489
:10729000DE3840E064E08C2F0E94DE3840E065E09C
:1072A0008C2F0E94DE3840E06CE08C2F0E94DE388C
:1072B00040E06DE08C2F0E94DE3882E08093E70989
:1072C000D5C0C091E709C23089F54CE16AE08C2F46
:1072D0000E94DE3840E0642F8C2F0E94DE384FEF92
:1072E00061E08C2F0E94DE3840E06C2F8C2F0E94D2
:1072F000DE3840E063E08C2F0E94DE3840E064E03E
:107300008C2F0E94DE3840E065E08C2F0E94DE3832
:1073100040E06CE08C2F0E94DE3840E06DE08C2F66
:107320000E94DE3883E08093E709A0C0C091E7099E
:10733000C33089F54CE16AE08C2F0E94DE3840E0D2
:10734000642F8C2F0E94DE384FEF61E08C2F0E945B
:10735000DE3840E062E08C2F0E94DE3840E06C2F87
:107360008C2F0E94DE3840E064E08C2F0E94DE38D3
:1073700040E065E08C2F0E94DE3840E06CE08C2F0E
:107380000E94DE3840E06DE08C2F0E94DE3884E001
:107390008093E7096BC0C091E709C43089F54CE1DF
:1073A0006AE08C2F0E94DE384CEF60E08C2F0E9448
:1073B000DE384FEF61E08C2F0E94DE3840E062E063
:1073C0008C2F0E94DE3840E063E08C2F0E94DE3874
:1073D00040E06C2F8C2F0E94DE3840E065E08C2F5F
:1073E0000E94DE3840E06CE08C2F0E94DE3840E0E6
:1073F0006DE08C2F0E94DE3885E08093E70936C06F
:10740000C091E709C53081F54CE16AE08C2F0E94FC
:10741000DE3840E0642F8C2F0E94DE3840EF61E0C0
:107420008C2F0E94DE3840E062E08C2F0E94DE3814
:1074300040E063E08C2F0E94DE3840E064E08C2F57
:107440000E94DE3840E06C2F8C2F0E94DE3840E036
:107450006CE08C2F0E94DE3840E06DE08C2F0E94A3
:10746000DE381092E70902C01092E709CF911F9110
:1074700008959B9AA39A4CE16AE080E00E94DE386E
:1074800040E064E1842F0E94DE3840E0642F842FC6
:107490000E94DE384FEF61E080E00E94DE3840E07D
:1074A00062E0842F0E94DE3840E063E0842F0E9477
:1074B000DE3840E064E0842F0E94DE3840E065E082
:1074C000842F0E94DE3840E06CE0842F0E94DE387A
:1074D00040E06DE0842F0E94DE384CE16AE081E0FC
:1074E0000E94DE3840E064E181E00E94DE3840E046
:1074F000642F81E00E94DE384FEF61E0862F0E940A
:10750000DE3840E062E081E00E94DE3840E063E087
:1075100081E00E94DE3840E064E081E00E94DE38D5
:1075200040E065E081E00E94DE3840E06CE081E010
:107530000E94DE3840E06DE081E00E94DE384CE1E0
:107540006AE082E00E94DE3840E064E182E00E946E
:10755000DE3840E0642F82E00E94DE384FEF61E0C9
:1075600082E00E94DE3840E062E0862F0E94DE3832
:1075700040E063E082E00E94DE3840E064E082E0C8
:107580000E94DE3840E065E082E00E94DE3840E0A4
:107590006CE082E00E94DE3840E06DE082E00E9414
:1075A000DE384CE16AE083E00E94DE3840E064E1CE
:1075B00083E00E94DE3840E0642F83E00E94DE38E2
:1075C0004FEF61E083E00E94DE3840E062E083E05C
:1075D0000E94DE3840E063E0862F0E94DE3840E003
:1075E00064E083E00E94DE3840E065E083E00E94D2
:1075F000DE3840E06CE083E00E94DE3840E06DE081
:1076000083E00E94DE384CE16AE084E00E94DE38CC
:1076100040E064E184E00E94DE384CEF60E084E00A
:107620000E94DE384FEF61E084E00E94DE3840E0E7
:1076300062E084E00E94DE3840E063E084E00E9483
:10764000DE3840E064E0862F0E94DE3840E065E0EE
:1076500084E00E94DE3840E06CE084E00E94DE3886
:1076600040E06DE084E00E94DE384CE16AE085E0B5
:107670000E94DE3840E064E185E00E94DE3840E0B0
:1076800065E185E00E94DE3840E0642F85E00E94DD
:10769000DE3840EF61E085E00E94DE3840E062E0E5
:1076A00085E00E94DE3840E063E085E00E94DE383D
:1076B00040E064E085E00E94DE3840E065E0862F2F
:1076C0000E94DE3840E06CE085E00E94DE3840E059
:1076D0006DE085E00E94DE3808950F931F93CF93ED
:1076E000082FC62F142F20E030E0613611F421E07E
:1076F00030E080E090E0C13411F481E090E0822B32
:10770000932B892B91F060E0812F0E94C93821E0F2
:1077100030E0002E02C0220F331F0A94E2F7482FF8
:10772000422B60E0812F0E94DE3820E030E0C2363C
:1077300011F421E030E080E090E0C23411F481E007
:1077400090E0822B932B892B89F061E0812F0E949E
:10775000C93821E030E002C0220F331F0A95E2F75A
:10776000482F422B61E0812F0E94DE38CF911F917C
:107770000F9108950F931F93CF93082FC62F142FA7
:1077800020E030E0613611F421E030E080E090E06C
:10779000C13411F481E090E0822B932B892BA1F06E
:1077A00060E0812F0E94C93821E030E0002E02C045
:1077B000220F331F0A94E2F7922F9095482F492306
:1077C00060E0812F0E94DE3820E030E0C23611F404
:1077D00021E030E080E090E0C23411F481E090E0FC
:1077E000822B932B892B99F061E0812F0E94C9385D
:1077F00021E030E002C0220F331F0A95E2F7922FFA
:107800009095482F492361E0812F0E94DE38CF9167
:107810001F910F9108950F931F93CF93182FC62F89
:10782000042F20E030E0613611F421E030E080E008
:1078300090E0C13411F481E090E0822B932B892BEE
:1078400029F0412F64E1802F0E94DE3820E030E0F3
:10785000C23611F421E030E080E090E0C23411F44F
:1078600081E090E0822B932B892B29F0412F65E159
:10787000802F0E94DE38CF911F910F9108950F93B2
:107880001F93CF93082FC62F142F50E020E030E035
:10789000613611F421E030E080E090E0C13411F471
:1078A00081E090E0822B932B892B71F062E1812F94
:1078B0000E94C93821E030E0002E02C0220F331FA1
:1078C0000A94E2F7582F522B20E030E0C23611F430
:1078D00021E030E080E090E0C23411F481E090E0FB
:1078E000822B932B892B69F063E1812F0E94C93889
:1078F00021E030E002C0220F331F0A95E2F7582F33
:10790000522B412F6C2F852F0E940B3CCF911F9142
:107910000F9108950F931F93CF93082FC62F142F05
:1079200050E020E030E0613611F421E030E080E00A
:1079300090E0C13411F481E090E0822B932B892BED
:1079400081F062E1812F0E94C93821E030E0002EF1
:1079500002C0220F331F0A94E2F7922F9095582FFE
:10796000592320E030E0C23611F421E030E080E01D
:1079700090E0C23411F481E090E0822B932B892BAC
:1079800079F063E1812F0E94C93821E030E002C024
:10799000220F331F0A95E2F7922F9095582F592303
:1079A000412F6C2F852F0E940B3CCF911F910F917F
:1079B00008951F93CF93C82F162F40E020E030E0AA
:1079C000813611F421E030E080E090E0C13411F420
:1079D00081E090E0822B932B892B29F062E1812FAB
:1079E0000E94C938482F20E030E0C23611F421E06F
:1079F00030E080E090E0C23411F481E090E0822B2E
:107A0000932B892B29F063E1812F0E94C938482FDD
:107A1000842F9927CF911F9108950F931F93CF9390
:107A2000182FC62F042F40E020E030E0613611F41B
:107A300021E030E080E090E0C13411F481E090E09A
:107A4000822B932B892B29F062E1802F0E94C93869
:107A5000482F20E030E0C23611F421E030E080E031
:107A600090E0C23411F481E090E0822B932B892BBB
:107A700029F063E1802F0E94C938482F81E090E00F
:107A800002C0880F991F1A95E2F784239927CF9196
:107A90001F910F9108950E94341485E49AE0909309
:107AA000DC0A8093DB0A1092DD0A1092D40A10924D
:107AB000D50A84ED9AE00E943C148823D1F71092F5
:107AC000D30A8DE49AE09093E80A8093E70A109233
:107AD000E90A1092E00A1092E10A80EE9AE00E9410
:107AE0003C148823D1F71092DF0A85E59AE0909341
:107AF000F40A8093F30A1092F50A1092EC0A10929D
:107B0000ED0A8CEE9AE00E943C148823D1F7109283
:107B1000EB0A8DE59AE09093000B8093FF0A109298
:107B2000010B1092F80A1092F90A88EF9AE00E946D
:107B30003C148823D1F71092F70A85EF99E09093CF
:107B40006D0A80936C0A10926E0A1092650A82E0A8
:107B50008093660A85E69AE00E943C148823D1F758
:107B60008DEF99E09093780A8093770A1092790AC2
:107B70001092700A82E08093710A80E79AE00E9476
:107B80003C148823D1F785E09AE09093830A809390
:107B9000820A1092840A10927B0A82E080937C0A07
:107BA0008BE79AE00E943C148823D1F78DE09AE09D
:107BB00090938E0A80938D0A10928F0A1092860AF3
:107BC00082E08093870A86E89AE00E943C1488232A
:107BD000D1F785E19AE09093990A8093980A1092E0
:107BE0009A0A1092910A82E08093920A81E99AE0BF
:107BF0000E943C148823D1F78DE19AE09093A40A67
:107C00008093A30A1092A50A10929C0A82E08093A6
:107C10009D0A8CE99AE00E943C148823D1F785E202
:107C20009AE09093AF0A8093AE0A1092B00A109235
:107C3000A70A82E08093A80A87EA9AE00E943C148F
:107C40008823D1F78DE29AE09093BA0A8093B90A1B
:107C50001092BB0A1092B20A82E08093B30A82EBC0
:107C60009AE00E943C148823D1F785E39AE0909330
:107C7000C50A8093C40A1092C60A1092BD0A82E017
:107C80008093BE0A8DEB9AE00E943C148823D1F7C2
:107C90008DE39AE09093D00A8093CF0A1092D10A94
:107CA0001092C80A82E08093C90A88EC9AE00E9488
:107CB0003C148823D1F708958091D30A8823E1F0FA
:107CC0008091D30A813059F483ED9AE001960E94A5
:107CD0003C14882389F482E08093D30A0DC08091FC
:107CE000D30A823049F483ED9AE001960E944E1542
:107CF000882311F48093D30A8091DF0A8823E1F06E
:107D00008091DF0A813059F48FED9AE001960E944C
:107D10003C14882389F482E08093DF0A0DC08091AF
:107D2000DF0A823049F48FED9AE001960E944E15E9
:107D3000882311F48093DF0A8091EB0A8823E1F015
:107D40008091EB0A813059F48BEE9AE001960E9403
:107D50003C14882389F482E08093EB0A0DC0809163
:107D6000EB0A823049F48BEE9AE001960E944E15A0
:107D7000882311F48093EB0A8091F70A8823E1F0BD
:107D80008091F70A813059F487EF9AE001960E94BA
:107D90003C14882389F482E08093F70A0895809147
:107DA000F70A823049F487EF9AE001960E944E1557
:107DB000882311F48093F70A0895CF93DF93EC01A1
:107DC00085E69AE00E944E15882309F046C080910E
:107DD000670A9091680AAA27BB2788839983AA8398
:107DE000BB83E0916C0AF0916D0A80818D83E091F4
:107DF0006C0AF0916D0A81818E83E0916C0AF0919A
:107E00006D0A82818F83E0916C0AF0916D0A838103
:107E10008887E0916C0AF0916D0A84818987E091EE
:107E20006C0AF0916D0A85818A87E0916C0AF09165
:107E30006D0A86818B87E0916C0AF0916D0A8781CB
:107E40008C8780916B0A8C8385E69AE00E943C14B3
:107E50008823D1F781E090E0BBC280E79AE00E94DE
:107E60004E15882309F046C08091720A9091730ADA
:107E7000AA27BB2788839983AA83BB83E091770ACB
:107E8000F091780A80818D83E091770AF091780AE9
:107E900081818E83E091770AF091780A82818F83C5
:107EA000E091770AF091780A83818887E091770AD8
:107EB000F091780A84818987E091770AF091780AB5
:107EC00085818A87E091770AF091780A86818B878D
:107ED000E091770AF091780A87818C878091760A01
:107EE0008C8380E79AE00E943C148823D1F781E0DC
:107EF00090E06EC28BE79AE00E944E15882309F04D
:107F000046C080917D0A90917E0AAA27BB2788836C
:107F10009983AA83BB83E091820AF091830A8081CE
:107F20008D83E091820AF091830A81818E83E091B2
:107F3000820AF091830A82818F83E091820AF09114
:107F4000830A83818887E091820AF091830A848181
:107F50008987E091820AF091830A85818A87E0917E
:107F6000820AF091830A86818B87E091820AF091E0
:107F7000830A87818C878091810A8C838BE79AE0C2
:107F80000E943C148823D1F781E090E021C286E86A
:107F90009AE00E944E15882309F046C08091880A15
:107FA0009091890AAA27BB2788839983AA83BB83D8
:107FB000E0918D0AF0918E0A80818D83E0918D0A87
:107FC000F0918E0A81818E83E0918D0AF0918E0A64
:107FD00082818F83E0918D0AF0918E0A8381888758
:107FE000E0918D0AF0918E0A84818987E0918D0A53
:107FF000F0918E0A85818A87E0918D0AF0918E0A30
:1080000086818B87E0918D0AF0918E0A87818C871B
:1080100080918C0A8C8386E89AE00E943C14882325
:10802000D1F781E090E0D4C181E99AE00E944E1539
:10803000882309F046C08091930A9091940AAA2758
:10804000BB2788839983AA83BB83E091980AF09128
:10805000990A80818D83E091980AF091990A818133
:108060008E83E091980AF091990A82818F83E09142
:10807000980AF091990A83818887E091980AF09193
:10808000990A84818987E091980AF091990A8581FB
:108090008A87E091980AF091990A86818B87E0910E
:1080A000980AF091990A87818C878091970A8C832E
:1080B00081E99AE00E943C148823D1F781E090E0A6
:1080C00087C18CE99AE00E944E15882309F046C0CA
:1080D00080919E0A90919F0AAA27BB278883998343
:1080E000AA83BB83E091A30AF091A40A80818D83C7
:1080F000E091A30AF091A40A81818E83E091A30A02
:10810000F091A40A82818F83E091A30AF091A40ADE
:1081100083818887E091A30AF091A40A84818987EA
:10812000E091A30AF091A40A85818A87E091A30ACD
:10813000F091A40A86818B87E091A30AF091A40AAA
:1081400087818C878091A20A8C838CE99AE00E94B7
:108150003C148823D1F781E090E03AC187EA9AE0A5
:108160000E944E15882309F046C08091A90A90917B
:10817000AA0AAA27BB2788839983AA83BB83E09195
:10818000AE0AF091AF0A80818D83E091AE0AF09142
:10819000AF0A81818E83E091AE0AF091AF0A8281AD
:1081A0008F83E091AE0AF091AF0A83818887E091D6
:1081B000AE0AF091AF0A84818987E091AE0AF0910E
:1081C000AF0A85818A87E091AE0AF091AF0A868175
:1081D0008B87E091AE0AF091AF0A87818C878091FE
:1081E000AD0A8C8387EA9AE00E943C148823D1F779
:1081F00081E090E0EDC082EB9AE00E944E1588236A
:1082000009F046C08091B40A9091B50AAA27BB270D
:1082100088839983AA83BB83E091B90AF091BA0A53
:1082200080818D83E091B90AF091BA0A81818E83B1
:10823000E091B90AF091BA0A82818F83E091B90A7C
:10824000F091BA0A83818887E091B90AF091BA0A5D
:1082500084818987E091B90AF091BA0A85818A8779
:10826000E091B90AF091BA0A86818B87E091B90A48
:10827000F091BA0A87818C878091B80A8C8382EB4F
:108280009AE00E943C148823D1F781E090E0A0C0DE
:108290008DEB9AE00E944E15882309F046C080912C
:1082A000BF0A9091C00AAA27BB2788839983AA8313
:1082B000BB83E091C40AF091C50A80818D83E0916F
:1082C000C40AF091C50A81818E83E091C40AF091BD
:1082D000C50A82818F83E091C40AF091C50A838127
:1082E0008887E091C40AF091C50A84818987E0916A
:1082F000C40AF091C50A85818A87E091C40AF09189
:10830000C50A86818B87E091C40AF091C50A8781EE
:108310008C878091C30A8C838DEB9AE00E943C1479
:108320008823D1F781E090E053C088EC9AE00E9466
:108330004E15882309F046C08091CA0A9091CB0A55
:10834000AA27BB2788839983AA83BB83E091CF0A9E
:10835000F091D00A80818D83E091CF0AF091D00A0C
:1083600081818E83E091CF0AF091D00A82818F8340
:10837000E091CF0AF091D00A83818887E091CF0AFB
:10838000F091D00A84818987E091CF0AF091D00AD8
:1083900085818A87E091CF0AF091D00A86818B8708
:1083A000E091CF0AF091D00A87818C878091CE0A24
:1083B0008C8388EC9AE00E943C148823D1F781E0FA
:1083C00090E006C0188219821A821B8280E090E039
:1083D000DF91CF910895CF93DF93DC018091D30A91
:1083E000882339F483ED9AE09093040B8093030B78
:1083F00021C08091DF0A882339F48FED9AE09093B1
:10840000040B8093030B16C08091EB0A882339F488
:108410008BEE9AE09093040B8093030B0BC080913A
:10842000F70A882309F072C087EF9AE09093040B53
:108430008093030BE091030BF091040B0084F18512
:10844000E02DED018D818083E091030BF091040B11
:108450000084F185E02D8E818183E091030BF09102
:10846000040B0084F185E02D8F818283E091030B62
:10847000F091040B0084F185E02D88858383E091E1
:10848000030BF091040B0084F185E02D8985848332
:10849000E091030BF091040B0084F185E02D8A85B7
:1084A0008583E091030BF091040B0084F185E02DAE
:1084B0008B858683E091030BF091040B0084F1859A
:1084C000E02D8C858783E091030BF091040B8C8168
:1084D0008783E091030BF091040B8D919C91948321
:1084E0008383E091030BF091040B1286E091030B60
:1084F000F091040B1182E091030BF091040B1282B6
:10850000E091030BF091040B81E08083DF91CF9128
:10851000089588EE99E00E94DD3E882361F188EE9F
:1085200099E00E94DA1188EE99E00E94DD3E8823EE
:1085300011F188EE99E00E94DA1188EE99E00E942C
:10854000DD3E8823C1F088EE99E00E94DA1188EEC2
:1085500099E00E94DD3E882371F088EE99E00E9448
:10856000DA1188EE99E00E94DD3E882321F088EE42
:1085700099E00E94DA110895FF920F931F93CF9311
:10858000DF93CDB7DEB760970FB6F894DEBF0FBEAE
:10859000CDBF20E0822F99278C010B5F144FF8018B
:1085A00080818C7F8083F22EF394BE016F5F7F4FBA
:1085B0008F2D0E94CE3488898170982F990F990F42
:1085C000990FF80180818370892B80832F2D2B30A8
:1085D00008F360960FB6F894DEBF0FBECDBFDF91F3
:1085E000CF911F910F91FF900895FC0180818370BE
:1085F0009927009719F0019731F0089580818D72C5
:108600008162808308959081892F807FA1F493FDFA
:1086100005C0892F8E7F866080830895808182FFC8
:1086200003C08B7F808303C08081846080838081CE
:108630008C7F826080830895FC01808183709927FC
:1086400081309105BCF0833091051CF0039731F027
:10865000089580818F708362808308959081892F2F
:10866000807F41F4892F8C7F808393FD03C0892F05
:10867000887F808308959927853C910509F457C028
:10868000863C9105ACF4823C9105C9F1833C91058F
:108690003CF4803C910519F1813C910541F17AC08F
:1086A000833C910509F45EC0843C9105C1F172C020
:1086B000813D910561F1823D910544F4863C91052F
:1086C000F1F1873C910509F442C064C0823D9105F7
:1086D00009F450C0833D910509F454C05BC0309B40
:1086E00003C081E090E0089580E090E00895319922
:1086F00003C081E090E0089580E090E00895329911
:1087000003C081E090E0089580E090E008954999E9
:1087100003C081E090E0089580E090E008953499EE
:1087200003C081E090E0089580E090E008953599DD
:1087300003C081E090E0089580E090E008953699CC
:1087400003C081E090E0089580E090E0089586B154
:10875000992787FD9095809590958827990F881F78
:1087600099270895339903C081E090E0089580E04F
:1087700090E008954A9903C081E090E0089580E078
:1087800090E008954B9903C081E090E0089580E067
:1087900090E0089580E090E0089530E0832F9927DD
:1087A000FC01EB5FF44F2081822F807F41F0822F0C
:1087B000807F982F9051822F8F70892B80833F5F0D
:1087C0003B3060F3E5E0FBE0309B04C0CF010E944A
:1087D000F54203C0CF010E941C43E6E0FBE0319963
:1087E00004C0CF010E94F54203C0CF010E941C4388
:1087F000E7E0FBE0329904C0CF010E94F54203C0DC
:10880000CF010E941C43E8E0FBE0499904C0CF017E
:108810000E94F54203C0CF010E941C43E9E0FBE047
:10882000349904C0CF010E94F54203C0CF010E94D9
:108830001C43EAE0FBE0359904C0CF010E94F542F9
:1088400003C0CF010E941C43EBE0FBE0369904C05B
:10885000CF010E94F54203C0CF010E941C43ECE00F
:10886000FBE0379904C0CF010E94F54203C0CF015D
:108870000E941C43EDE0FBE0339904C0CF010E944D
:10888000F54203C0CF010E941C43EEE0FBE04A9991
:1088900004C0CF010E94F54203C0CF010E941C43D7
:1088A000EFE0FBE04B9904C0CF010E94F542089530
:1088B000CF010E941C4308959927853C910509F436
:1088C00051C0863C9105ACF4823C9105B1F1833CEA
:1088D00091053CF4803C910511F1813C910531F109
:1088E0006BC0833C910509F452C0843C910599F119
:1088F00063C0813D910541F1823D91053CF4863C88
:108900009105B9F1873C9105D9F156C0823D910599
:1089100009F444C0833D910509F447C04DC08091DE
:10892000050B869586958170992708958091060B91
:10893000869586958170992708958091070B869575
:1089400086958170992708958091080B8695869564
:108950008170992708958091090B8695869581707D
:108960009927089580910A0B86958695817099279D
:10897000089580910B0B86958695817099270895AF
:1089800080910C0B8695869581709927089580912A
:108990000D0B8695869581709927089580910E0B11
:1089A0008695869581709927089580910F0B8695FD
:1089B00086958170992708958EEF90E00895109222
:1089C000B60087E08093B0001092B2008EE48093EE
:1089D000B30082E08093700008950E94DF441092FB
:1089E000120B1092130B1092140B1092150B109285
:1089F0001A0B10921B0B0E94BC420E94E0050E94C1
:108A000055300895CF93C82F8091100B882311F013
:108A10001092100BA8950E948942C23011F00E945A
:108A20005C3EC23009F471C08091110B882309F4B7
:108A300046C08091110B81508093110B0E94221629
:108A40008091120B8F5F8093120B823040F0109256
:108A5000120B0E94CD430E94CB160E941A078091F0
:108A6000130B8F5F8093130B843040F01092130B25
:108A70000E9449170E947D560E9488538091140BD2
:108A80008F5F8093140B8A3030F01092140BC1303A
:108A900011F00E94C2118091150B8F5F8093150B0E
:108AA000843168F01092150B80911A0B8F5F8093C0
:108AB0001A0B0E94F5380E9471180E94771180915C
:108AC0001A0B8A3010F110921A0B8091160B9091AC
:108AD000170BA091180BB091190B0196A11DB11D98
:108AE0008093160B9093170BA093180BB093190B50
:108AF0000E945D3180911B0B8F5F80931B0B8C3329
:108B000020F010921B0B0E941C31CF910895809190
:108B1000160B9091170BA091180BB091190BBC017B
:108B2000CD0108951F920F920FB60F9211248F93CB
:108B30001092B20081E08093100B8091110B8F5F37
:108B40008093110B8F910F900FBE0F901F9018956F
:108B50000E9427520E94DA5360E076E980E090E0BC
:108B60000E94F553089504C00E946D520E94C052A5
:108B70000E9457528823C1F70895FC0190E061508C
:108B80006F3F21F0819198276150E0F7892F992755
:108B900008950F931F938C01FC0181818150682FF0
:108BA000C80101960E94BD45F80180838181992703
:108BB000BC01C8010E9488521F910F910895AF9285
:108BC000BF92CF92DF92EF92FF920F931F93CF93BA
:108BD000DF93CDB7DEB7C35ED0400FB6F894DEBFEB
:108BE0000FBECDBF6C01FC0181818150682FC60191
:108BF00001960E94BD45D6019C91981711F00C94E6
:108C0000B551F6018281882309F0F8C08381992744
:108C10008135910509F449C0823591053CF48033D2
:108C2000910589F08035910561F1E8C083359105A2
:108C300009F48EC0833591050CF478C08435910514
:108C400009F4B2C0DBC08E01035D1F4F80E5D8017F
:108C50001D928A95E9F785E18EA71FA680E888AB6B
:108C6000F601848189AB992796012B5F3F4FAC01B8
:108C7000B901CE01C2960E946365C8010E94C94530
:108C8000BDC08E01035D1F4F80E5D8011D928A95FE
:108C9000E9F785E08EA71FA680EA88AB0E94E32E45
:108CA00089ABC8010E94C945A9C0F601B4800F2E46
:108CB000FDE2EF2EFF24F02DEC0EFD1E80E5D70126
:108CC0001D928A95E9F789E18EA71FA681EA88ABF4
:108CD0008E0103581F4FB8018B2D0E940D2FB9AA8A
:108CE0008CE0FE01F296D8010D9001928A95E1F791
:108CF000F801848595859FAF8EAF8685FE01E05C87
:108D0000FF4F8083F8018785FE01EF5BFF4F808373
:108D10009927AC01BE0163577F4FCE018E5B9F4FF9
:108D20000E946365C7010E94C94568C00E949B2ECE
:108D3000FE01BD9680E5DF011D928A95E9F784E08A
:108D40008EA71FA682EA88ABCF010E94C94556C0F4
:108D5000F601458156818481FE01ED51FF4F8083EC
:108D6000813108F04BC080E5FE01BD9611928A95D5
:108D7000E9F787E18EA71FA683EA88AB5BAB4AAB16
:108D8000FE01ED51FF4F808189ABFE01F4969927DA
:108D9000DA01019724F00E9447660192FACFCE01D2
:108DA0008D960E94C9452AC0F6014581568184816D
:108DB000FE01ED51FF4F8083813100F5F6013796BA
:108DC0009927DA01019724F001900E945466FACFA6
:108DD000DE019D9680E5FD0111928A95E9F787E015
:108DE0008EA71FA684EA88AB5BAB4AABFE01ED51B0
:108DF000FF4F808189ABCD010E94C945F601828178
:108E0000813011F00C94BE5183819927AA27BB278A
:108E1000FC013197EB36F10510F00C94A751E65B9D
:108E2000FF4FEE0FFF1F0590F491E02D09940E9473
:108E3000F32CF601B4808B2D8150823210F00C940B
:108E4000BE5120E0AE01475F5F4F822F9927DA01C4
:108E5000A80FB91FF601E80FF91F82858C932F5FC9
:108E60002F3098F3F6018581898386818A838781F3
:108E70008B83838D948D9E838D83858D8F83808559
:108E8000888781858C83818D888F828D898F6B2DDA
:108E9000CE0101960E941A346B2DCE0101960E94DC
:108EA0006E201DA685E08EA711E01FA781E888AB84
:108EB00019AACE018D960E94C945812F0E940245B4
:108EC0000C94BE51F601B4808B2D8150823208F093
:108ED00047C06B2DCE0101960E945F348EE18EA7B4
:108EE00081E08FA782E888ABB9AA89818AAB8A81A1
:108EF0008BAB8B818CAB8C818EAB8D819E81FE0187
:108F0000E85BFF4F918380838F81FE01E65BFF4F1B
:108F1000808320E0BE016F5F7F4FAE01475F5F4FF0
:108F2000822F9927DC01A60FB71FFA01E80FF91F5E
:108F30008081FD0186AB2F5F2F3090F388858DAB4C
:108F4000888DFE01EA5BFF4F8083898DFE01E95B1E
:108F5000FF4F8083CE018D960E94C9450C94BE516F
:108F6000FFEFBF1611F00C94BE51FE01ED51FF4F03
:108F70001082FE01ED51FF4F8081982F823210F058
:108F80000C94BE510F2EF3EEEF2EFF24F02DEC0EBD
:108F9000FD1E6E010894C11CD11C8E01075F1F4F7E
:108FA000892F8F5F682FCE0101960E945F348EE17A
:108FB0008EA781E08FA782E888ABD7018C918F5F65
:108FC00089AB89818AAB8A818BAB8B818CAB8C819D
:108FD0008EAB8D819E81FE01E85BFF4F9183808384
:108FE0008F81FE01E65BFF4F808320E0822F99276F
:108FF000DC01AC0DBD1DF801E80FF91F8081FD01FA
:1090000086AB2F5F2F3090F388858DAB888DFE0166
:10901000EA5BFF4F8083898DFE01E95BFF4F808310
:10902000CE018D960E94C94581E00E940245D7017C
:109030008C918F5F8C93982F823208F4B1CF0C946F
:10904000BE510E94F32CF601B480AE0143585F4F2D
:1090500096012B5F3F4F8FE0DA01F90101900D92ED
:109060008A95E1F7F6018489FA018787BA018B2D89
:109070000E94B13481E08FA783E888ABB9AA85E06C
:109080008EA7CE018D960E94C9450C94BE51F60163
:10909000B4808B2D81508A3010F581E08FA784E851
:1090A00088ABB9AA8E0103581F4FB8018B2D0E94BF
:1090B000CE348FE0FE01F296D8010D9001928A9590
:1090C000E1F7F8018785FE01EF5BFF4F808385E1C3
:1090D0008EA7CE018D960E94C9450C94BE51FFEF1C
:1090E000BF1611F00C94BE51FE01ED51FF4F1082DE
:1090F000FE01ED51FF4F8081982F8B3010F00C94C2
:10910000BE51BB24B3948E0103581F4F0F2EFFE0B6
:10911000AF2EF02D0F2EF1E4EF2EFF24F02DEC0EEC
:10912000FD1E0F2EF3EECF2EDD24F02DCC0EDD1E16
:10913000BFA684E888AB892F8F5F89ABB8010E94F6
:10914000CE34FE01F296D8012A2D0D9001922A9577
:10915000E1F7F8018785D7018C9385E18EA7CE01D1
:109160008D960E94C9458B2D0E940245F601808193
:109170008F5F8083982F8B30D8F20C94BE510E9461
:10918000F32C0E94061BA8950E94141EA8950E940D
:109190007C1FA8950E94DD10A8950E944956A895AD
:1091A0000E943706A8950E94C2300E945B0F81E0A2
:1091B0008FA786E888AB84E08EA7CE018D960E94AB
:1091C000C9450C94BE5184E18EA781E08FA787E842
:1091D00088AB8DE0A7E7B1E0FE01F1960D9001921A
:1091E0008A95E1F70E9487459B01AC01AA27BB271E
:1091F0008EAFBB27A52F942F832F8FAFFE01E05C8E
:10920000FF4F2083CE018D960E94C9450C94BE511C
:109210000C9400000C94BE51C60104960E94A83222
:1092200081E08FA789E888AB84E08EA7CE018D9678
:109230000E94C9450C94BE5181E08FA78AE888AB93
:109240008CE08EA7CE01C1960E94B832CE018D96D9
:109250000E94C9450C94BE51CE0187960E943F2AB8
:1092600081E08FA781EA88AB8FA189AB88A58AAB03
:1092700089A58BAB8AA58CAB8BA58DAB8CA58EAB52
:109280008AE08EA7CE018D960E94C9450C94BE51EE
:10929000F601B480F1E2FB1500F1BE016E5D7F4F77
:1092A0008B2D0E94312B81E08FA782EA88ABB9AA6F
:1092B0008BA18BAB8CA18EAB8AA18AAB8DA19EA119
:1092C000892F99278CAB8DA18DAB8AE08EA7CE011B
:1092D0008D960E94C9450C94BE512FEFB21611F025
:1092E0000C94BE51FE01ED51FF4F1082FE01ED5175
:1092F000FF4F8081982F823210F00C94BE51FF24D2
:10930000F3948F01BE016E5D7F4F892F8F5F0E94A6
:10931000312BFFA682EA88ABD8018C918F5F89AB95
:109320008BA18BAB8CA18EAB8AA18AAB8DA19EA1A8
:10933000892F99278CAB8DA18DAB8AE08EA7CE01AA
:109340008D960E94C9458F2D0E940245F8018081AB
:109350008F5F8083982F8232A8F20C94BE51CE0189
:109360004A960E94FB2B8AE08EA781E08FA780EAB5
:1093700088AB88A189AB8E8D8AAB8A8D9B8D892F16
:1093800099278BAB8A8D8CAB8D8D8DAB8C8D8EABF5
:10939000CE018D960E94C9450C94BE51F6016481A0
:1093A00080E00E942A2384E08EA781E08FA783EAD1
:1093B00088ABCE018D960E94C945E0C7DE01A3535C
:1093C000BF4FF60184818C938581FD018183F60175
:1093D0008681FD018283F6018781FD018383F60189
:1093E0008085FD018483F6018185FD018583F60179
:1093F0008285FD018683F6018385FD018783CD018A
:109400000E94322384E08EA781E08FA784EA88AB94
:10941000CE018D960E94C945B1C7FE01E358FF4FAA
:10942000A0E0B0E080E190E021E08030920719F404
:109430000E944F6603C0182E0E944F66F601848179
:109440009581A681B781FE01EF57FF4F80839183FD
:10945000A283B383DE01A358BF4FF6018085FD01CF
:109460008087F6018185FD018187F6018285FD01F6
:109470008287A0E0B0E080E190E021E080309207B8
:1094800019F40E94606603C0182E0E94606684E092
:109490008EA781E08FA780EC88ABCE018D960E94CD
:1094A000C9456CC7FE01E358FF4FA0E0B0E080E182
:1094B00090E021E08030920719F40E944F6603C0CB
:1094C000182E0E944F668BE08EA781E08FA781EC5B
:1094D00088ABFE01EF57FF4F80819181A281B3815C
:1094E00089AB9AABABABBCABFE01E358FF4F8085B9
:1094F0008DAB81858EAB82858FABCE018D960E9420
:10950000C9453CC78AE38EA781E08FA780ED88AB71
:10951000FE01F196A8E8B0E082E190E021E0803021
:10952000920719F40E944F6603C0182E0E944F66DE
:10953000FE01ED5BFF4FAAE9B0E082E190E021E09F
:109540008030920719F40E944F6603C0182E0E94C3
:109550004F66FE01EB5AFF4FADEBB0E082E190E0C9
:1095600021E08030920719F40E944F6603C0182E44
:109570000E944F66CE018D960E94C945FFC684E1C8
:109580008EA781E08FA78EED88ABFE01F196ACEA45
:10959000B0E080E190E021E08030920719F40E9471
:1095A0004F6603C0182E0E944F66CE018D960E9412
:1095B000C945E4C60E94C23084E08EA781E08FA72F
:1095C00081ED88ABCE018D960E94C945D7C688E053
:1095D0008EA781E08FA78FED88AB0E9454318BABB3
:1095E0000E9458319AAB89ABFE01ED51FF4FACEBB5
:1095F000B0E081E090E021E08030920719F40E9411
:109600004F6603C0182E0E944F66FE01ED51FF4FBA
:1096100080818CABCE018D960E94C945AFC6FE01FC
:10962000E358FF4F80E5DF011D928A95E9F7ACEB27
:10963000B0E081E090E021E08030920719F40E94D0
:10964000606603C0182E0E946066FE01E358FF4F5B
:10965000A5E8B0E081E090E021E08030920719F4C5
:109660000E94606603C0182E0E946066FE01E358E7
:10967000FF4FA6E8B0E082E090E021E08030920762
:1096800019F40E94606603C0182E0E94606684E090
:109690008EA781E08FA780EE88ABCE018D960E94C9
:1096A000C9456CC6F601858196819093660E8093BC
:1096B000650E878190859093680E8093670E8185F3
:1096C000928590936A0E8093690E838580936B0ECA
:1096D000848580936C0E858580936D0E8785908937
:1096E0009093700E80936F0E868580936E0E8189A5
:1096F0008093710E82898093720E83898093730E9A
:10970000E5E6FEE0A0E7B0E08FE090E021E0803009
:10971000920719F40E94606603C0182E0E946066CA
:1097200085E08EA791E09FA785EA88AB99ABCE0133
:109730008D960E94C94522C684E18EA781E08FA73D
:1097400086EA88AB19AA8091E200863269F480919A
:10975000E300843049F48091E400833129F484E605
:1097600090E09BAB8AAB46C08091E2008E3169F4F9
:109770008091E300843049F48091E400833129F43E
:109780008DE790E09BAB8AAB35C08091E2008E30D4
:1097900069F48091E300843049F48091E4008331DE
:1097A00029F48AEF90E09BAB8AAB24C08091E20061
:1097B000863069F48091E300843049F48091E400BC
:1097C000833129F484EF91E09BAB8AAB13C0809185
:1097D000E200823069F48091E300843049F48091A2
:1097E000E400833129F488EE93E09BAB8AAB02C09E
:1097F0001BAA1AAA8091670E9091680E9DAB8CAB44
:109800008091690E90916A0E9FAB8EAB80916B0E2A
:1098100088AF80916C0E89AF80916D0E8AAF809178
:109820006F0E9091700E9DAF8CAF80916E0E8BAFCE
:109830008091710E8EAF8091720E8FAF8091730EFA
:10984000FE01E05CFF4F8083CE018D960E94C945EA
:1098500095C5DE01AB52BF4FF60184818C938581A3
:10986000FD018183D60116968CE0FE01E952FF4F7F
:109870000D9001928A95E1F7FE01ED51FF4F1082A4
:10988000FE01ED51FF4F8081982F8C30A0F49E0196
:109890002B523F4FDF01F901E90FF11D828188232F
:1098A00021F08F3F11F0815082838C918F5F8C93D8
:1098B000982F8C3080F3CE018B529F4F0E945A32EA
:1098C00084E08EA781E08FA787EA88ABCE018D96D2
:1098D0000E94C94553C58E010B521F4FC8010E94FB
:1098E000783282E18EA781E08FA788EA88ABD80121
:1098F0008C9189ABF80181818AABFE01ED51FF4F5C
:109900001082FE01ED51FF4F8081982F8C3080F442
:109910009801DF01F901E90FF11D82818F3F11F0FC
:109920008F5F82838C918F5F8C93982F8C3090F314
:109930008CE0DE01A952BF4FFE01F3960D9001921B
:109940008A95E1F7CE018D960E94C94517C5F601AB
:109950008481FE01E358FF4F8083D60115968EE087
:10996000FE01E258FF4F0D9001928A95E1F7FE014A
:10997000ED51FF4F1082FE01ED51FF4F8081982F76
:109980008E30A0F49E0123583F4FDF01F901E90F0B
:10999000F11D8181882321F08F3F11F08150818357
:1099A0008C918F5F8C93982F8E3080F3DE01A358BB
:1099B000BF4FF6018389FD018787F6018489FD0188
:1099C000808BD60155968EE0FE01E257FF4F0D9039
:1099D00001928A95E1F7FE01ED51FF4F1082FE01E1
:1099E000ED51FF4F8081982F8E30A0F49E012358B7
:1099F0003F4FDF01F901E90FF11D8189882321F033
:109A00008F3F11F08150818B8C918F5F8C93982FB9
:109A10008E3080F3CE0183589F4F0E94883284E0BD
:109A20008EA781E08FA789EA88ABCE018D960E9430
:109A3000C945A4C48E0103581F4FC8010E94983223
:109A400083E28EA781E08FA78AEA88ABD8018C9148
:109A500089ABFE01ED51FF4F1082FE01ED51FF4F2A
:109A60008081982F8E3080F49801DF01F901E90F91
:109A7000F11D81818F3F11F08F5F81838C918F5F0A
:109A80008C93982F8E3090F38EE0DE01A258BF4F5A
:109A9000FE01F2960D9001928A95E1F7DE01A3583E
:109AA000BF4FFD018785FE01E05CFF4F8083FD0114
:109AB0008089FE01EF5BFF4F8083FE01ED51FF4F78
:109AC0001082FE01ED51FF4F8081982F8E3080F47F
:109AD0009D01DF01F901E90FF11D81898F3F11F02F
:109AE0008F5F818B8C918F5F8C93982F8E3090F34A
:109AF0008EE0DE01A257BF4FFE01EE5BFF4F0D90DF
:109B000001928A95E1F7CE018D960E94C94536C42F
:109B1000F601B48085819927982F88272681820FA6
:109B2000911DBC018B2D0E94762C85E08EA781E0D3
:109B30008FA782EC88ABB9AACE018D960E94C94549
:109B40001DC4F601B4808CE08EA781E08FA783EC62
:109B500088ABB9AA8B2D0E94342C8AAB8B2D0E9426
:109B6000502C892F99278BAB8B2D0E94502C8CABBE
:109B70008B2D0E949F2C892F99278DAB8B2D0E94B6
:109B80009F2C8EAB8B2D0E94B72C892F99278FABE2
:109B90008B2D0E94B72C88AFCE018D960E94C945AF
:109BA000EDC320E0F601848181FD21E0F60184818E
:109BB00082FD2260F6018181863029F46581822F41
:109BC0000E94CF2CDBC360E0822F0E94CF2CD6C333
:109BD0000E94D42C84E08EA781E08FA785EC88AB0F
:109BE000CE018D960E94C945C9C3F601B4809E017D
:109BF00023583F4F9581492F4170D9018C91887F1F
:109C00009670842B892B8C9386819781F90192839E
:109C10008183F60180859185F90194838383F60120
:109C20008685F9018187F6018785F9018287F6012A
:109C300082859385F90196838583F60184859585D0
:109C4000F90190878783F6018089F9018387F601FE
:109C50008189F9018487F6018289F9018587F601F6
:109C60008389F9018687D60154968FE0FE01E45777
:109C7000FF4F0D9001928A95E1F7F60183A1F9015A
:109C8000868FF60184A1F901878FF60185A1F9017C
:109C900080A3F60186A1F90181A315E0D60197966C
:109CA000FE01E156FF4F812F0D9001928A95E1F759
:109CB000F60184A595A5A6A5B7A5F90187A390A748
:109CC000A1A7B2A7F60180A9F90183A7B9018B2D3D
:109CD0000E943A3381E08FA782ED88AB1EA7B9AA14
:109CE000CE018D960E94C94549C3F601B4808E010C
:109CF00003581F4FB8018B2D0E94723381E08FA74C
:109D000083ED88AB81E38EA7B9AAD8019C91292F56
:109D100021708AA9887F9670822B892B8AABF801E3
:109D2000818192819CAB8BAB838194819EAB8DAB07
:109D300081858BAF82858CAF8581968198AF8FAB03
:109D4000878190859AAF89AF83858DAF84858EAFEB
:109D500085858FAF8685FE01E05CFF4F80838FE0B5
:109D6000DE01A457BF4FFE01EF5BFF4F0D90019244
:109D70008A95E1F7F801868DFE01E05BFF4F808355
:109D8000F801878DFE01EF5AFF4F8083F80180A113
:109D9000FE01EE5AFF4F8083F80181A1FE01ED5ACA
:109DA000FF4F808385E0DE01A156BF4FFE01EC5AD4
:109DB000FF4F0D9001928A95E1F7F80187A190A5D8
:109DC000A1A5B2A5FE01E75AFF4F80839183A2832C
:109DD000B383F80183A5FE01E35AFF4F8083CE01D0
:109DE0008D960E94C945CAC2F601B480AE0143589F
:109DF0005F4F828DDA018C93838DFA018183F601A6
:109E0000848DFA018283F6018681FA018383F6014B
:109E10008781FA018483F6018085FA018583F60142
:109E20008185FA018683F6018285FA018783F6012E
:109E3000858DFA01878BC6010B962FE0FE01EB574B
:109E4000FF4FDC010D9001922A95E1F7BA018B2DAD
:109E50000E94AA3381E08FA784ED88AB85E08EA7AE
:109E6000B9AACE018D960E94C94588C2F601B48078
:109E70008E0103581F4FB8018B2D0E94E23381E001
:109E80008FA785ED88AB8FE18EA7B9AAD8018C91F9
:109E9000FE01E95BFF4F8083F8018181FE01E85BF1
:109EA000FF4F8083F8018281FE01E75BFF4F8083D3
:109EB000F80183818BAB84818CAB85818DAB8681EE
:109EC0008EAB87818FAB8789FE01E65BFF4F808376
:109ED0008FE0DE01AB57BF4FFE01F8960D90019267
:109EE0008A95E1F7CE018D960E94C94547C2F601D9
:109EF0003496AAEEB8E082E090E021E0803092074C
:109F000019F40E94606603C0182E0E94606681E00A
:109F10008FA783EE88AB84E08EA7CE018D960E943A
:109F2000C9452CC281E08FA784EE88AB84E18EA75F
:109F3000FE01F196AAEEB8E082E090E021E08030E8
:109F4000920719F40E944F6603C0182E0E944F66B4
:109F5000CE018D960E94C94511C2F601B480C6019A
:109F60000596BC018B2D0E94C83281E08FA788ED39
:109F700088AB85E08EA7B9AACE018D960E94C9450F
:109F8000FDC1F601B48081E08FA789ED88AB8EE139
:109F90008EA7B9AABE016E5C7F4F8B2D0E94013344
:109FA000CE018D960E94C945E9C1F6018481809356
:109FB000790E858180937A0E868180937B0E8781CE
:109FC00080937C0E808580937D0E818580937E0EAC
:109FD000828580937F0E83858093800EE9E7FEE083
:109FE000AEE6BFE088E090E021E08030920719F40F
:109FF0000E94606603C0182E0E94606681E08FA7F1
:10A0000085EE88AB84E08EA7CE018D960E94C9456F
:10A01000B5C181E08FA786EE88AB8CE08EA78091DA
:10A02000790E89AB80917A0E8AAB80917B0E8BABD7
:10A0300080917C0E8CAB80917D0E8DAB80917E0EDD
:10A040008EAB80917F0E8FAB8091800E88AFCE015A
:10A050008D960E94C94592C1F6013496AEE8BFE0E4
:10A060008CE490E021E08030920719F40E94606651
:10A0700003C0182E0E946066F60184818093810ED1
:10A080008581982F97708091820E887F892B80938D
:10A09000820E87898093830E808D982F9770809190
:10A0A000840E887F892B8093840E82A58093850EF1
:10A0B00083A5982F97708091860E887F892B809337
:10A0C000860E85AD8093870E86AD982F9770809110
:10A0D000880E887F892B8093880E81E08FA787EE7A
:10A0E00088AB84E08EA7CE018D960E94C94546C1FB
:10A0F00081E08FA788EE88AB80E58EA7FE01F19600
:10A10000AEE8BFE08CE490E021E08030920719F4E3
:10A110000E944F6603C0182E0E944F66CE018D9696
:10A120000E94C9452BC1F6013496AAEDBFE089E033
:10A1300090E021E08030920719F40E94606603C02D
:10A14000182E0E946066F6013D96A3EEBFE089E0FE
:10A1500090E021E08030920719F40E94606603C00D
:10A16000182E0E94606681E08FA789EE88AB84E09C
:10A170008EA7CE018D960E94C94500C181E08FA7B0
:10A180008AEE88AB87E18EA7FE01F196AAEDBFE0CB
:10A1900089E090E021E08030920719F40E944F6638
:10A1A00003C0182E0E944F66FE01FA96A3EEBFE090
:10A1B00089E090E021E08030920719F40E944F6618
:10A1C00003C0182E0E944F66CE018D960E94C9458D
:10A1D000D5C0C60105960E943C3581E08FA786ED6B
:10A1E00088AB85E08EA7CE018D960E94C945C6C07A
:10A1F00081E08FA787ED88AB8DE18EA7CE01C29657
:10A200000E944C35CE018D960E94C945B7C0F6011B
:10A21000B480C60104960E945C3581E08FA78AED68
:10A2200088AB85E08EA7B9AACE018D960E94C9455C
:10A23000A5C0F601B48081E08FA78BED88AB8AE4DE
:10A240008EA7BE016F5C7F4F8B2D0E948935CE019A
:10A250008D960E94C94592C0F601B4808B2D0E9454
:10A26000461181E08FA78CED88ABB9AA85E08EA757
:10A27000CE018D960E94C94581C0F6014481558169
:10A2800081E08FA78DED88AB86E18EA75AAB49ABF5
:10A29000FE01ED51FF4F1082FE01ED51FF4F808115
:10A2A000982F8031C8F48E010F5F1F4FBF01892F97
:10A2B00099279C01200F311F840F951FAA27BB27C8
:10A2C000ABBFFC018791F90182ABDB018C918F5F01
:10A2D0008C93982F803158F3CE018D960E94C945FA
:10A2E0004DC0F6013496AEE5BFE080E190E021E09C
:10A2F0008030920719F40E94606603C0182E0E94F5
:10A30000606681E08FA781EE88AB84E08EA7CE01E6
:10A310008D960E94C94532C081E08FA782EE88AB3E
:10A3200084E18EA7FE01F196AEE5BFE080E190E00A
:10A3300021E08030920719F40E944F6603C0182E66
:10A340000E944F66CE018D960E94C94517C081E0DC
:10A350008FA780E888AB85E08EA7F601838189AB63
:10A36000CE018D960E94C94509C085E08EA71FA623
:10A3700081E088ABCE018D960E94C945CD51DF4F5B
:10A380000FB6F894DEBF0FBECDBFDF91CF911F9106
:10A390000F91FF90EF90DF90CF90BF90AF90089516
:10A3A000CF93DF93CDB7DEB72A970FB6F894DEBF11
:10A3B0000FBECDBF81E08B8388E88C8384E08A83E5
:10A3C000CE0101960E94C9452A960FB6F894DEBFC9
:10A3D0000FBECDBFDF91CF9108950F931F93CF9301
:10A3E000DF93CDB7DEB7C055D0400FB6F894DEBFCF
:10A3F0000FBECDBF8A0121E02B832DE52C839E83E8
:10A400008D836F8320E0261780F4AE01485F5F4F95
:10A41000822F9927DA01A80FB91FF801E80FF91F59
:10A4200080818C932F5F261798F38FE08A83CE016B
:10A4300001960E94C945C05BDF4F0FB6F894DEBF9E
:10A440000FBECDBFDF91CF911F910F91089548ECC2
:10A4500050E060E070E08DE19BE00E94706510923A
:10A46000E50B1092E60B10921C0B0895382F2091EB
:10A47000E60B8DE19BE0FC01E20FF11D3083809142
:10A48000E60B8F5F8093E60B80911C0B8F5F8093B0
:10A490001C0B80911C0B883C18F00E9427520895D9
:10A4A0008091E60B883C10F01092E60B0895909195
:10A4B000E60B8091E50B981738F08091E60B9091B0
:10A4C000E50B891B992708959091E60B8091E50B88
:10A4D000981B892F8853992708952091E50B8DE1CA
:10A4E0009BE0FC01E20FF11DE0818091E50B8F5FA5
:10A4F0008093E50B80911C0B815080931C0B809105
:10A50000E50B883C10F01092E50B8E2F99270895EB
:10A510000F931F93CF93DF93EC018B0180EC0E948C
:10A520001B54015010408FEF0F3F180709F188812D
:10A530009927803C910521F08B3D910541F00EC09B
:10A540008BED0E941B548CED0E941B540AC08BEDB6
:10A550000E941B548DED0E941B5403C088810E94F1
:10A560001B542196015010408FEF0F3F1807F9F64A
:10A5700080EC0E941B54DF91CF911F910F910895A1
:10A580000F931F93382F8091E70B9927009719F0AD
:10A590000197C1F059C0303C09F056C01092E80B49
:10A5A0002091E80B8AEE9BE0FC01E20FF11D308365
:10A5B0002F5F2093E80B81E08093E70B84E6809384
:10A5C000E90B42C0303C99F58091E80B8230F0F005
:10A5D0008091E80B0AEE1BE0F801E80FF11D3083D3
:10A5E0008F5F8093E80B82E08093E70B1092E90B7A
:10A5F000A8016091E80BC8010E942F53C8010E9476
:10A60000DF451092E70B1092E80B1EC01092E80B8A
:10A610002091E80B8AEE9BE0FC01E20FF11D3083F4
:10A620002F5F2093E80B84E68093E90B0DC0209107
:10A63000E80B8AEE9BE0FC01E20FF11D3083809174
:10A64000E80B8F5F8093E80B8091E80B893620F050
:10A650001092E70B1092E80B1F910F910895FC01E7
:10A66000DA0161506F3FF1F02081822F9927803C01
:10A67000910521F08B3D910519F010C0319610C065
:10A6800031962081822F99278C3D910521F08D3DB7
:10A69000910519F003C020EC01C02BED2D933196EC
:10A6A000615010F708958091E90B882389F080911B
:10A6B000E90B81508093E90B9091E90B992341F4C8
:10A6C0008091E70B813021F49093E80B9093E70B96
:10A6D000089585B1807F85B984B1876084B981E5AB
:10A6E0008CBD81E08DBD08958EBD0DB407FEFDCFFC
:10A6F0008EB5992708950E94D8539C9AA4988FE00C
:10A700008093540CA4986A9862980895A498089528
:10A71000CF93DF93CDB7DEB728970FB6F894DEBF9F
:10A720000FBECDBFA49B18C0629914C08091530C7A
:10A73000853050F0A4980E942B2182E28093110171
:10A740001092890E1092740E8091530C8F5F80933B
:10A75000530C02C01092530CCE0101960E94FB2BA9
:10A7600029813A8181E590E0289FA001299F500D21
:10A77000389F500D1124CA01880F892F881F990B0B
:10A7800091950E94D9538D81882319F48F81882354
:10A7900011F0A49A01C0A49828960FB6F894DEBFD1
:10A7A0000FBECDBFDF91CF9108958093540C0895D3
:10A7B000089508951092560C1092550C86E08093DF
:10A7C000C20088E98093C10060E875E280E090E013
:10A7D0000E94F55381E08093F20E1092F30E0895DB
:10A7E0009093560C8093550C08959B01AC01DC01AD
:10A7F000CB01689412F8880F991FAA1FBB1F1694EB
:10A80000D1F780509C4DAB40BF4F689413F8220F96
:10A81000331F441F551F1694D1F7BC01CD010E9470
:10A82000D365DA01C9010197292F33272093C50089
:10A830008093C4000895982F8091C00085FFFCCFBD
:10A840009093C60008950F931F93CF93DF938C01CD
:10A85000EB0121978FEFCF3FD80751F0F80181919D
:10A860008F010E941B542197FFEFCF3FDF07B1F705
:10A8700081E090E0DF91CF911F910F9108951F9299
:10A880000F920FB60F9211242F933F934F935F9324
:10A890006F937F938F939F93AF93BF93EF93FF93A8
:10A8A0008091C6000E943652FF91EF91BF91AF9107
:10A8B0009F918F917F916F915F914F913F912F91D8
:10A8C0000F900FBE0F901F901895DC01FB014150B7
:10A8D00050408FEF4F3F580741F081918D93415089
:10A8E00050408FEF4F3F5807C1F70895DC01FB013F
:10A8F000415050408FEF4F3F580769F091918D9133
:10A90000891719F081E090E00895415050408FEF91
:10A910004F3F580799F780E090E00895CF93DF9379
:10A92000DC01FB0160E0462F91E0562F80818032F0
:10A9300031F4692F9F5F319680818032D1F380811D
:10A94000882379F08081803219F4442309F4492F57
:10A950008081803209F040E09F5F319680818823BA
:10A9600089F7442331F48081882311F4492F01C0F1
:10A97000462F262F3327E901C91BD109EC0FFD1FF4
:10A980003196842F9927821B930B0197181619066D
:10A9900024F4942F961B915001C090E091509F3F5A
:10A9A00029F081918D935F5F9150D8F71C925F5F82
:10A9B000852F9927DF91CF910895FC0190E0819137
:10A9C000882331F09F5F8191882311F09F3FD1F759
:10A9D000892F99270895DC01FB018081882329F0C4
:10A9E00081918D9380818823D9F71C9208950F93CC
:10A9F0001F93CF93DF93082F162FFA0141E0C0E198
:10AA0000D7E2C901BE010E94C0656115710581F0E0
:10AA10006C9FC0016D9F900D7C9F900D1124281B91
:10AA2000390B862F805D8193440F01E015E00AC049
:10AA3000153040F0002319F080E3819302C080E2DA
:10AA400081934F5FC8EED3E0C901BE010E94C0658B
:10AA50006115710581F06C9FC0016D9F900D7C9F09
:10AA6000900D1124281B390B862F805D81934F5F39
:10AA700001E014E00AC0143040F0002319F080E334
:10AA8000819302C080E281934F5FC4E6D0E0C901A8
:10AA9000BE010E94C0656115710581F04F5F6C9F1A
:10AAA000C0016D9F900D7C9F900D1124281B390BC8
:10AAB000862F805D819301E013E00AC0133040F0DF
:10AAC0004F5F002319F080E3819302C080E28193FD
:10AAD000C9016AE070E00E94C0656115710591F0DE
:10AAE0004F5FCB01880F991F880F991F880F991FFF
:10AAF000860F971F860F971F281B390B862F805DA7
:10AB000081930AC0123040F04F5F002319F080E3B8
:10AB1000819302C080E28193822F805D81931082B5
:10AB2000842F9927DF91CF911F910F910895FC01F8
:10AB3000262F862F82958F708A3038F06AE00E9427
:10AB4000A065892F8F5B819309C0862F82958F70B6
:10AB50006AE00E94A065892F805D8193822F8F70AB
:10AB60008A3038F06AE00E94A065892F8F5B80836D
:10AB70000895822F8F706AE00E94A065892F805D02
:10AB800080830895EF92FF920F931F937C018B01B6
:10AB9000872F9927682FC7010E949755C801907089
:10ABA000682FC7010E9497551F910F91FF90EF905A
:10ABB0000895CF92DF92EF92FF920F931F936C0153
:10ABC0007A018B01CB01AA27BB27BC01C6010E94D9
:10ABD000C255D801C701A070B070BC01C6010E9467
:10ABE000C2551F910F91FF90EF90DF90CF90089585
:10ABF0001F93CF93DF93CDB7DEB768970FB6F89466
:10AC0000DEBF0FBECDBF10E0BE016F5F7F4F812F53
:10AC10000E94E233412F5527CA01880F991F880FE0
:10AC2000991F880F991F9C01241B350BF901E95AC4
:10AC3000F34F898184838A8185838B8186838C818C
:10AC400080838D8181838E818283F901E65AF34F5F
:10AC50008F81382F337088858370282F220F220F21
:10AC6000888D982F9295907F822F832B892B8083BC
:10AC7000FA01E35AF24F10821F5F143128F26896EE
:10AC80000FB6F894DEBF0FBECDBFDF91CF911F91FD
:10AC900008951F93CF93DF93CDB7DEB768970FB6B4
:10ACA000F894DEBF0FBECDBF10E0A89519821A82BE
:10ACB0001B821C821D821E821F821886188E8FE0C6
:10ACC000189FC00111248858994FBC01CE010996E4
:10ACD0000E944F65BE016F5F7F4F812F0E94AA3394
:10ACE0001F5F143110F368960FB6F894DEBF0FBEE5
:10ACF000CDBFDF91CF911F910895CF93C0E086E043
:10AD0000C89FC0011124FC01EB51F34FF093E40CF8
:10AD1000E093E30C80819181009719F00197918372
:10AD20008083E091E30CF091E40C828193810097A1
:10AD300019F0019793838283E091E30CF091E40C86
:10AD400084819581009719F00197958384832C2F36
:10AD50003327C901880F991F880F991F880F991FE2
:10AD6000821B930BFC01E95AF34F8081882319F46D
:10AD70008181882321F08C2F8F5D0E94CE57CF5F79
:10AD8000C43108F4BCCFCF9108959927873091053D
:10AD900009F466C088309105ACF48430910509F45B
:10ADA0003EC08530910534F48230910511F103974E
:10ADB00059F198C08530910509F43CC0069709F413
:10ADC00044C090C08A30910509F46BC08B30910566
:10ADD00044F48830910509F44EC0099709F456C02F
:10ADE00081C08B30910509F467C00C9709F46FC0DE
:10ADF00079C080EC0E945C44882319F081E090E0E7
:10AE0000089580E090E0089581EC0E945C448823DE
:10AE100019F081E090E0089580E090E0089582ECE0
:10AE20000E945C44882319F081E090E0089580E05E
:10AE300090E0089581ED0E945C44882319F081E040
:10AE400090E0089580E090E0089584EC0E945C44D6
:10AE5000882319F081E090E0089580E090E0089563
:10AE600085EC0E945C44882319F081E090E008950D
:10AE700080E090E0089586EC0E945C44882319F0FD
:10AE800081E090E0089580E090E0089587EC0E94D2
:10AE90005C44882319F081E090E0089580E090E020
:10AEA000089583EC0E945C44882319F081E090E0CF
:10AEB000089580E090E0089582ED0E945C4488232C
:10AEC00019F081E090E0089580E090E0089583ED2E
:10AED0000E945C44882319F081E090E0089580E0AE
:10AEE00090E0089580E090E008950F93CF93DF9372
:10AEF000CDB7DEB721970FB6F894DEBF0FBECDBF3A
:10AF000089838150843170F000E021E0AE014F5F11
:10AF10005F4F69E071E08EE891E00E943D2F80E094
:10AF200090E007C089819927FC01E45AF24F8081A3
:10AF3000992721960FB6F894DEBF0FBECDBFDF91E3
:10AF4000CF910F9108950F93CF93DF93CDB7DEB7D5
:10AF500021970FB6F894DEBF0FBECDBF8983843131
:10AF600060F000E021E0AE014F5F5F4F64E171E00F
:10AF70008EE891E00E943D2F07C089812DE53DE0DC
:10AF8000F901E80FF11D608321960FB6F894DEBF3A
:10AF90000FBECDBFDF91CF910F910895FF920F9318
:10AFA0001F93CF93DF93CDB7DEB721970FB6F894F9
:10AFB000DEBF0FBECDBF1982813209F46DC082326F
:10AFC00019F481E0898368C0833219F482E08983AF
:10AFD00063C0843219F483E089835EC0853219F43A
:10AFE00084E0898359C0863219F485E0898354C08E
:10AFF000873219F486E089834FC0883219F487E0DC
:10B0000089834AC0893219F488E0898345C08A322D
:10B0100019F489E0898340C08B3219F48AE089836E
:10B020003BC08C3219F48BE0898336C08D3219F421
:10B030008CE0898331C08E3219F48DE089832CC075
:10B040008F3219F48EE0898327C0803319F48FE0A2
:10B05000898322C0813319F480E189831DC0823342
:10B0600019F481E1898318C0833319F482E189835B
:10B0700013C0843319F483E189830EC000E021E01A
:10B08000AE014F5F5F4F69E471E08EE891E00E948E
:10B090003D2F80E090E087C700E0102FF02E29813F
:10B0A00086E0289FC00111248B51934F9093E40CAC
:10B0B0008093E30C3327C901880F991F880F991FCC
:10B0C000880F991F821B930BFC01E95AF34F808173
:10B0D000882309F49BC18981282F3327C901880F50
:10B0E000991F880F991F880F991F821B930BFC01D2
:10B0F000E95AF34F80818F3F11F411E087C18981B4
:10B10000282F3327C901880F991F880F991F880F8F
:10B11000991F821B930BFC01E95AF34FE0818E2F9C
:10B1200082508B3008F04DC08E2F0E94C556482F9C
:10B130008981282F3327C901880F991F880F991FEC
:10B14000880F991F821B930BFC01E65AF34F8081F5
:10B1500082958F7080FF02C081E04827442361F010
:10B16000E091E30CF091E40C80819181892B11F442
:10B1700011E04CC110E04AC1A091E30CB091E40C85
:10B180008981282F3327C901880F991F880F991F9C
:10B19000880F991F821B930BFC01E95AF34F94818E
:10B1A00085E0989FC00111248D939C93E091E30C5E
:10B1B000F091E40C8081918101969183808310E06D
:10B1C00025C18981282F3327C901880F991F880F2E
:10B1D000991F880F991F821B930BFC01E95AF34FAB
:10B1E000E0818E2F8D50803208F04DC08F5F0E941D
:10B1F0004911482F8981282F3327C901880F991FAA
:10B20000880F991F880F991F821B930BFC01E65A28
:10B21000F34F808182958F7080FF02C081E04827C4
:10B22000442361F0E091E30CF091E40C8081918182
:10B23000892B11F411E0EAC010E0E8C0A091E30C02
:10B24000B091E40C8981282F3327C901880F991FF9
:10B25000880F991F880F991F821B930BFC01E95AD5
:10B26000F34F948185E0989FC00111248D939C93A6
:10B27000E091E30CF091E40C80819181019691833F
:10B28000808310E0C3C08981282F3327C901880F2C
:10B29000991F880F991F880F991F821B930BFC0120
:10B2A000E95AF34FE0818E2F8D52823208F04DC063
:10B2B0008F5F0E94B52B482F8981282F3327C90122
:10B2C000880F991F880F991F880F991F821B930B56
:10B2D000FC01E65AF34F808182958F7080FF02C097
:10B2E00081E04827442361F0E091E30CF091E40C05
:10B2F00080819181892B11F411E088C010E086C013
:10B30000A091E30CB091E40C8981282F3327C90167
:10B31000880F991F880F991F880F991F821B930B05
:10B32000FC01E95AF34F948185E0989FC0011124F4
:10B330008D939C93E091E30CF091E40C80819181DA
:10B3400001969183808310E061C08981282F332783
:10B35000C901880F991F880F991F880F991F821B99
:10B36000930BFC01E95AF34FE0818E2F8F548F30FD
:10B3700008F04CC08F5F0E947557482F8981282F95
:10B380003327C901880F991F880F991F880F991FAC
:10B39000821B930BFC01E65AF34F808182958F70DC
:10B3A00080FF02C081E04827442361F0E091E30C74
:10B3B000F091E40C80819181892B11F411E026C079
:10B3C00010E024C0A091E30CB091E40C8981282FF7
:10B3D0003327C901880F991F880F991F880F991F5C
:10B3E000821B930BFC01E95AF34F948185E0989FEF
:10B3F000C00111248D939C93E091E30CF091E40C37
:10B400008081918101969183808310E08981282F2A
:10B410003327C901880F991F880F991F880F991F1B
:10B42000821B930BFC01E95AF34F8181882311F4AD
:10B43000082F9FC18981282F3327C901880F991FA1
:10B44000880F991F880F991F821B930BFC01E95AE3
:10B45000F34F81818F3F11F401E08BC18981282F47
:10B460003327C901880F991F880F991F880F991FCB
:10B47000821B930BFC01E95AF34F9181892F825073
:10B480008B3008F04EC0892F0E94C556482F898105
:10B49000282F3327C901880F991F880F991F880FFC
:10B4A000991F821B930BFC01E65AF34F8081829512
:10B4B0008F7081FF02C081E04827442361F0E09152
:10B4C000E30CF091E40C82819381892B11F401E06B
:10B4D00050C100E04EC1A091E30CB091E40C898111
:10B4E000282F3327C901880F991F880F991F880FAC
:10B4F000991F821B930BFC01E95AF34F958185E05C
:10B50000989FC0011124FD0193838283E091E30C95
:10B51000F091E40C8281938101969383828300E011
:10B5200028C18981282F3327C901880F991F880FC7
:10B53000991F880F991F821B930BFC01E95AF34F47
:10B540009181892F8D50803208F04EC08F5F0E940C
:10B550004911482F8981282F3327C901880F991F46
:10B56000880F991F880F991F821B930BFC01E65AC5
:10B57000F34F808182958F7081FF02C081E0482760
:10B58000442361F0E091E30CF091E40C828193811B
:10B59000892B11F401E0EDC000E0EBC0A091E30CB9
:10B5A000B091E40C8981282F3327C901880F991F96
:10B5B000880F991F880F991F821B930BFC01E95A72
:10B5C000F34F958185E0989FC0011124FD0193837D
:10B5D0008283E091E30CF091E40C828193810196E7
:10B5E0009383828300E0C5C08981282F3327C90156
:10B5F000880F991F880F991F880F991F821B930B23
:10B60000FC01E95AF34F9181892F8D52823208F063
:10B610004EC08F5F0E94B52B482F8981282F33277A
:10B62000C901880F991F880F991F880F991F821BC6
:10B63000930BFC01E65AF34F808182958F7081FF56
:10B6400002C081E04827442361F0E091E30CF091CF
:10B65000E40C82819381892B11F401E08AC000E01F
:10B6600088C0A091E30CB091E40C8981282F332786
:10B67000C901880F991F880F991F880F991F821B76
:10B68000930BFC01E95AF34F958185E0989FC00127
:10B690001124FD0193838283E091E30CF091E40C8B
:10B6A0008281938101969383828300E062C08981C5
:10B6B000282F3327C901880F991F880F991F880FDA
:10B6C000991F821B930BFC01E95AF34F9181892F3B
:10B6D0008F548F3008F04DC08F5F0E947557482FF0
:10B6E0008981282F3327C901880F991F880F991F37
:10B6F000880F991F821B930BFC01E65AF34F808140
:10B7000082958F7081FF02C081E04827442361F059
:10B71000E091E30CF091E40C82819381892B11F488
:10B7200001E027C000E025C0A091E30CB091E40C3B
:10B730008981282F3327C901880F991F880F991FE6
:10B74000880F991F821B930BFC01E95AF34F9581D7
:10B7500085E0989FC0011124FD0193838283E091CD
:10B76000E30CF091E40C82819381019693838283B0
:10B7700000E08981282F3327C901880F991F880F7E
:10B78000991F880F991F821B930BFC01E95AF34FF5
:10B790008281882311F4F82EA4C18981282F3327B0
:10B7A000C901880F991F880F991F880F991F821B45
:10B7B000930BFC01E95AF34F82818F3F19F4FF2468
:10B7C000F3948FC18981282F3327C901880F991FCE
:10B7D000880F991F880F991F821B930BFC01E95A50
:10B7E000F34F9281892F82508B3008F04FC0892F00
:10B7F0000E94C556482F8981282F3327C901880FF9
:10B80000991F880F991F880F991F821B930BFC01AA
:10B81000E65AF34F808182958F7082FF02C081E0EB
:10B820004827442369F0E091E30CF091E40C848113
:10B830009581892B19F4FF24F39453C1FF2451C13E
:10B84000A091E30CB091E40C8981282F3327C90122
:10B85000880F991F880F991F880F991F821B930BC0
:10B86000FC01E95AF34F968185E0989FC0011124AD
:10B87000FD0195838483E091E30CF091E40C8481D5
:10B880009581019695838483FF242BC18981282F7C
:10B890003327C901880F991F880F991F880F991F97
:10B8A000821B930BFC01E95AF34F9281892F8D5033
:10B8B000803208F04FC08F5F0E944911482F898164
:10B8C000282F3327C901880F991F880F991F880FC8
:10B8D000991F821B930BFC01E65AF34F80818295DE
:10B8E0008F7082FF02C081E04827442369F0E09115
:10B8F000E30CF091E40C84819581892B19F4FF24E9
:10B90000F394EFC0FF24EDC0A091E30CB091E40CE0
:10B910008981282F3327C901880F991F880F991F04
:10B92000880F991F821B930BFC01E95AF34F9681F4
:10B9300085E0989FC0011124FD0195838483E091E7
:10B94000E30CF091E40C84819581019695838483C6
:10B95000FF24C7C08981282F3327C901880F991F69
:10B96000880F991F880F991F821B930BFC01E95ABE
:10B97000F34F9281892F8D52823208F04FC08F5F32
:10B980000E94B52B482F8981282F3327C901880FA2
:10B99000991F880F991F880F991F821B930BFC0119
:10B9A000E65AF34F808182958F7082FF02C081E05A
:10B9B0004827442369F0E091E30CF091E40C848182
:10B9C0009581892B19F4FF24F3948BC0FF2489C03F
:10B9D000A091E30CB091E40C8981282F3327C90191
:10B9E000880F991F880F991F880F991F821B930B2F
:10B9F000FC01E95AF34F968185E0989FC00111241C
:10BA0000FD0195838483E091E30CF091E40C848143
:10BA10009581019695838483FF2463C08981282FB3
:10BA20003327C901880F991F880F991F880F991F05
:10BA3000821B930BFC01E95AF34F9281892F8F549B
:10BA40008F3008F04EC08F5F0E947557482F898154
:10BA5000282F3327C901880F991F880F991F880F36
:10BA6000991F821B930BFC01E65AF34F808182954C
:10BA70008F7082FF02C081E04827442369F0E09183
:10BA8000E30CF091E40C84819581892B19F4FF2457
:10BA9000F39427C0FF2425C0A091E30CB091E40CDF
:10BAA0008981282F3327C901880F991F880F991F73
:10BAB000880F991F821B930BFC01E95AF34F968163
:10BAC00085E0989FC0011124FD0195838483E09156
:10BAD000E30CF091E40C8481958101969583848335
:10BAE000FF242981822F9927AC01440F551F440F51
:10BAF000551F440F551F481B590BDA01A95AB34F64
:10BB00008C91882309F47FC1FD018181882309F488
:10BB10007AC18281882309F476C1FA01E65AF34F8B
:10BB2000E0818E2F837009F084C0112309F43EC098
:10BB30000023E1F18E2F86958695837061F46F2D39
:10BB4000822F0E94A357FF2019F081E090E02BC2C2
:10BB500080E090E028C28981282F3327C901880F0F
:10BB6000991F880F991F880F991F821B930BFC0147
:10BB7000E65AF34F8081869586958370823079F4FA
:10BB800060E01F1509F461E089810E94A3571F1529
:10BB900019F481E090E007C280E090E004C261E027
:10BBA00089810E94A35781E090E0FDC14981242F43
:10BBB0003327C901880F991F880F991F880F991F74
:10BBC000821B930BFC01E65AF34F80818695869584
:10BBD0008370823049F4FF2039F461E0842F0E94A1
:10BBE000A35781E090E0DFC14981242F3327C901A9
:10BBF000880F991F880F991F880F991F821B930B1D
:10BC0000FC01E65AF34F808186958695682F637014
:10BC1000613041F4FF2031F0842F0E94A35781E06E
:10BC200090E0C1C160E089810E94A35780E090E06C
:10BC3000BAC14981242F3327C901880F991F880F62
:10BC4000991F880F991F821B930BFC01E65AF34F33
:10BC5000E0818E2F8370823009F045C01017E1F526
:10BC60008E2F86958695837061F46F2D842F0E94A8
:10BC7000A357FF2019F081E090E095C180E090E0AB
:10BC800092C18981282F3327C901880F991F880FF6
:10BC9000991F880F991F821B930BFC01E65AF34FE3
:10BCA0008081869586958370823079F460E01F15D7
:10BCB00009F461E089810E94A3571F1519F481E0FE
:10BCC00090E071C180E090E06EC161E089810E94E6
:10BCD000A35781E090E067C160E089810E94A3578B
:10BCE00080E090E060C1112319F4002309F448C0FA
:10BCF0004981242F3327C901880F991F880F991F65
:10BD0000880F991F821B930BFC01E65AF34F808129
:10BD100086958695837061F46F2D842F0E94A357BA
:10BD2000FF2019F081E090E03EC180E090E03BC14F
:10BD30004981242F3327C901880F991F880F991F24
:10BD4000880F991F821B930BFC01E65AF34F8081E9
:10BD5000869586958370823061F46F2D842F0E94C2
:10BD6000A357FF2019F081E090E01DC180E090E032
:10BD70001AC161E089810E94A35781E090E013C15C
:10BD80004981242F3327C901880F991F880F991FD4
:10BD9000880F991F821B930BFC01E65AF34F808199
:10BDA00086958695682F6370613041F4FF2021F1FC
:10BDB000842F0E94A35781E090E0F5C04981242F91
:10BDC0003327C901880F991F880F991F880F991F62
:10BDD000821B930BFC01E65AF34F80818695869572
:10BDE0008370823049F4FF2039F461E0842F0E948F
:10BDF000A35781E090E0D7C060E089810E94A357FB
:10BE000080E090E0D0C02981822F9927AC01440FB7
:10BE1000551F440F551F440F551F481B590BDA017E
:10BE2000A95AB34F8C91882309F452C0FD01818136
:10BE3000882309F44DC0FA01E65AF34F80818370DC
:10BE400091F4112349F0002339F061E0822F0E9420
:10BE5000A35781E090E0A7C060E089810E94A357CA
:10BE600080E090E0A0C04981242F3327C901880FCA
:10BE7000991F880F991F880F991F821B930BFC0134
:10BE8000E65AF34F80818370823081F4101739F4C1
:10BE900061E0842F0E94A35781E090E084C060E0BD
:10BEA00089810E94A35780E090E07DC0112311F4A6
:10BEB000002339F061E089810E94A35781E090E07E
:10BEC00072C060E089810E94A35780E090E06BC05F
:10BED0002981822F9927AC01440F551F440F551F0C
:10BEE000440F551F481B590BDA01A95AB34FFD01E6
:10BEF0008181882309F455C08281882309F451C0C7
:10BF0000FA01E65AF34F808186958695837091F405
:10BF1000112349F0002339F061E0822F0E94A357DA
:10BF200081E090E040C060E089810E94A35780E0FA
:10BF300090E039C04981242F3327C901880F991F08
:10BF4000880F991F880F991F821B930BFC01E65ADB
:10BF5000F34F8081869586958370823081F4101727
:10BF600039F461E0842F0E94A35781E090E01BC068
:10BF700060E089810E94A35780E090E014C0112303
:10BF800011F4002339F061E089810E94A35781E018
:10BF900090E009C060E089810E94A35780E090E0B2
:10BFA00002C080E090E021960FB6F894DEBF0FBE8D
:10BFB000CDBFDF91CF911F910F91FF900895CF9347
:10BFC000DF93CDB7DEB721970FB6F894DEBF0FBE73
:10BFD000CDBF282F04B603FE28C0FE013196ACEB7E
:10BFE000B0E081E090E031E08030930719F40E94E6
:10BFF0004F6603C0182E0E944F668981843190F4E9
:10C000008F5F8983FE013196ACEBB0E081E090E078
:10C0100031E08030930719F40E94606603C0182E47
:10C020000E94606684B7877F84BF809160008861CA
:10C03000809360002093600080916000886080930E
:10C04000600021960FB6F894DEBF0FBECDBFDF9122
:10C05000CF910895EF92FF920F931F937B018C0174
:10C0600020E030E040E05FE40E948E6288239CF094
:10C0700020E030E040E05FECC801B7010E94786149
:10C08000DC01CB01BC01CD010E94286360507040EF
:10C090008040904804C0C801B7010E9428631F91E6
:10C0A0000F91FF90EF900895A0E0B0E0EAE5F0E690
:10C0B0000C9410668C017B015A01DC018C9182305A
:10C0C00058F0FB019081923010F4A7010BC184302D
:10C0D00029F4943009F4A6C0A80104C19430A9F34E
:10C0E000923009F4A9C0823081F3F801C280D38074
:10C0F000FB0162817381F80124813581468157817A
:10C10000F7016480758086809780C601861B970B37
:10C1100097FDD8C080970CF46CC06C157D050CF0B1
:10C12000ADC0662477244301F8016181F701818164
:10C13000681709F499C0662309F491C0621A730A5A
:10C14000840A950AA401930157FDC0C0F50111822C
:10C15000B60119012A0179018A0139014A010894BD
:10C160006108710881089108FFEF6F16FFEF7F06E5
:10C17000FFEF8F06FFE39F06F0F4A8019701220F5F
:10C18000331F441F551F19012A01B6016150704029
:10C190006B0179018A0139014A010894610871082B
:10C1A000810891088FEF68168FEF78068FEF880669
:10C1B0008FE3980610F383E0D5018C9357FC64C09D
:10C1C000F501248335834683578373836283A501F6
:10C1D00089C06F5F7F4FD401C30181709070A070E0
:10C1E000B0709694879477946794682A792A8A2AFB
:10C1F0009B2A6C157D056CF311C00894C11CD11CE1
:10C20000DA01C90181709070A070B07056954795A1
:10C2100037952795282B392B4A2B5B2BC616D7062B
:10C2200064F382CFF8019181FB018181981709F4B1
:10C2300053CF41EA51E056C0823009F04DCF88E03B
:10C24000DA01F80101900D928A95E1F7F8018181F8
:10C25000FB0191818923FA018183A50143C026193D
:10C2600037094809590970CFF5016183B601260DD8
:10C27000371D481D591D19012A019DCF6B0120E072
:10C2800030E040E050E050CFD201C101B695A79513
:10C290009795879521E030E040E050E0222233225C
:10C2A00044225522282A392A4A2A5B2AF501248267
:10C2B0003582468257820894C11CD11CD382C28227
:10C2C000A50110C0909581959F4F24CF81E0F50185
:10C2D0008183B60150954095309521953F4F4F4F42
:10C2E0005F4F37CFCA01E2E1CDB7DEB70C942C66C1
:10C2F000A0E2B0E0EEE7F1E60C941E66DC01CB01B3
:10C30000898F9A8FAB8FBC8F2D8F3E8F4F8F58A305
:10C31000BE016F5F7F4FCE0149960E9462648E011D
:10C32000075F1F4FB801CE014D960E946264AE01B7
:10C330004F5E5F4FB801CE0101960E9454600E948B
:10C340007A63DC01CB01BC01CD01E4E0A0960C9442
:10C350003A66A0E2B0E0EFEAF1E60C941E66DC017A
:10C36000CB01898F9A8FAB8FBC8F2D8F3E8F4F8FD4
:10C3700058A3BE016F5F7F4FCE0149960E94626451
:10C380008E01075F1F4FB801CE014D960E94626477
:10C390008A8591E089278A87AE014F5E5F4FB80199
:10C3A000CE0101960E9454600E947A63DC01CB01A9
:10C3B000BC01CD01E4E0A0960C943A66A8E1B0E09F
:10C3C000E4EEF1E60C941866DC01CB01898B9A8BC4
:10C3D000AB8BBC8B2D8B3E8B4F8B588FBE016F5F11
:10C3E0007F4FCE0141960E9462648E01075F1F4F0E
:10C3F000B801CE0145960E946264FE013196298102
:10C40000223008F45FC03985323010F4B8017BC0A7
:10C4100081819A8589278183243009F455C022308F
:10C4200009F452C0343009F454C0323009F458C011
:10C430006B817C818B859C85681B790B2D813E816E
:10C440004F815885ED84FE840F8518892E153F0590
:10C450004007510730F4220F331F441F551F61500E
:10C4600070407C836B8380E090E0A0E0B0E4AA247D
:10C47000BB2465012E153F054007510740F0A82A4F
:10C48000B92ACA2ADB2A2E193F09400B510BB6954F
:10C49000A79597958795220F331F441F551F009727
:10C4A000A105B10539F7D601C5018F779070A0704D
:10C4B000B07080349105A105B105A9F0A482B582C0
:10C4C000C682D782BF011FC02317E1F761EA71E07E
:10C4D0001AC01D821E821F8218861C821B82F2CF08
:10C4E00084E08983EFCFA7FC05C021153105410504
:10C4F000510521F380E490E0A0E0B0E0A80EB91E61
:10C50000CA1EDB1EDBCFCB010E947A63DC01CB01AC
:10C51000BC01CD01EAE068960C943466A8E1B0E075
:10C52000E4E9F2E60C941E66DC01CB01898B9A8B60
:10C53000AB8BBC8B2D8B3E8B4F8B588FBE016F5FAF
:10C540007F4FCE0141960E9462648E01075F1F4FAC
:10C55000B801CE0145960E9462648981823018F04C
:10C560008985823018F42FEF3FEF09C0B801CE0162
:10C5700001960E94DC64282F332727FD3095C901DE
:10C58000E4E068960C943A66A8E0B0E0EAECF2E6E3
:10C590000C941C669B01AC017B018C01EE2417FD01
:10C5A000E394FF2400271127EA8221153105410574
:10C5B000510539F482E08983CE0101960E947A63A5
:10C5C00043C083E089836EE170E0CB01EE2031F55A
:10C5D00079018A01A80197012030E0E03E07E0E000
:10C5E0004E07E0E45E0798F479018A01EE0CFF1C27
:10C5F000001F111F0197BC01A8019701E0E0EE1692
:10C60000E0E0FE06E0E00E07E0E41E0768F3ED82DE
:10C61000FE820F8318877C836B83CECF2030E0E0CF
:10C620003E07E0E04E07E0E85E0741F0EE24FF241D
:10C630008701E21AF30A040B150BCCCF7C836B83C2
:10C6400060E070E080E09FECE6E028960C943866AD
:10C65000ACE0B0E0EEE2F3E60C942066DC01CB0146
:10C6600089879A87AB87BC87BE016F5F7F4FCE01FA
:10C6700009960E9462648981823011F0823028F428
:10C6800060E070E080E090E031C0843039F02B81D0
:10C690003C8137FDF5CF2F3131056CF08A8188233D
:10C6A00029F060E070E080E090E820C06FEF7FEF5D
:10C6B0008FEF9FE71BC08EE190E0821B930B2D81D3
:10C6C0003E814F81588504C05695479537952795EB
:10C6D0008A95D2F78A81882339F050954095309514
:10C6E00021953F4F4F4F5F4FCA01B901E2E02C96B1
:10C6F0000C943C66A0E0B0E0E0E8F3E60C9416662B
:10C70000882499245401DC01FC012481358146816F
:10C7100057818181082F112760E070E08C91823071
:10C7200020F46FEF70E04061A4C0843009F464C06D
:10C73000823009F463C0211531054105510509F422
:10C7400098C0FD0182819381FFEF82389F070CF032
:10C7500050C0A2E8EA2EAFEFFA2EE81AF90A8AE1F1
:10C76000E816F1040CF06BC06B0181E090E0A0E0F2
:10C77000B0E00E2C04C0880F991FAA1FBB1F0A949B
:10C78000D2F70197A109B10982239323A423B523EA
:10C790000097A105B10519F0F1E0CF2ED12C04C00E
:10C7A0005695479537952795EA94D2F7C601AA275B
:10C7B00097FDA095BA2F282B392B4A2B5B2BDA013A
:10C7C000C9018F779070A070B07080349105A10579
:10C7D000B105D1F1215C3F4F4F4F5F4F2030E0E07A
:10C7E0003E07E0E04E07E0E45E0708F161E070E03C
:10C7F0001EC0803891053CF06FEF70E020E030E023
:10C8000040E050E036C0BC0161587F4FDA01C901F9
:10C810008F779070A070B07080349105A105B1053C
:10C82000D1F0215C3F4F4F4F5F4F57FD1BC097E04A
:10C8300056954795379527959A95D1F71AC020E0D8
:10C8400030E040E050E0BBCF27FFC8CF205C3F4F37
:10C850004F4F5F4FC3CF27FFE8CF205C3F4F4F4F75
:10C860005F4FE3CF56954795379527956F5F7F4F7D
:10C87000DECF822E932E942F9F778A2D8078A82E3C
:10C88000A92A962F9795992797958A2D8F77A82E65
:10C89000A92A76956795962F9F778B2D8078B82E4D
:10C8A000B92A902F9795992797958B2D8F77B82E2A
:10C8B000B92AD501C401BC01CD01ECE0CDB7DEB78A
:10C8C0000C943266CF93DF93FC01DB0140815181F0
:10C8D0002281622F6F7770E0221F2227221F93810F
:10C8E000892F880F822B282F3327991F9927991F6B
:10C8F000ED0199832115310541F44115510561057B
:10C900007105E1F482E08C9354C02F3F310509F4A6
:10C9100041C02F573040FD013383228383E08C9345
:10C9200087E0440F551F661F771F8A95D1F7706403
:10C93000ED014C835D836E837F833BC022E83FEF34
:10C94000F901C7E0440F551F661F771FCA95D1F73D
:10C9500083E08C93403080E0580780E0680780E4F3
:10C96000780778F4440F551F661F771F2150304019
:10C97000F9014030C0E05C07C0E06C07C0E47C0710
:10C9800088F3ED01FB83EA83FD01448355836683CD
:10C9900077830FC0411551056105710519F484E0D5
:10C9A0008C9307C064FF03C081E08C93C1CF1C92BD
:10C9B000BFCFDF91CF9108950F931F93CF93DF9354
:10C9C000FC01DB018081823018F09C91923018F4D8
:10C9D00061E070E05EC08430C1F0843001F19430D9
:10C9E00009F447C0823009F44BC0823009F44EC0CC
:10C9F0009230A9F04181ED0189814817B9F04423B3
:10CA000089F08FEF9FEFBC0144C0943031F7EB0108
:10CA10008981682F77278181681B71093AC08181DC
:10CA2000882379F781E090E0BC0133C02281338113
:10CA3000ED018A819B81821793070CF32817390730
:10CA40009CF00481158126813781FD016481758107
:10CA500086819781601771078207930780F2061716
:10CA600017072807390778F4442359F281E090E04A
:10CA7000DBCFFD018181882321F281E090E0D4CFDA
:10CA8000923009F0B2CF60E070E003C0ED0189811F
:10CA9000F2CFCB01DF91CF911F910F910895FB0150
:10CAA000DC0105900D920020E1F70895FB01DC0107
:10CAB00004C08D910190801921F441505040C8F775
:10CAC000881B990B0895FB01DC0140FF05C002C0E3
:10CAD00001900D9201900D9242505040C8F7089578
:10CAE000DC0140FF03C001C06D936D934250504084
:10CAF000D8F70895FB01DC0101900D920020E1F7C9
:10CB00000895629FD001739FF001829FE00DF11D97
:10CB1000649FE00DF11D929FF00D839FF00D749FB7
:10CB2000F00D659FF00D9927729FB00DE11DF91F63
:10CB3000639FB00DE11DF91FBD01CF0111240895C0
:10CB4000991B79E004C0991F961708F0961B881F5F
:10CB50007A95C9F780950895AA1BBB1B51E107C0C0
:10CB6000AA1FBB1FA617B70710F0A61BB70B881F7D
:10CB7000991F5A95A9F780959095BC01CD0108950C
:10CB800097FB092E07260AD077FD04D0E5DF06D0F3
:10CB900000201AF4709561957F4F0895F6F79095EF
:10CBA00081959F4F0895A1E21A2EAA1BBB1BFD0180
:10CBB0000DC0AA1FBB1FEE1FFF1FA217B307E4077C
:10CBC000F50720F0A21BB30BE40BF50B661F771FD4
:10CBD000881F991F1A9469F76095709580959095B4
:10CBE0009B01AC01BD01CF01089597FB092E0526DD
:10CBF0000ED057FD04D0D7DF0AD0001C38F4509572
:10CC00004095309521953F4F4F4F5F4F0895F6F770
:10CC100090958095709561957F4F8F4F9F4F0895A8
:10CC20002F923F924F925F926F927F928F929F923C
:10CC3000AF92BF92CF92DF92EF92FF920F931F932A
:10CC4000CF93DF93CDB7DEB7CA1BDB0B0FB6F894DB
:10CC5000DEBF0FBECDBF09942A88398848885F841B
:10CC60006E847D848C849B84AA84B984C884DF808C
:10CC7000EE80FD800C811B81AA81B981CE0FD11D70
:10CC80000FB6F894DEBF0FBECDBFED010895F99940
:10CC9000FECFB2BDA1BDF89A119600B40895F7DF9A
:10CCA00001921A94E1F70895F999FECFB2BDA1BDA2
:10CCB00000BC11960FB6F894FA9AF99A0FBE08952F
:0ACCC0000190F2DF1A94E1F70895E5
:10CCCA00012E2E2F63616E5F696E7075742E63007C
:10CCDA006E222E2E2F6368616E6E656C732E630052
:10CCEA0053657175656E63652023310053657175EF
:10CCFA00656E63652023320053657175656E6365E1
:10CD0A002023330053657175656E636520233400F3
:10CD1A00455233002E2E2F656570726F6D63686100
:10CD2A006E6E656C732E630050434D30004552336E
:10CD3A00004C4F4730340050434D207665722039FD
:10CD4A002E3136004F425220383434300B002E2E0A
:10CD5A002F7669727475656C5F696E7075742E636F
:0ACD6A0000000000000000000000BF
:00000001FF
